:040000000C94BB0C95
:100004000C9400000C9400000C9400000C9400006C
:100014000C9400000C9400000C9455610C940000A6
:100024000C9400000C94A6140C9400000C94000092
:100034000C9400000C9400000C9400000C945814D0
:100044000C9400000C94075E0C9400000C94435E26
:100054000C9400000C9400000C9400000C9400001C
:100064000C9400000C9400000C9400000C9400000C
:100074000C9400000C94B05F0C9400000C94F3609A
:100084000C9400000C940000000001000200040025
:10009400080010002000400080000001000200045D
:1000A4000008001000200040008000010204081035
:1000B40020408000B803C20B80100000BC03C20BB8
:1000C400821F0000C603C20B81030000CE03C20BD3
:1000D40001040300D803C30B01060500E203C50BAA
:1000E40001800000EE03CC0B020F0000F603C60BE8
:1000F400020F0000FE03C80B020FD0120604CA0B45
:100104000110000010041A0C011000001A04CB0B9B
:10011400000100002204CE0B010801002C04CF0BC7
:10012400030801003A04D00B030700004204E60B65
:10013400017F3F004C04E50B010500005604D10B80
:10014400030400005E04E40B01641E006A04D20B85
:10015400000100007604D30B000100008204E30BCD
:10016400010200008E04D40B000100009C04D50B96
:10017400020F0000A804D70B020FE703B204190C06
:100184000163000010051B0C011000001A051C0C73
:1001940001020200BE04D90B03080100C404DA0BF7
:1001A40003080000CA04DB0B03080000D004DC0BC6
:1001B40003080000D604DD0B03080000DC04DE0B9A
:1001C40003080000E204DF0B03080000E804E70B67
:1001D400040A2E00F004F10B040A2E00F804FB0BB1
:1001E400040A2E000005050C040A2E0008050F0C55
:1001F400040A2E0000000000FF0000002205000297
:100204002A0504043005080736050C0536058C0656
:100214003C0580094405100B4C05500C5605400361
:100224005E05140A6805180870051C010000000228
:10023400280060009800D00008014001210C5800FB
:100244002D0B2D002B0B2B004D0A4D00808182833A
:100254008400002188898A8B8C8D8E8F310B31200C
:1002640041424300320B322044454600330B3320D5
:10027400474849004D0A4D0000000000340B34206B
:100284004A4B4C00350B35204D4E4F00360B362073
:10029400505152002B0A2B0000000000370B37206E
:1002A40053545500380B382056575800390B392011
:1002B400595A2F002D0A2D0000000000430C430062
:1002C40000000000300B3020202E2C002C0A2C00C3
:1002D400000000003D0A43520000000000004A01F3
:1002E400460032002100004B004A01460032004D16
:1002F400000096004A0146003200540000E1004A22
:1003040001460032003D0000F000000032005000C1
:100314002D0000F000500032005000470000F000B3
:10032400A000320050004B0000F000F000320050FA
:10033400002B00005800B4000400380038002138B5
:1003440003006A6100008700C800640032003D4673
:1003540003006E65696E00000800C8006400320086
:10036400215603004B004A01460032004D000000B4
:1003740001000100E60063004D0000000000A00041
:100384001B00007105D700A0001A02007105690066
:100394000000180400730569001E011906007305A6
:1003A40050726F64756B74200000537061727465D1
:1003B400202000005F4944005F52733233324944C5
:1003C40000005F526F74617465005F5461737465FB
:1003D4006E5800005F54617374656E5900005F4489
:1003E400656661756C744B6579002A436F6465308A
:1003F40000002A436F64653100002A436F6465324C
:1004040000002A4D61784D6F64756C005F4572770A
:100414004D6F64756C002A546973636845005F4DC1
:10042400795465726D4E72005F4D617374657254D8
:1004340065726D7300005F454D6F646500005F4534
:1004440043726564577472005F5273304D6F646514
:1004540000005F5634756E6435005F50756C7365CB
:1004640054696D6500005F41736B43726564697420
:1004740000005F53656E64446562697400005F4305
:1004840072656469744D6F6465005F437265646985
:10049400744D6173746572002A5461626C6553749F
:1004A400617274002A5461626C65456E64002A4668
:1004B40069727374426F6E5000002A4A6F62310091
:1004C4002A4A6F6232002A4A6F6233002A4A6F62F4
:1004D40034002A4A6F6235002A4A6F6236002A4A7B
:1004E4006F6237005F4572726F7231005F457272DE
:1004F4006F7232005F4572726F7233005F457272C1
:100504006F7234005F4572726F7235005F467265B8
:100514006967616265005F4B6F6D6D6100005461D6
:100524007374657200004C69745A00004C656974F8
:10053400540050756C7300005461737420300000D3
:1005440073657269656C6C0073657269656C2032E1
:10055400000054617374203200005461737420707D
:1005640061720000466F6C676554000053776974CC
:1005740063680000706F7274696F6E696572656E8E
:1005840000002E666F6C67650000506F7274696FAF
:100594006E656E207369636865726E004368656694
:1005A4002D4D656E75004B206C697374656E00008B
:1005B4004B206C6F65736368656E00004B2064723A
:1005C40075636B656E0054206C697374656E00000E
:1005D40054206C6F65736368656E00005420647208
:1005E40075636B656E0053797374656D0000506FAD
:1005F4007274696F6E004B726564697465004B7246
:1006040065642E436C7200006D616E2E506F7274BF
:10061400696F6E00546573740000506172616D659A
:100624007465720050726F64756B746500004B657D
:100634006C6C6E65720056656E74696C650030A0F2
:100644000531AA0532B40533C00534CA0535D405CD
:1006540036E00546EA0541F20543FA054402064A36
:100664000C060000000030EA05371806391E06386B
:100674002806423206453A06000000004572726FB1
:1006840072004F70742E0000496D70756C73000019
:1006940054696D656F7574008006300C00050000A8
:1006A4008606330C000300008C06310C00050000A4
:1006B4009406320C001400002E202C3041424331A9
:1006C40044454632474849334A4B4C344D4E4F35E6
:1006D400505152365354553756575838595A2F3962
:1006E4000500C11100000300D90B00000300C11173
:1006F4000300170E0300D90B00000500E0080000FA
:100704000A00C1110A00170E0A00D90B0A00C11110
:100714000A00170E2800D90B00000000000000009A
:1007240000000000000000000000000000000000C5
:100734000000070C182022204D994D40114048918B
:100744004720222018C007000000070C1F3FEE3F7F
:100754007277727FFF7F777F783FEE3F1FC007007D
:100764000000000000000C183DEE3F3FEE3F1FC8A4
:100774000F0700020000000000000000000000025B
:1007840007080F1FCE3F1FC80F070002000000001C
:10079400000000000007080F0F880F376F7F7FFFEE
:1007A4007F3260070F80000000000000000200029A
:1007B40007080F1FCE3F3FEE3F1AC0070F8000000F
:1007C400000000000000000000000006000F0F0001
:1007D40006000000000000000000FFFFFFFFFFFF15
:1007E400FFFFFFF9FFF0F0FFF9FFFFFFFFFFFFFF3F
:1007F400FFFF0000000000000600091088101088A8
:1008040010090006000000000000FFFFFFFFFFFFCB
:10081400F9FFF6EF77EFEF77EFF6FFF9FFFFFFFF52
:10082400FFFF000000000E01006A1E33286161888A
:100834006133001E000000000000000000078C0C63
:10084400186618186C0C078003030C0F03000300D0
:100854000000020003038C0302CC020280020200A7
:100864000E1E001E0C00000000000C000E0B0809F8
:100874000CC40E0B4C0938C478784C3103CC0301FA
:1008840080000000020202271FCC18306770306C11
:10089400181FC22702000200000000000010001808
:1008A4001C001E1F081F1F001E1C00181000000043
:1008B40000000000000088010388070F881F0F88CC
:1008C4000703880100800000000000000207080FF1
:1008D4001FC0020200020200021FC80F070002002C
:1008E4000000000819198819198819198819198814
:1008F40019198000198819000000000E1F36CC66F3
:1009040066CC6636CC1E06CC0606CC0606CC0600A3
:10091400000000081F30C03030081F30CC301F8C5E
:100924000000CC301F800000000000000000000028
:10093400000000000000000000000E1F1FEE1F005A
:1009440000000200070F8C1F0200020200020200D6
:10095400021FC80F0700021FC00000000207080F93
:100964001FC0020200020200020200020200020092
:100974000000000002020002020002020002020063
:10098400021FC80F07000200000000000000000062
:1009940001080101CE3F01C8010100000000000070
:1009A400000000000000000004000C1C0E3F1C00AE
:1009B4000C04000000000000000000000000000023
:1009C400000000000000400040400040400E7F0056
:1009D4000000000000000000088C1838EF7F38EC9D
:1009E4001808800000000000000000000000000063
:1009F40000000207080F1FCE3F7FF0000000000038
:100A04000000000000000000000F7F3FEC1F0F807B
:100A140007020000000000000000000000000000C9
:100A240000000000000000000000000000000000C2
:100A340000000600060F000F0F000F0F000606004F
:100A440006000000060006000000000000198819D6
:100A540019881900000000000000000000000000D8
:100A640000000006060666063FFC0C0CC819198C2B
:100A74007F3300333300000000000600061F8C3F64
:100A84003600363F8C1F06CC063FC81F0600060002
:100A94000000000000001338387E3801C803070046
:100AA4000E1C0E3870EE600000000000070D88195F
:100AB40019801B0E001E3E063333C8313BC61E0090
:100AC40000000E000E0E000606000C0000000000E0
:100AD400000000000000000000000380060E000C6F
:100AE4001C001C1C001C1C001C0C000E060803002F
:100AF40000001C000607000303880303880303881F
:100B04000303000706001C000000000000000C3670
:100B140036C81F0F0C3F0F081F36CC3600000000EC
:100B24000000000000000000060006060C3F3FC065
:100B3400060600060000000000000000000000009F
:100B440000000000000000000000000E0E000E0671
:100B5400000C000000000000000000000C3F3FC03B
:100B64000000000000000000000000000000000081
:100B740000000000000000000000000E0E000E0047
:100B8400000000010000370000EC010380070E00A4
:100B94001C3800706000000000000F8E3F3067605A
:100BA40060FB616333666C33787036303FE80F0066
:100BB40000000300071F001F0300030300030300DA
:100BC400030300031FEE1F0000001FCE3F7073607D
:100BD400607E0001C80307000E1C00387FFF7F0001
:100BE40000001FCE3F7073600037000FEC0F0063EE
:100BF400006037703FEC1F00000001CC0307CC0EEF
:100C04001CCC3870CC607FFF7F00CC0000CC00008F
:100C140000007FFF7F600060600C7F3FE7000033CF
:100C2400006037703FEC1F00000003CC070E001C6F
:100C34003800307FCE7F7073606037703FEC1F00E8
:100C440000007FFF7F00660000CC000188010300E4
:100C5400030600060C000C0000000F8C1F38E63061
:100C6400306E381FCE3F7073606037703FEC1F00EA
:100C740000001FCE3F7073606037703FFF1F006E2F
:100C84000001C8031F001E00000000000000000057
:100C94000E000E0E00000000000E000E0E000000FC
:100CA40000000000000000000E000E0E0000000016
:100CB400000E000E0E000606000C00CC0103800797
:100CC4000E001C3800381C000E07080301CC00007D
:100CD4000000000000000000000E3F3FE000000E96
:100CE4003F3FE0000000000000003000381C000E10
:100CF40007080301CC010380070E001C38003000F4
:100D040000001F8C3F70E66060EC01038007060062
:100D1400060600000600060000001FCE3F306B6789
:100D24006FBB6D6DBB6D6DBE6F67C0703FCC0F0048
:100D340000000600060F000F0F081919881930CC9F
:100D44003F3FC6606066600000007F087F61CC6042
:100D540060CC617F8C7F60E660606E607FC87F00DE
:100D640000000F8C1F38E630600060600060600097
:100D740060306E381FC80F0000007F087F61CC60B0
:100D840060666060666060666060CC617F807F00E2
:100D940000007FEE7F6000606000607F887F6000FD
:100DA400606000607FEE7F0000007FEE7F60006087
:100DB4006000607F887F60006060006060006000A9
:100DC40000000FCE1F38603060006063EE63606621
:100DD400603066381FEE0F00000060666060666079
:100DE4006066607FEE7F606660606660606660007B
:100DF40000001F881F0600060600060600060600FF
:100E0400060600061F881F0000000066000066003A
:100E1400006600006600006660606C703FC81F00DA
:100E24000000606E6061C86367006E7C007C6E00C9
:100E340067638C6160E660000000600060600060D1
:100E44006000606000606000606000607FEE7F00B2
:100E54000000606E7070EE7979E66F6F66666666A4
:100E6400606066606066600000006066707066784E
:100E74006C666C66666663666361EE6060E660007D
:100E840000000F081F39CC306066606066606066E1
:100E94006030CC391F800F0000007F8C7F60E660DB
:100EA40060666060EC7F7F8060600060600060006E
:100EB40000000F081F39CC306066606066606066B1
:100EC4006333CC391FE60F0000007F8C7F60E6603F
:100ED40060666060EC7F7F8067638C6160E66000C1
:100EE40000001F8C3F70E6606000703F8C1F00E6BE
:100EF40000606E703FC81F0000003FCC3F06000634
:100F040006000606000606000606000606000600A1
:100F1400000060666060666060666060666060666F
:100F240060606C303FC81F000000606660606C3019
:100F340030CC3019881919800F0F000F06000600F5
:100F44000000606660606660606660606666666633
:100F54006F79EE7070E66000000060666030CC303F
:100F640019800F0600060F081930CC306066600047
:100F7400000060666030CC301988190F000F06003D
:100F8400060600060600060000007FEE7F00CC0087
:100F94000180030600060C00183000307FEE7F004D
:100FA40000001F881F1800181800181800181800CF
:100FB400181800181F881F0000000000406000700F
:100FC40038001C0E0007038C0100E700003000000D
:100FD40000001F881F018801018801018801018820
:100FE400010188011F881F0000000200070F8C1DEB
:100FF40038E77060300000000000000000000000CE
:1010040000000000000000000000000000000000DC
:10101400000000000000007FFF7F000007070007BA
:1010240006000603000000000000000000000000AD
:101034000000000000000000000C1F3FE6001FEE4F
:101044003F6066607FEE3F0000006000606000600B
:1010540060086F7FCE70606660606E607FC87F00DE
:10106400000000000000000000081F3FC670600080
:10107400606006703FC81F00000000660000660044
:1010840000661F3FEE716066606066703FEE1F0091
:10109400000000000000000000081F3FC6707FEC45
:1010A4007F6000703FC81F00000007880F1C0018F5
:1010B4001800187F007F180018180018180018006E
:1010C4000000000000000000000E1F3FE670606E8C
:1010D400703FE61F006E003FC83F60006060006024
:1010E40060006F7F8C7160CC6060CC6060CC60000D
:1010F400000000000006000600000E0E00060600B8
:10110400060600061F881F00000000000001880179
:101114000008030388010188010188010188191F5F
:10112400800F3000303000303008313380373E00DB
:101134003E37083331CC300000000E000E060006A6
:101144000600060600060600060600061F881F00A5
:1011540000000000000000000008597FCE7F666692
:1011640066666666666666000000000000000000B1
:1011740000083F3FCE303066303066303066300095
:10118400000000000000000000081F3FCE706066F1
:1011940060606E703FC81F00000000000000000087
:1011A40000087F7FCE6060666070EC7F6F80606057
:1011B4000060000000000000000E1F3FE670606643
:1011C4006070EE3F1F660000660000000000000033
:1011D400000C373FE638300030300030300030004B
:1011E400000000000000000000003F7F80607F08D6
:1011F4003F0188017F803F0000000000181800189C
:1012040018007F7F00181800181800181F880F0096
:101214000000000000000000000660606660606678
:1012240060606E703FE61F000000000000000000D8
:10123400000660606C3030C81919800F0F0006007A
:101244000000000000000000000666666666666630
:10125400666F6C3F39C810000000000000000000F9
:10126400000C6071C83B1F000E1F083B71CC60006E
:101274000000000000000000000C3030C819198084
:101284000F0F000606000C0C001800000000000000
:10129400000C7F7F800306000C1800307FCC7F0099
:1012A400000003CC070E000C0C000C1C00381C00C2
:1012B4000C0C000C0E0C0703C0000600060600060A
:1012C40006000600000606000606000606000600E4
:1012D40000003C003E070003030003038C0103806D
:1012E4000303000307003E3C00000000001C6C36B2
:1012F4006380000000000000000000000000000007
:10130400000000000000000006000F198C30606629
:10131400607FEE7F00000000000000001E006007F8
:101324007E0700F01EF060F77EF7FBDE1F00E0078B
:10133400FF0700F81FF8E0FFFFFF00000F00E002C6
:10134400EF0200780F78E07AEF7AF7BD1F00E0072C
:10135400FF0700F81FF8E0FFFFFF23000002000072
:10136400100000050000FE0500182800FE04001807
:101374002400F90F00F80F0070001F7180237280A1
:101384002A73111574111C75151B76151A77181C00
:10139400781521050100FF000000013F2B02001019
:1013A400072100000100072300100000FD300007A2
:1013B4003300113068FF0000E500800001000100E7
:1013C40001020004033010040000080202090000B6
:1013D4000A00000C00000D00000F000010000011B6
:1013E4000700120000130000FD500010B01B11078D
:1013F40000FD5000121E01FD500013001F291F00A4
:10140400FD5000200000210000FE01002B0C00FE16
:1014140000002B20003000003106033200023507A3
:10142400013604043706063805013907073C00066F
:101434003D070850000051EF00520000533F01FEE9
:1014440001006000A7FE00006000276101006A003F
:1014540000800000810000820000830000840000FE
:10146400850000901000920007930700953F0397B2
:101474000000980000070100FD5000072100072329
:1014840000FD5000077301FF000000000000000091
:10149400F8000000FF000000FF0000007F80001E35
:1014A4000F80007FE7C0007FFFE0003FFFE0000700
:1014B400FFC00001FFC00001FF800001FF0003FF27
:1014C400FE0007FFFC0007FFF00003FFF00003FF2E
:1014D400FE00001FFFC001FFFFF001FFFFF801FF46
:1014E400FFF8007FFFF80007FE00003FFF00007FC9
:1014F400FF80007FFF80007FC100001FE000001F0D
:10150400F000001FF000000FE0000007C00000071B
:10151400C0000007C00000078000000300000003B3
:1015240000000002000000000000000000000000B5
:10153400E000000000000003900000000000000E26
:10154400180000000000003808000000000000C07F
:1015540018000000000003807000000000000C016F
:10156400C00000018006300700000003C00F401CCB
:1015740000000006E01DC0700000000C3039C1C03E
:10158400000000181871C7180000001C0CE1DC7C76
:101594000000000E07C3F1C400000007038607061D
:1015A40000000003800E1C0200000001C01C300378
:1015B40000000000E03818010080000070700FC1C6
:1015C40083C0000038E003E08E6006001DC00020E8
:1015D400FC200F000F8000307030198007000010CD
:1015E400003030C00000001800E060600000000817
:1015F400038060300000000C0E003018000000046E
:101604003800180C00000006E0000C06000000037F
:1016140080000603000000000000030180000000B9
:1016240000000180C000C0C060C030C030C030C005
:1016340030C030C030C030C030C030C030E0307056
:101644003018300C30043FFC3FFC2564002B003E76
:101654003E006B65696E204B726564697400436F6C
:101664006C6F72546F75636820567320312E353455
:101674000049443D00202047433D00202036346B80
:10168400004B653A00496E3A0043616C69627261CD
:1016940074696F6E004F4B00546F74616C20002DA1
:1016A4002D2D2D0054696E79200054696E792062C5
:1016B400616400204C006B65696E20454570726F53
:1016C4006D004D4F44554C2053544F5000446174A9
:1016D400612000696E697400533F000066616C7399
:1016E4006368657220546973636820005469736386
:1016F4006820766F6E204B20004665686C6572200A
:101704000056656E74696C20616B74697600546967
:101714006D656F757400435349204E722000436F0A
:10172400646520006B65696E204B726564697400A2
:1017340066616C73636865722054697363680054EE
:101744006973636820766F6E204B005831393931E4
:10175400303000504C5520203A00436F6465203AE5
:10176400005469736368203A004D42005053004DA1
:1017740031004F310053500043500044590062750A
:101784007379004D50002067657370657272740040
:10179400256400004162726563686E756E67004B74
:1017A400656C6C6E65722000546F74616C004D6FD3
:1017B40064756C2000202000433F0073656300497A
:1017C4006D7000504C553A20005370617274653A44
:1017D40020005072313A20005072323A200046758F
:1017E4006E6374203A20005479703A20003A2056EF
:1017F4003A2020302B2030003A003A20544F3A202F
:10180400003A2050733A200053703A004B204D6F39
:101814006465204A6F62204A6F62466C6167730098
:101824004B20004D6F646520004A6F6220200056F3
:101834002020204572722050676C20496D7020541E
:101844004F005620005061757365004B656C6C6EDB
:1018540065723A004D49004D42004D43004D500021
:101864004D4C0074657374202E2E004F4E002530AD
:101874003258002530345800253664002533642E50
:101884002530326400253564002564002532640067
:1018940025336400444400004B230042530042219A
:1018A40000424600542300544F004952004D5A0050
:1018B40042510042520043530056530056430049DC
:1018C4004C00426600004B23005423004245004371
:1018D40045004241004453004342002350224153F7
:1018E4004349492D492F4F222C22312E3030222CAE
:1018F400323030382D30312D30313B0023482245F1
:10190400636F222C22312E3030222C323030382D8D
:1019140030312D30313B0023532245636F222C227A
:10192400312E3030222C323030382D30312D3031C0
:101934003B00504F00504632333B50550025640065
:101944002B302B303B0025640025303258002E30DC
:1019540030004F4E00006D696B726F746F75636871
:10196400000001002D4E414E00000100E10E6619F9
:101974000000F894EE27ECBBF1E0F5BFE5BFE0937F
:101984006C00F8E1F1BDE1BD8DE0A2E0BB27ED9371
:101994008A95E9F780E090E1A0E0B1E0ED9301974A
:1019A400E9F7EEE6F9E185919591009761F0A5914B
:1019B400B59105901590BF01F00105900D92019726
:1019C400E1F7FB01F0CFEFEFEDBFE0E1EEBFC0E0E8
:1019D400D3E00C941D160A9902C0E1E00895E0E0FA
:1019E4000895A0913E0CA13031F40E94376C0E94FE
:1019F40067670E94486C0895A0913E0CA13031F4B1
:101A04000E94376C0E94526C0E94486C0895E881D1
:101A1400E03011F01C9A01C01C9832C00E94566C30
:101A24000E94566C0E945B6CEFE3F0E00E94606CD5
:101A340008951A93A0910403A43081F4E0910F0453
:101A4400E093100410E0183048F4ABE01A9FF00162
:101A5400E052FD4F0E94666C1F5FF5CF3FC0A0911E
:101A64000403A43039F4E881E0931004E0E0E09347
:101A74000F0406C0E881E0930F04E0E0E093100453
:101A8400219608951A93A0910403A43019F110E04B
:101A9400143000F50E946A6C3196E491EA93DFDF1A
:101AA400E0E0E09310040E94736CEBE0F1E00E942C
:101AB4007D6C0E947D6CFA93EA930E946A6CE491B7
:101AC400EA930E946A6C32960E94826C0E94994347
:101AD4001F5FDECF0E94856C0E948A6C1991089565
:101AE4002A970E94CC7D30E010E000E047ED50E002
:101AF40028E0E0911A0CE03019F020E149E650E0CA
:101B0400321710F00C94C30D0E948E6CE13090F1EA
:101B14000E948E6CE03870F0EEE00E94946CEEE46B
:101B2400F6E1FA93EA930E948E6CEF70EF5F0E94E5
:101B34009C6C07C0ECE0EA9392DFE8E5EE83E0E01A
:101B4400EF830E94736CA02FB0E0E7E3F0E00E9403
:101B5400467BE40FF51F0E947D6CFA93EA93EDE255
:101B6400F0E0FA93EA930E948E6CEA930E94566C1A
:101B74000E94A66C1F5F143011F410E00F5F3F5FEA
:101B8400BFCF0E94856C0E9429490E94D37D619633
:101B940008950E94AC6CECE0EA9361DFEAE3F3E0C1
:101BA4000E94666CEBE0EA935ADF0E94B06C0E94DC
:101BB400B56CEAEAF0E00E94BA6CE0913B0CF0915B
:101BC4003C0CE491EA93E0913B0CF0913C0C31968F
:101BD4000E94C16C0E94994301E00E94C46C0E945F
:101BE400C76C11F00F5FF9CF0E94D56C031718F47E
:101BF400E0E0E093C0050E94D56C11E00E94DC6C2B
:101C04000E94C76C11F0153008F021C00E94B06C1E
:101C14000E94DF6CE0E4F0E00E94467B3496FA9385
:101C2400EA93E2EEF0E00E94BA6C0E94DC6C0E943F
:101C3400E26CE491EA930E94DC6C0E94E26C3196BF
:101C44000E94C16C0E9499433F5F1F5FD7CF0E94DF
:101C54008A6C0E94D57D34C427970E94CC7D22E3F0
:101C640054E0A0910403A43011F426E453E010E0FE
:101C7400143010F00C94890E00E0051710F00C9449
:101C8400870EE12FEE0FEE0FE00F3E2F0E94DC6C6B
:101C94000E94EE6C3196E4910E94946C0E94DC6C7C
:101CA4000E94EE6C3296FA93EA930E943669ED85AF
:101CB400E03039F4AF81A13210F4E0E0EF83E0E0EA
:101CC400E887A02FBB27E22FE85FF0E00E94467B65
:101CD4003896FA93EA930E94DF6CEAE3F0E00E94FC
:101CE400467BE55BFF4F0E94F36C0E947D6CFA9388
:101CF400EA930E94DC6C0E94EE6CE491EA930E94E9
:101D0400566C0E94A66C0F5FB8CF1F5FB1CF0E94C4
:101D14008A6C0E94D37D2E96089522970E94F86CB7
:101D2400A13059F40E94FD6CABE2B1E00E94717BDA
:101D34002E2F57E1E2ECF0E008C00E94FD6C0E94F7
:101D4400016D2E2F53E0E7EEF0E0EE83FF830E9457
:101D5400066DA0911908A13081F4E9ECF0E00E942D
:101D64001D6D0E94246D0E94296DEBE2EA93E1E56A
:101D7400F6E10E94826C0E949943E3E0F0E00E9445
:101D84001D6D0E942F6D0E94296D0E94346D0E946A
:101D9400386D3F5FE091C20BAFEE0E94507BF0E0E4
:101DA400EE83FF8311E0E091C30B1E17C0F500E042
:101DB400E091C20B0E1788F50E943E6D59F10E9406
:101DC400456DE09310040E94C46CAE81BF810E94F3
:101DD400467B33960E94F36C0E94DF6C0E94467B24
:101DE400DF010E944F6D0E94526DEA85FB85349796
:101DF400FA93EA930E94296D0E94346D0E94386D13
:101E04003A930E94A720EF3F29F0ADE05A9FF001DA
:101E14000E94576D3F5F0F5FCBCF1F5FC4CF0E94FF
:101E2400856C0E948A6CCAC022970E94CC7DE2E530
:101E3400F7E0EE83FF8340E0443190F4AE81BF814C
:101E440011960E945F6D1396EFEFEC93AE81BF8104
:101E5400EC93EE81FF813496EE83FF834F5FECCFEA
:101E6400E091C20BA0EF0E94507B2E2F0E94FD6CCC
:101E7400A0E4B1E00E94717B5E2F0E94066D21FEFA
:101E840023C00E94646D0E94646DEFEAF0E0FA934F
:101E9400EA930E94696D0E94346D0E94386D0E941D
:101EA4006F6DE6EBF0E0FA93EA930E94646D0E9492
:101EB400246D0E94696DEFE7EA93E3E5F6E1FA9396
:101EC400EA93E0E0F0E011C00E94646D0E94646D4A
:101ED400E8EEF0E0FA93EA93E52F0E94766DFA9328
:101EE400EA930E94346DEBE8FBE0FA93EA930E94D4
:101EF40099433F5F11E0E091C30B1E1710F00C945F
:101F0400DA0F00E0E091C20B0E1710F00C94D80F1A
:101F14000E943E6D11F40C94D50FA0919B0BE0E848
:101F2400EA23E03821F0A091E30BA23019F40E94D7
:101F3400456D0AC00E94796DE03011F4E0E001C003
:101F4400E8E0E0930F04E7E0E0931004A02FBB2740
:101F5400E22FF0E00E94467B3396FA93EA930E94C4
:101F64004F6D0E94DF6C0E94467B3396FA93EA938E
:101F74000E94296D0E94696D0E94346D0E94386D23
:101F84004E2FA0911E08E32F0E947E6DEA0FFB1FC7
:101F940043833A930E94A720EF3F29F0ADE04A9F84
:101FA400F0010E94576D3F5F0F5FACCF1F5FA3CF5F
:101FB4000E94856C0E948A6C0E94AF350E94D37D7A
:101FC40028960895E1E0E0930D04E2E0E0930E0426
:101FD400E0E0E0931004ECE0E0930F04ECE5F3E0C0
:101FE4000E94666CEAE0E0930F04EAE4F3E00E94E6
:101FF400666C0E94294908951A93A981A43029F492
:10200400A0E021FCA1E0A03009F426C0E9810E94EF
:10201400856D0490E9810E948B6DE491A02DAE1B27
:10202400A2501A2F0E946F6DE4EBF0E0FA93EA934A
:10203400EB810E948B6D0E94F97B3296FA93EA93AE
:10204400EAE3F0E00E94936DEFE7EA93E3E5F6E15B
:102054000E94826C0E9499431881229608951A93D3
:102064000A930E949A6D0E9494180E94796D0E2F13
:10207400E4E3F2E00E94F97B33971E2F0E94566C32
:102084000E94566C0E945B6C0E949F6D0A930E9492
:10209400904BECE3F0E00E94A46D0E949546E2E0D0
:1020A400E0930E04E091990BEF70E09310040E940A
:1020B400AB6DEFE0E0931004AA81A13051F40E94CB
:1020C400B36D0E94B56C0E947A46E6E5F6E10E9483
:1020D400B86D21FE0DC0E4E0EA938EDFECE3F2E09C
:1020E4000E94BC6DEEE3F2E00E94BC6D0E94444984
:1020F400A0DC80C0E8810E948B6D0E94BC6DEA81E7
:102104000E94856D0E94BC6D0E94D246E881EA93CC
:1021140073DFC4C11A930A93EC81EA93EBDF1AEEDE
:10212400EC810E94856D0490EC810E948B6DE4919A
:10213400A02DAE1BA2500A2FAC81A43029F4A0E03C
:1021440021FCA1E0A03009F409C01EEAAA81BB81E8
:102154001B96E0E0EC93EC81EA934EDF0E94456D20
:10216400E0931004EC810E94C16DFF93EF930E94F1
:10217400646DEE810E948B6D0E94F97B31960E9402
:10218400936D0E94C46CFA93EA93EC85E058EA9349
:102194000E94566C0E94C76D0E949943AF91BF91F3
:1021A400EC93EC810E948B6D0E94BC6DEE810E94C9
:1021B400856D0E94BC6D0E94444919810881259651
:1021C40008950E94CC6D0E94016D8F010E94566C8F
:1021D4000E94566C0E945B6C0E94CF6D0E94B36D8E
:1021E4000E947A46EA81EA930E9494180E94AB6D99
:1021F4000E94D66D19810881239608950E94CC6DA2
:102204000E94016D8F010E94566C0E94566C0E94C0
:102214005B6C0E94CF6D0E94B36D0E947A46EC8184
:10222400FD810E94B86DAA81BB810E94C27D24F405
:10223400A030E0E1BE070CF006C0EA81FB81FA930E
:10224400EA930E943541AA81BB81A130E0E1BE0737
:1022540024F0A030E1E1BE070CF00AC0A7EEBBE019
:10226400EA81FB81E150F0410E94E06D0E94E86D3B
:102274000E94D66D19810881269608950E94CC6D1E
:102284000E94016D8F010E94566C1A930A930E945A
:102294004449E0E0E0933D0C099119910895E881E7
:1022A400EA930E9494180E94741FE03051F10E9436
:1022B400EE6D0E94566C0E94F26D0E94AB6D0E94FE
:1022C400F66DE881EA930E94F420E8830E94FA6D97
:1022D4003B9734F00E94FA6D0E94056EE9E40BC04E
:1022E400A3EEB6E00E94096E0E940C6E0E94116E6D
:1022F4000E94166EE3E7EA930E941446E2E0E0933C
:102304000E04CCC00E94A768E0E0E0930F04A09103
:102314000403A43019F4E8E6F3E002C0E4E7F3E0D0
:10232400FA93EA930E94794308950E94A1460E9479
:10233400A7680E94FA68E1E0E0930D040E94EE6D44
:10234400E6E0F0E00E941A6EE2E6F6E10E94B86D63
:102354000E94566CE7E0F0E00E941A6EE5E7F6E1B1
:102364000E94B86D0E941E6EEA930E944241E9E702
:10237400F6E10E94B86DE0910403EA930E944241A1
:10238400EFE7F6E10E94B86D08952A971A930A932D
:102394000E94566C0E94566C0E945B6CE4E6F0E06E
:1023A4000E94606C00E010E01530B0F4053020F4B9
:1023B4000E94236EE03009F40DC00E94566C0E9406
:1023C400C46C0E941A6E0E942A6E0E94236E0E94A0
:1023D4002F6E0F5F1F5FE8CF0E94316E0E947A4616
:1023E400E5E8F6E10E94B86DE091420CEA930E94A0
:1023F4004241E091410CEA930E9448410E94B06C32
:102404000E94B36D0E947A46E9E8F6E10E94B86D35
:10241400E0912306EA93E5E0EA930E94F840E09114
:102424001A0CE03079F10E94B06CE2E0F0E00E9416
:102434001A6EE09128060E94346E0E94646D0E9418
:102444007A46E0912806E295EF70E695E695AE2F80
:10245400E0912906EE0FEE0FEA0F0E94346E0E94FF
:10246400B56C0E947A46E0912906E295EF70AE2F92
:10247400E0912A06E295E07FEA0FEA93E6E0EA9328
:102484000E94F840198108817DC1E881E064E7B9C0
:10249400369A349BFECF349AE4B1F5B1219608956F
:1024A400E881F981AA81BB81AE17BF071CF4EA1B3E
:1024B400FB0B06C0A881B981EA81FB81EA1BFB0BF7
:1024C4002496089528970E94CE7DEFE0E093610062
:1024D400E1E00E943A6EE5E00E94416E0E94486E7F
:1024E400E0936F05F0937005E0917B05F0917C0516
:1024F400E0936D05F0936E05E1E0EA93C6DFE093A7
:102504007B05F0937C05EFE0E0936100E8E00E9436
:102514003A6EEAE00E94416E0E944D6EE0936B05B4
:10252400F0936C05E0917905F0917A05E0936905E3
:10253400F0936A05E0E0EA93A8DFE0937905F0936D
:102544007A050E944D6EA0916B05B0916C05EA0F5F
:10255400FB1FA0917905B0917A050E94526E8F01FC
:102564000E94486EA0916F05B0917005EA0FFB1FA1
:10257400A0917B05B0917C050E94526E9F01E09171
:102584006B05F0916C050E94596EFF93EF930E94C6
:102594004D6E0E94596EAF91BF91EA0FFB1FFF93DE
:1025A400EF93E0917905F0917A050E94596EAF910D
:1025B400BF91EA0FFB1FE0937505F0937605E09158
:1025C4006F05F09170050E945F6EFF93EF930E9478
:1025D400486E0E945F6EAF91BF91EA0FFB1FFF939D
:1025E400EF93E0917B05F0917C050E945F6EAF91C3
:1025F400BF91EA0FFB1FE0937705F0937805A09154
:102604007505B0917605E4E1F0E00E94187B0E2E8A
:10261400A0917705B0917805E4E1F0E00E94187B81
:10262400E02919F00E944945ABC00093710510934D
:1026340072052093730530937405A0916405A63444
:1026440028F4E0916405EF5FE09364050E94656EF1
:10265400989724F40E946A6E98970CF00EC0A0918B
:102664006405AA3019F4E1E0E0936105A0916405E2
:10267400A83219F4E2E0E09361050E94656E99972F
:1026840024F00E946A6E99970CF47AC0E091670571
:10269400EF5FE09367050E946F6E0E94656E0E9473
:1026A400746E0E947B6E0E94806E0E944B7B7F93AF
:1026B4006F93FF93EF93A2E0B0E00E94147C0F01AC
:1026C4000E946F6EDF01F001EA1BFB0BAF91BF911B
:1026D4008F919F910E94896E0E947B6E0E948E6EE4
:1026E4000E946A6E0E94746E0E94936EAC81BD81DA
:1026F4008E819F81EFE3F1E060E070E00E944B7B0C
:102704007F936F93FF93EF93A6E0B0E00E94147C55
:102714000F010E948E6EDF01F001EA1BFB0BAF91EB
:10272400BF918F919F910E94896E0E94936EE09158
:102734001204E03049F4E885F985E0935905F093F3
:102744005A05EC81FD810AC0EC81FD81E0935905B5
:10275400F0935A050E94806E0E94E07AE0935B0534
:10276400F0935C05E0915905F0915A05FA93EA93C8
:10277400E0915B05F0915C05FA93EA930E94D144E1
:102784000E94D57D2C9608951A930E94A146E2E0FA
:10279400E0930E04E2E3F0E00E947D6C0E94986EE8
:1027A400EDE8F6E10E94B86DE4E1EA930E94A140ED
:1027B400E0E9F1E00E949C6EE4E1EA930E94A1400A
:1027C400A0916705A13010F0A895FACF10E014305D
:1027D40010F00C944714E2E0E0930D040E94A06E04
:1027E400DF010E94BC6DFD0132960E94BC6D0E9407
:1027F40095460E94A06E3496E491EA930E94144692
:10280400E1E0E0930D04A0916705AF3110F4A895C1
:10281400FACFEAE0EA930E94A1400E94A06EDF0191
:1028240035960E94F97BBF01FD010E94A66EDB0173
:102834000E94247C0E94AD6E0E94DF6CE8E2F0E00E
:102844000E94467BE65AFF4F0E94986E0E94A06E3B
:102854000E94A66E0E94056EA0916705AE3110F02D
:10286400A895FACF0E94A06EDF010E94BC6DFD0105
:1028740032960E94BC6DE8E1F0E0FA93EA93E8E254
:10288400F0E00E94606C1F5FA2CF0E94AD6EEAEF81
:10289400F0E00E94986EE9E9F6E10E94B86DE0ED7F
:1028A400F7E00E949C6E0E94A1465FC10E94B26E36
:1028B4000A93E4E6E2BF78940E94934403DEE6B30D
:1028C400AFEFEA27E093420CE091410CE03009F0CD
:1028D40002C0E091420CE0933108A3E6BBE00E9401
:1028E400C16EE091630BE77031F4A0910A04E0E457
:1028F400EA27E0930A04E091630BEF7131F4A091AD
:102904000A04E3E8EA27E0930A040E9447660E9467
:102914009321E2B3EF700E2EA0911408B091150824
:10292400EFE0F0E0AE27BF27EA23FB230E94F97A09
:10293400E029E2BBE0911408E07111F41D9A01C092
:102944001D980991199114C00E94B26EE6E0E4BD8D
:10295400E0B1E295EF70AE2FE0916300E071EA2BF5
:102964001E2F0E949F6D0E946A210E942166199168
:10297400E991EFBFF991E991B991A991999189915F
:1029840079916991F9901990099018950E944B6575
:102994000E94D1650E94DA500E94B01E08951A93D5
:1029A400A8950E94A742E13011F00C943215E091F1
:1029B400C605E1501E2FA091C505A13021F40E9447
:1029C400C76EE03009F40CC0ADE01A9FF001E15F7E
:1029D400FC4FBF01E081E260DB01EC930E94CE6E0C
:1029E400A091C505A23011F0A43089F40E94C76EED
:1029F400E093DB050E94D36E31F0FD01E15FFC4FF3
:102A0400E081E27009F403C01A930E94DC6EA09185
:102A1400C505A33019F41A930E946227A091C50535
:102A2400A53029F4E091C605EA930E948F27A0916E
:102A3400C505A830A9F4E0E0EA93E091C605EF7774
:102A4400EA930E9467181E2F1F3F51F0E0E0EA93BB
:102A54000E94A140E12FE058E093DB05E0932D06AE
:102A6400E0910A04E07821F1E0910A04EF77E09321
:102A74000A040E946D49E0910A04E07131F0E0918A
:102A84000A04E270EA930E947B45E4EEEA930E9412
:102A94008D66A0913E0CA13021F4A0911908A430B8
:102AA40009F406C0E0EBEA930E948D66E093410CC2
:102AB400A0913D0CA13039F4E0913F0CF091400C11
:102AC4000E94E06E09F401C0D9DB60DF4EC01A93A6
:102AD4000E94A146E1E0F0E00E94826C0E947A46E6
:102AE40010E00E94EA6E0E94566C0E949F6D0E9444
:102AF4007A46E0912108E03049F4ECE9F6E10E94DD
:102B0400B86D0E94F06E0E94166E1E5FA09121089F
:102B1400A130F0F0E0912108E150EA930E94C3183B
:102B2400A091B40BAD3229F40E94F96E0E94BE7DCF
:102B340079F0E4EBFBE00E94E86DE6E0F0E0FA9364
:102B4400EA930E94066F0E94F96E0E94166E1E5F41
:102B5400E0912108EF5FE09321081C3020F4A0915C
:102B64002108AB3008F001C0BECF199108951A9323
:102B74000E94A146E981E03019F4E0E0E0931E08E8
:102B8400A981A230A9F410E0A0911E08A13010F090
:102B94001C3008F00DC0E0911E08E150E0931E08BF
:102BA4000E940A6F19F40E94186F09F01F5FECCF9E
:102BB4000E94EA6E10E00E94566C0E949F6D0E9473
:102BC4007A46A0911E08A03408F50E940A6F19F4F1
:102BD4000E94186FD1F0E0911E08EA930E949418A5
:102BE4000E94AB6D0E94566C0E94066F0E94236F78
:102BF4000E94056EE8E7EA930E9414460E94F66D6F
:102C04000E94286F0E94166E1E5F05C0E3EAF6E17B
:102C14000E94B86D1E5FE0911E08EF5FE0931E08EE
:102C24001C3020F4A0911E08A13408F001C0C3CFC9
:102C3400188122960895E0E0E5BFE0936D00E093EB
:102C44006C00EBBBEFEFEABBE0E0E8BBE7BBE5BB46
:102C5400EFEFE4BBE0EFE2BBE1BBE0E2E3B9ECEBB6
:102C6400E2B9E0E0E0936200E0936100EFE0E0931A
:102C74006500E0936400E0E0E0BFE7E0E3BFE4E682
:102C8400E2BFE0E0E1BFEFBDEEBDEDBDECBDE7BDF1
:102C9400E6BDEBBDEABDE9BDE8BDE0937900E09394
:102CA4007800E3E0E5BDE6E0E4BDE0E0E3BDE09309
:102CB4008B00EAE0E0938A00E0E0E0938900E0938F
:102CC4008800E0938100E0938000E2E1E0938700D4
:102CD400E4E3E0938600E0E0E0938500E093840081
:102CE400E0938300E0938200E0936A00E0E3EABFAC
:102CF400E0E4E9BFE8BFE1E4E7BFE0E0E0937D00A2
:102D0400EBB9E8EDEAB9E6E0E0939500E0E0E093A2
:102D14009000E7E6E9B9E0E0E0939B00E8EDE0939A
:102D24009A00E6E0E0939D00E0E0E0939800E3E39E
:102D3400E0939900E0E8E8B9E0E0E0BDE0E4E7B959
:102D4400E7E8E6B9E0B5EF7EE0BDE0E2E0937000CD
:102D5400E0E0E0937200E4E4E0937400EFE1E1BDAD
:102D6400EFE0E1BD0E94E45D0E942C4B0E946C45A3
:102D74007894E1E0EA930E94090D0E941E6EE53109
:102D840028F0A9E0B0E0E0E00E942C7CCEDA21E05B
:102D940030E0E0EEEA930E948D66E09332080E94F0
:102DA400316F3F5FA0913208A43511F03A3008F03A
:102DB40001C0EFCF30E0E0EBEA930E948D66EF3F75
:102DC40019F0E1E0E0933E0C0E94316F3F5FA09167
:102DD4003E0CA03011F43A3008F001C0ECCF0E9450
:102DE400B36D0E94B06C0E947A46A0913208A4355B
:102DF40081F4E2EEEA930E948D66E0933208E8EAF9
:102E0400F6E10E94B86DE0913208EA930E941446FC
:102E140008C0E0E0E093320820E0EEEAF6E10E9428
:102E2400B86DA0913E0CA13021F4E7EBF6E10E94CD
:102E3400B86D92D0E03059F40E94B36DE9E0F0E04F
:102E44000E941A6EEAEBF6E10E94B86D20E00E943F
:102E54006F6E0F01A2E0B0E00E94147C0E161F06F4
:102E640054F40E948E6E0F01A6E0B0E00E94147C20
:102E74000E161F060CF088DC203071F40E94B36D2E
:102E8400EAE0F0E00E941A6EE6ECF6E10E94B86D0A
:102E9400A8950E94346FFCCF0E9496360E94B36DB1
:102EA400E9E0F0E00E941A6EE1EDF6E10E94B86DEF
:102EB4000E94371BE03019F0E7EDF6E102C0E9E9C2
:102EC400F6E1FA93EA930E942B460E945966E1E0E8
:102ED400EA930E94A14000E010E00436E0E01E07FF
:102EE40024F40E94D165E03009F005C00E94316FDE
:102EF4000F5F1F4FF2CF0436E0E01E072CF0A091C5
:102F04006705AF3108F040DC4ADD0E9401320E94BF
:102F1400671DFACFFFCF0E94376F17FD02C0103034
:102F240011F4E0E05DC3E12F5BC30E94376F17FD2E
:102F340010E01A3008F41F5F0E94446F51C30E94CE
:102F4400376F17FD02C0103011F4E0E049C311508F
:102F54000E94446FE1E044C31A930A9310E0E4E64C
:102F6400F0E00E949C6EA8950E94A766E03021F4D0
:102F7400E0EA0E944F6F09F002C001E001C000E0E6
:102F84000E94B8661F5F003011F4153008F001C0CC
:102F9400E6CFE02F0991199108950E94546F3DC422
:102FA4000E94546F0E94616F0895A881B9810E94A4
:102FB400C27D24F4A83EE3E0BE070CF005C00E94E5
:102FC400646F0E941A670DC3E0E00BC3EA81E0302E
:102FD40011F4EFEFEA83A881B9810E94C27D24F441
:102FE400A83EE3E0BE070CF006C00E94646FED81CA
:102FF400EA930E9446675AC10E94CE7D20E030E0E9
:10300400283EE3E03E077CF4A8953A932A93CDDF6B
:103014001E2F1F3F29F0EFEFEA933A932A93D6DF4E
:103024002F5F3F4FEDCF0E94D57D4DC01A930A9379
:10303400E0E0F0E0E093430CF093440CAA81A03468
:1030440058F40E946D6FE55FFB4F8F010E94746F0F
:10305400E3E4FCE00E947D6FE091430CF091440CAA
:1030640023C11A931FEF1F5F1A93E0DFA981BA816E
:10307400EA17FB0711F0113408F001C0F4CFE12F77
:10308400188114C11A930A93A091C20BE091C30B47
:10309400EA9FF001A0911E08EA0F0E2F013408F0F8
:1030A4000FE310911E08101758F41A93BFDFAA817A
:1030B400BB81EA17FB0711F4E12F03C01F5FF3CFB5
:1030C400EFEF19810881249608950E94CC7D10E0C9
:1030D400103418F50E94DF6CE8E2F0E00E94467BB1
:1030E400E050FC4FAF01E0EAEA93FA0170960E94C7
:1030F400816FEC713E2FE0EAEA93FA013F960E9459
:10310400816F0E2FEF81E31719F4EE81E01709F0B8
:1031140002C0E12F03C01F5FDBCFEFEF0E94D37D1E
:10312400289608951A930A93E0918A0BAA81EA17C4
:10313400C1F0A03468F40E946D6FE050FC4F8F0121
:103144000E94856F0E947D6FEA81E0938A0B09C01B
:10315400EFEFE0938A0B0E94906F0E94956FE093CB
:10316400950BA2C01A930A930E946D6FE050FC4F16
:103174008F01AA81A03420F40E94856F0E94616FA0
:1031840093C01A930A93E091B30BAA81EA17A1F0B2
:103194000E949F6F40F40E94AB6F0E947D6FEA8192
:1031A400E093B30B09C0EFEFE093B30B0E94B66F4B
:1031B4000E94956FE093BE0B77C01A930A930E9406
:1031C4009F6F20F40E94AB6F0E94616F6DC01A93D1
:1031D4000A93E091340CAA81EA1751F10E94BB6F63
:1031E40008F50E94746FE5E3FCE00E947D6FEA81BC
:1031F400E093340CE0E0E0932B06A091360CA13070
:1032040020F0A091360CA83008F00BC0A9EDBBE06B
:10321400E091360C0E94C56FAE0FBF1FEC91E09396
:103224002B0606C0EFEFE093340CE0E0E093350C9E
:103234003BC01A930A930E94BB6F30F40E94746FD0
:10324400E5E3FCE00E94616F2FC01A930A93E091BA
:103254002F0CAA81EA17C1F00E94C86F70F4E0EA4B
:10326400EA930E94B56C1A930A93E0E3FCE00E948F
:103274007D6FEA81E0932F0C07C0EFEFE0932F0CF2
:103284000E94D26F0E940B690FC01A930A930E9486
:10329400C86F50F4E0EAEA930E94B56C1A930A935B
:1032A400E0E3FCE00E94616F198108812396089590
:1032B4000E94D26F0E940B69E881EF5FE093310CAA
:1032C400D2C124970E94CC7D0E94D96F0E940B69C1
:1032D400AA85A03478F5AB85A13010F0A63008F0AB
:1032E40007C0EB850E94C56F0E94E06F0E94F36FD8
:1032F400EB85E030F9F4E0E0EE83EF83E887E987DB
:1033040040E050E020E030E02530E0E03E0784F487
:10331400F9010E94E06F0E94F36F0E94236F4E0F29
:103324005F1F0E94286F0E94F86F2F5F3F4FECCF02
:103334000E9403703FC11A930A93AB81A13010F02D
:10334400A63008F01CC0EB810E94C56F0E94FD7A74
:103354000E94F97ADF01EA810E941470E8E0F0E04B
:103364000E94467BE050FA4E8F01E0EAEA930E9405
:10337400B06C1A930A93EDE1FCE00E94616F19812D
:1033840008810C94AE1E0E94CE7DEC810E941870C0
:10339400E83109F459C00E941D70309729F00E9449
:1033A4001D700E942270EC830E94681F0E2F10E093
:1033B400101710F00C94261A0E94267082DFAFE1D9
:1033C400BCE00E94C16EA091210CB091220C8091AE
:1033D400230C9091240C0E942B700E94DB7AE093C2
:1033E400210CF093220C6093230C7093240C0E9404
:1033F4002670A1DFE0EAEA93EE810E94C56FEE0F2A
:10340400FF1FE050F04F0E94816FE270D9F4ED810C
:10341400E093250C0E941D70309751F40E941E6E9B
:103424000E943270EF5EF84DDF010E94387002C0D6
:103434000E941D70E093260CF093270C0E943D70AF
:103444000E9442701F5FB4CF0E94D57D26960895D6
:103454001A930A930E944870ECE2F0E00E944F70C5
:103464000E9453700E94587010E01034D8F41A93DC
:1034740059DEE0912208EA931A9323DF0E946170D7
:10348400EA0FFB1F0F010E9461700E946970DF0147
:10349400CB010E94286F0E94DB7AD0010E94F47B4A
:1034A4001F5FE3CFA0911908A330B9F500E0003104
:1034B400A0F50E94C46C0E946E7069F510E01A3089
:1034C40050F5E02FE05DEA93ECEDF6E10E947370B5
:1034D400E12FE05D0E947A70E1F40E947F700E9407
:1034E4008670EA0FFB1FFF93EF930E9486700E9481
:1034F40069707F936F93FF93EF930E943362AF9150
:10350400BF918F919F910E94DB7AAF91BF910E94EE
:10351400F47B1F5FD4CF0F5FCACF10E01A3090F452
:103524000E9486700E946970A0912908B0912A08AF
:1035340080912B0890912C080E94DB7A0E9458708D
:103544001F5FECCF0C94F61E24970E94CC7DEA8575
:10355400EA936CDD9F01022E032A39F13A932A93F0
:1035640080DD1E2F40E050E0E0E0EE83EF83E8874B
:10357400E987AA851A17B1F4012F003498F40A9345
:1035840055DD2E173F0761F4EB85EA930A9399DE24
:103594000E94236F4E0F5F1F0E94286F0E94F86FD6
:1035A4000F5FEBCF0E94037005C0EB85EA93EB85B8
:1035B400EA9387DE0E94D37D2C9608951A93A895EA
:1035C400A981A63068F40E94D96F0E940B6910E0AB
:1035D400103430F4E981EA931A93ADDE1F5FF8CF1B
:1035E4001881229608951A9311E0163020F41A9344
:1035F400E5DF1F5FFACF6AC3E1E0E093350CE093A7
:10360400360C31C0A8950E94B66FEEEAF3E0FA9347
:10361400EA930E94B06C0E948D70E093BC0B0E94F0
:103624009670E093BD0BE0E0E093BE0B1CC0A89540
:10363400EAE8FBE00E949D70E9E2F0E00E944F702E
:103644000E94906FE4EAF3E0FA93EA930E94B06C6C
:103654000E948D70E093930B0E949670E093940BFC
:10366400E0EBE093990B219608950E94CC7D0E9493
:10367400A270E03228F0AAE0B0E0E0E00E942C7CE6
:1036840000E08BDCA091BF0BB091C00BA633E2E14C
:10369400BE0741F110E01A3030F41A93B3DF1A93E5
:1036A4008CDD1F5FF8CF10E0103430F41A93BFDFC5
:1036B4001A9358DD1F5FF8CF10E0103830F41A93D6
:1036C4009BDF1A93B6DD1F5FF8CF8DDFA9E0B0E072
:1036D400E0E00E942C7CE6E3F2E1E093BF0BF09380
:1036E400C00B01E010E0183210F00C94CA1B0E94C9
:1036F400A7709F010E94A770AF010E94B170349619
:10370400E491E03011F0E13069F4D901AC910E9408
:10371400B1703596E491EA1720F40E94B1700E94CA
:10372400B87034C0E23091F4DA010E94EA7BE031EF
:10373400A7E2FA0714F4FF2342F40E94B17036960C
:103744000E94F97BDA01ED93FC9320C0E33049F445
:10375400D901AC91AF3F21F40E94B1700E94B870BE
:1037640015C0E43099F4D901AC91AF3F79F400E08D
:103774000E94B1703596E4910E1740F40E94B17026
:103784000E94B8702F5F3F4F0F5FF2CF1F5FABCF28
:1037940007DC10E0153060F41A9357DDA091300C6B
:1037A400A63020F01A9384DD1A936FDD1F5FF2CFE9
:1037B400E02F0C948D20E881EF5FE883A881A43684
:1037C40010F0E0E0E883E8810C940A210E94096E7D
:1037D400A5E0B0E00E94467B30960C940A21A091AB
:1037E400380CBB27E091370CA6C0F9DF329774F090
:1037F4000E94BD70E091370C0E94C4700E94616FFA
:10380400E091370CEA93D7DFE093370C08950E94D8
:10381400BD70E091380C0E94C470FA93EA930E9440
:1038240067670895E5E2FCE00E94CC700E94BD70D9
:10383400E091380C0E94C4700E94616FE091380CD2
:10384400EA93B9DFE093380C08950E94CE7DE0E05E
:10385400E093370CE093380C10E030E0343680F518
:10386400A8950E94BD703A93B1DFFA93EA93E5E21A
:10387400FCE00E947D6F00E0A091250CA13010F0C7
:10388400A03808F001C001E0E12FE03041F401303C
:1038940029F43093380C3093370C11E00FC0E13029
:1038A40031F4003019F43093370C12E007C0E230E1
:1038B40029F4013019F43093380C13E03F5FCECF74
:1038C40049C21A93A091D00BA870B9F010E0E98115
:1038D400FA810E94DF6CAE17BF077CF4ED81E093A0
:1038E400250CEB81FC81E851FC4F0E94D370E0E091
:1038F400F0E00E9442701F5FEACF18810C948F2081
:10390400E881EF5FE883A881A43610F0E0E0E88363
:10391400E8810C940A21E881E150E883A881A43667
:1039240010F0E3E6E883E8810C940A21A0913A0CB4
:10393400BB27E091390CF0E031960E94D870EC5925
:10394400FF4FDF01E4E6F0E00E94A37B08950E94AC
:10395400096EA5E0B0E00E94467BE050FE4F0C9457
:103964000A210E94DD70E881EA93C0D10C940A21F7
:103974001A9342DBE1E0E093870BA8C1A89510E01D
:10398400143680F41A93ABD1A0912A0CAF3F31F4D2
:103994000E94E070AF3FEFEFBE0711F01A93E1DF32
:1039A4001F5FEECF0E94E570689420F88FC10E94DB
:1039B400CE7D10913A0CAD81AA23CAF5E091390C61
:1039C400E11719F0AD81AA230AF030C01A9387D108
:1039D4000E94E070EE81FF81EA17FB0729F4E88575
:1039E400A0912A0CEA1709F01EC00E94EB70EC812A
:1039F400FD810E94E57AEA17FB0744F40E94F07007
:103A04000E94F970E0E0EC83ED830BC00E94F0703B
:103A1400EC83FD83E0E0F0E00E94F970E0E0E093E5
:103A24002A0C1A9363D10E94FE70C8CF46C0E0915D
:103A3400390CE11729F0AC81BD810E94C27D0CF0E4
:103A44001BC01A934CD10E94E070EE81FF81EA17EB
:103A5400FB0729F4E885A0912A0CEA1709F009C0AC
:103A64000E94F0700E94F9701A9340D1E0E0EC8358
:103A7400ED830E94FE70DBCFAC81BD810E94C27DCC
:103A84001CF454DF33970CF418C0E885E0932A0C37
:103A9400EE81FF810E940371EC81FD810E94F97027
:103AA400E091390CEA9322D1E091390CEA9328DFB2
:103AB400E093390CE0E0EC83ED83689420F8EC812A
:103AC400FD810E94D57D299608951A93A091450CF5
:103AD400A03059F4E091480CF091490CFA93EA9320
:103AE400E8EBFBE00E94087109F40BC0E1E0E0930D
:103AF400450CE091390CE093470CE091390CE093CC
:103B0400460CA091450CA13011F00C94EA1DE091F3
:103B14003A0CA091470CEA1711F40C94DB1DE091C8
:103B2400470CEA93F8DEE093470CEA93D8D0A091CF
:103B34002A0CA13010F0A03808F034C0E091460CF3
:103B4400EA93E9DEE093460CA091470CEA1749F1A9
:103B5400EA93CCD0E091E30BE030E9F410E01530C7
:103B6400D0F4ABE01A9FF001DF01E352FA4FE08199
:103B7400E03049F0FD01E452FA4FE081AE2FE091CC
:103B8400470CEA1709F005C00E940E71A091460C7B
:103B9400A0831F5FE4CF0E94DD70E091470CEA939D
:103BA400A5D006C00E94DD70E091470CEA939ED038
:103BB4000FC0E091460CE0933A0CE0E0E093450C32
:103BC400689420F80E948168E093480CF093490CB3
:103BD4007DC01A93A89510913A0CE091390CE11725
:103BE400C1F00E9414710E94C27D64F4EB81A09123
:103BF4002A0CEA1739F40E94E070E981FA81EA1785
:103C0400FB0709F003C0E12F1881A6C00E94FE70D3
:103C1400E4CFEFEF1881A0C00E94EB700E94C27D38
:103C240084F4E0912B06E87031F4E0912F08A09120
:103C34002A0CEA1731F40E9418710E942270E034B1
:103C440008F001C05CC10C946821A895E091390C7E
:103C5400A881EA1761F0E8810E941D7119F0E881DA
:103C64000C940A21E881EA934BDEE883EFCFEFEF6F
:103C74000C940A211A93A89510913A0CE091390CEE
:103C8400E117E1F00E9414710E94C27D8CF4E0916E
:103C94002B06E87031F4E0912F08A0912A0CEA1762
:103CA40039F40E94E070E981FA81EA17FB0709F010
:103CB40002C00C944F210E94FE70E0CFEFEF0C94F1
:103CC40050211A9310913A0C1A93BFDF1991089559
:103CD400E881EA9315DEE883EA93B7DF99C20E948C
:103CE400BD700E9424710E947D6F92C20E94BD70BB
:103CF4000E9424710E94616F8BC20E94CE7D0E943B
:103D0400E57010E030E0343628F5A8953A93E7DF03
:103D140000E0A0912A0CA03808F401E0E12FE03083
:103D240041F4013029F430933A0C3093390C11E00A
:103D34000FC0E13031F4003019F43093390C12E043
:103D440007C0E23029F4013019F430933A0C13E03F
:103D54003F5FD9CF0E94D57D249608951A930A9384
:103D6400A0911908A43009F43FC010912F080091C4
:103D7400540CE0913108E03059F0E0932F08689436
:103D840024F80E942D71E0E0E0933008E0E520C0C3
:103D9400E0913008E03021F0E0932F08E2E518C00C
:103DA400E0E0E0932F08E093540CE091C50BE03081
:103DB40031F0E091C50BE150EA930E94E918A0911B
:103DC400350CA17039F0E091C50BE0932F08E4E4C1
:103DD400E093540CA0912F081A1721F4A091540CCD
:103DE4000A1711F0689423F80991199108950E9413
:103DF4003371EBE0EC93EC81D8011696EC93EB81F4
:103E0400D8011796EC93D8011896E0E0F0E0ED9312
:103E1400FC93D80112960E944071D80114960E9416
:103E240040710E94457101C10E943371ECE0EC9332
:103E34000E94457134C21A9318E0113108F5E091DB
:103E44001408F0911508A981BA81EA27FB27BF015C
:103E54000E945171E623F723309781F00E9451713B
:103E6400A981BA81EA23FB23309731F01A93E0E069
:103E7400EA931A93BCDF02C01A93D6DF1F5FDDCF2B
:103E84000DC2A0911B0CA93030F0E0915C0CA09104
:103E94005B0CEA1709F414C0E0915C0CE03021F4E7
:103EA400E3E6EA93C1DF08C0E0911B0CEA93E0E08B
:103EB400EA93E3E6EA939BDFE0915C0CE0935B0C0E
:103EC4000895A0919B0BECE1EA230895A0919B0B2C
:103ED400A07411F0E2E00895A0919B0BA07809F082
:103EE400F5C10DC0A0918A0BAF3F09F4EFC1E9DF22
:103EF400E43009F4EBC1E5DFE03109F4E7C1E1E0C6
:103F040008950895A881AF3F11F4E0E081C1D9DF9D
:103F1400E43011F4E1E07CC1E0E07AC1A881A23090
:103F240019F4CFDFE83011F0E1E072C1E0E070C1D4
:103F3400A881B981AC91A130A8F0A881B981AC91D4
:103F4400A43180F4A881B981EC910E945C71EB5F8B
:103F5400FC4FE081EF770E2EA881B9811296EC9187
:103F6400E01509F002C0E1E011C1E0E00FC1A88151
:103F7400A13118F0E881E051E883E8810E94617181
:103F84000E946B71A091D10BA13018F0A881A430CC
:103F940009F006C0E6E9F0E00E94F97B0E946B712B
:103FA40037C1A881A13010F0A63008F006C0E8811E
:103FB4000E947671E15CF94F2AC1E0E029C1A88131
:103FC400A13010F0A63008F006C0E8810E94767196
:103FD400EC5BF94F1CC1E0E01BC10E94CE7DEC817B
:103FE400EA93EDDFEF731E2F1030E1F0EC81EA93DA
:103FF400E6DFE0743E2FE12FE150A1E00E94F17A68
:10400400A0912306EA230E2F303011F4003009F07A
:1040140002C0E1E008C0303011F0003009F402C001
:10402400E1E001C0E0E00E94D57D259608950E945C
:10403400CC7D00E00530A0F50A930E9427190E9468
:104044007B71A7E10A9FF001EE5CF94F0E949D701D
:10405400E4E1F0E00E944F70E091310CDA015096F7
:10406400EC93A091300CEFE3EA23AE2FE091330CF4
:10407400E295E07FEE0FEE0FEA0FDA015596EC932E
:10408400E091310CE1503E2F3F3F41F0E091320C82
:104094000E943270DA015196ED93FC930F5FCACF00
:1040A40010E01034C0F51A930E9494181A932ADF72
:1040B400E13079F5E0919E0BEA9373DFE1500E2F26
:1040C4000F3F39F10E947B71E12FDA011396EC93D3
:1040D400E0919E0BDA011496EC93E091A40BF0911D
:1040E400A50BDA011696ED93FC930E942B70A4E6BF
:1040F400B0E080E090E00E944B7BDF01CB01E091D7
:10410400A40BF091A50B0E94896EDA011A96ED9327
:10411400FC931F5FC6CF0E94D37D26960895A0917D
:104124001908A23031F0A83021F0A73011F0A530E1
:1041340009F40AC00E944870EFEFF0E00E944F704B
:1041440076DFE0E0E093A20608951A93E981E0584F
:10415400E98310E01530C0F4A3E21A9FF001EB5597
:10416400F94FE081AE2FE981EA1749F4F001EC55EB
:10417400F94FE081AE2FE0912F08EA1709F002C051
:10418400E12F03C01F5FE6CFEFEF18812296089559
:104194000E94CE7DED81EA93D8DF1E2F1F3FF1F000
:1041A400A3E21A9FF001ED55F94F9F01D901129630
:1041B400EC91EF77EC93EC81D901EC930E945C7164
:1041C400EF5EFC4FBF01E081EF77DB01EC93EC8104
:1041D4000E945C71E15FFC4FA1E0A083E12F0E948B
:1041E400D57DE4C40E94096E0E94827161F4E0915D
:1041F4004E0CEF5FE0934E0C0E94096EED55F94FA3
:10420400A0914E0CA0830E94096EED55F94FE081F8
:10421400219608951A931FEFE091D50BF091D60BD8
:10422400A981BA81AE17BF073CF0E091D70BF0919A
:10423400D80BEA17FB070CF412C00E9487710E9486
:10424400D7171E2F103031F01F3F21F0E0912F08B7
:10425400E11729F4E1E0E0935C0CE0E01FC0E0E04A
:10426400E0935C0C1AC01A930E948771D3DF1E2F4F
:10427400103099F01F3F39F4E0EEF6E1FA93EA9337
:10428400EB81FC8106C0E0EFF6E1FA93EA930E9429
:104294008C71FA93EA930E940011E12F18812396FE
:1042A4000895E0916505E03009F00895E0912C0649
:1042B400E03009F008950AC0E0916605E03009F0A5
:1042C4000895E0912D06E03009F00895E0E00895A6
:1042D4000E94CE7DE0912606F0912706AC81BD8137
:1042E400EA27FB279F0110E0153090F4F901E170F3
:1042F40049F0A7E11A9FF001EF5CF94FDF01EC915F
:10430400EF5FEC93D9010E948F719F011F5FECCF87
:10431400EC81FD81E0932606F09327060E94D57D6B
:1043240045C428970E94CC7D3091260610E01530B4
:10433400B8F5A7E11A9FF001EB5BF94F0081E12F7B
:10434400A1E00E94F17A2E2FE22FE32391F00038AE
:1043540010F0003C08F001C00F5F003C31F4E22F84
:10436400A0912306EA2BE0932306003808F400E822
:104374000FC0003408F40F5F003439F4EFEFE22784
:10438400A0912306EA23E0932306003808F000E016
:10439400A7E11A9FF001EB5BF94F00831F5FC7CFC2
:1043A400E0E0E0932C06E0E0F0E0E0931608F09300
:1043B4001708E0915C0CE03021F0E0911B0CEA93CB
:1043C400D6DDE0911D08EF5FE0931D08E091E40B5A
:1043D400A0911D08EA1751F4E091E40BF0E0A0E08D
:1043E400B1E00E940D7CEA1BE0931D08A09119081E
:1043F400A13019F0A93009F096C0A091630BB091D7
:10440400640BE4E1F0E00E94A37B309719F4E1E04F
:10441400E0931F0846DFE03019F04EDFE07809F43E
:1044240062C04ADFEF775E2F5A930E9494180E946D
:104434004F6DED55F94F5081503011F40C947522A5
:1044440051DDE13031F4E0911A08EA9367DDE030A0
:1044540009F449C00E9494710E941470EC91EC71AB
:10446400EC3021F4E0911D08E07851F40E94997138
:10447400EC91EA937CDD0E949E71EC91EA9377DDE6
:104484000E949971AC91A63070F5A3EEB6E00E943B
:104494004F6D0E940C6E0E94C16E0E949971EC9146
:1044A400EA937FDD1E2F1130F0F00E94A3710E9469
:1044B400A671CF010E94A3710E940C6E6D917C9134
:1044C400E12F0E947671EF5CF94F0E94AB71E60F09
:1044D400F71FDC01ED93FC93E12F0E947671EF5CF2
:1044E400F94FA0E0A08310E01530E8F40E94AE710B
:1044F40013965C915F3FA9F05A9374DE5E2F0E947D
:10450400B8710E94A3710E94A671BF010E94A37199
:104514000E940C6E0E94BE71AE81BF811296E0E0D3
:10452400EC931F5FE1CFA0911908A23039F0A830B5
:1045340029F0A53019F0A73009F0EAC1E0E0E093D2
:10454400200800E0053010F00C948A24A3E20A9FAE
:10455400F001ED55F94FEA87FB87AA85BB85AC913D
:10456400A03019F0A281A07809F0D0C1E091200810
:10457400EF5FE0932008AA85BB8513960E94EA7B2F
:10458400309771F0AA85BB8513960E94CB710E9467
:10459400D17129F4AA85BB8513960E944071B6C1D6
:1045A4008BDEE03021F00E94D17109F4AFC120E02C
:1045B40030E0333010F00C9435240E94DB71DF01BD
:1045C4000E94DC6C0E94E06DE887F987A181A270EB
:1045D40021F4A481B581109709F410C1E885F98507
:1045E400A181A47011F40C945723A181A87021F423
:1045F4000E947133E03009F457C00E94E171EBE08E
:10460400EC93A885B9850E94EE71A885B9851396A7
:10461400EC91AC85BD851796EC93EC85FD853896B9
:104624000F01E885F985A181E1E0EA230E94F57193
:10463400ED93FC93A885B98514960E94EA7BAC851A
:10464400BD851296ED93FC930E94F871AC85BD85EF
:104654001496ED93FC93A02FEAE0EA9FF001E30F98
:10466400EF5F0E94FE71E885F985A085B185E2E0DF
:10467400F0E00E94467BA885B9851896ED93FC93DB
:104684000E94F871309739F4A885B9851896E8EE38
:10469400F3E0ED93FC93E885F985A181E8E0EA2B4A
:1046A400A885B9851196EC936EC0E885F985A1813A
:1046B400A17031F4A885B98514960E94CB7143C0CA
:1046C4000E9407726EDCE1501E2F0E94AE7112969A
:1046D400EC91E03001F5AE81BF8153960E94C16E2A
:1046E400EE81FF81A189B289109751F00388148863
:1046F400AE81BF8151960E94EA7BE015F1050CF072
:1047040009C00E942F6D14DCE03011F00E940C727D
:104714000E9414720EC0E885F98534960E941C72BA
:104724000E94F5710E94D8700E94247253960E94D0
:104734004071E885F985A581AA232AF4A885B9855D
:1047440014960E944071A885B985EC91EC71EC3007
:1047540021F4E0911D08E078B1F4E885F985A4819D
:10476400B5815E971CF4A181A07209F404C0E885A8
:10477400F985A28106C00E940772F9DBE885F985F4
:10478400A381AA93F4DB0E94F871309791F0A88575
:10479400B98518960E94CB710E94F871309749F43C
:1047A4000E942F6DC5DBE03011F00E940C720E9454
:1047B40014720E94077211DCE03001F10E942F6D27
:1047C400B7DBE03049F00E940C72AA85BB85EC91FE
:1047D4000E945C710E94576DAA85BB851296EC916C
:1047E400E058AA85BB851296EC93E3E0E093240697
:1047F4000E940772E4DBEF73E0932506A885B98570
:1048040014960E94EA7B309761F52F5F323048F5A9
:10481400A885B98516960E94EA7B309789F0E885C9
:10482400F985A681B7810E942B72AA85BB85139650
:10483400ED93FC93A885B98516960E94407111C02A
:104844000E94DB71DF01E32FEF5FF0E00E94E06D77
:10485400E887F987A181EDEFEA23A885B985119648
:10486400EC933F5FA6CE233011F00C9488240E9471
:104874007133E03069F00E94E171E8E0EC93AA85BD
:10488400BB850E94EE71AA85BB85EC910E94FE71E6
:104894000E942F6D4DDBE03011F00E940C72AA854E
:1048A400BB85E0E0EC93EA85FB85A581ECE1EA2396
:1048B400E83061F50E941E6EAE2FEA85FB85E38D1C
:1048C400EA1741F4EA85FB85E48DE150EA930E94FE
:1048D40097171CC00E947133E030C1F00E94E1714F
:1048E400E3E0EC93AC85BD85EFEFEC931896EA8595
:1048F400FB85E38D0E943072AC85BD851296EA85F6
:10490400FB85E48D0E9430720E9434720F5F1ACED0
:104914000E943A7249F4A0911908A23021F0A830FB
:1049240011F0A53009F401C050C010E0153010F0AA
:104934000C94E7240E94AE7113965C915F3F11F4CE
:104944000C94E5240E94B871AE81BF81BD010E9420
:10495400BE71EE81FF8138960E941C720E944072E3
:104964000E9424720E94EA7BDF010E94C27DB4F49B
:10497400EE81FF81A681B7810E94C27D7CF4AE8165
:10498400BF810D901C90AE81BF8116960E94EA7B78
:10499400D001AE1BBF0B0E94C27D0CF014C0AE81CF
:1049A400BF81BD010D901C90EE81FF81A681B7816E
:1049B400F001EA1BFB0BDB01ED93FC935A93E5E05A
:1049C400EA930E94C5421F5FB1CFE0911C08E0301A
:1049D40041F4E0911608F0911708E0931408F0935D
:1049E40015080E94D37D2E9608950E94CE7DA09135
:1049F400C20BE091C30BE150EA9FF001EF5F1E2F61
:104A04002FE330E000911E08A091190CA13080F032
:104A1400E091190CE150A0911E08AE1728F0E09126
:104A2400190CE1503E2F04C0E091190CE2502E2FD6
:104A3400EC81E03049F1EF3F51F4A0911E08A11B35
:104A4400A31720F0E0911E08E11B0E2F1DC0EE3FBE
:104A540059F4E12FA0911E08AE0FA21720F4A091E3
:104A64001E08EA0F0E2F10C0EC3F49F4A091190C58
:104A7400A13020F0E091190CE1500E2F05C0AC815B
:104A8400A1501A9FF0010E2FE0911E08E01751F07B
:104A94000A930E949418A0918B0BAD3209F4032F52
:104AA40000931E080E94A146A0911908A83019F489
:104AB4000E94160F02C00E948F0E0E94D57D25967B
:104AC40008950E94CC7DFDD9E03111F40C94D525D4
:104AD40020E030E040E050E010E0133060F50E9448
:104AE40044720E940C6E0E94EA7B309711F10E947E
:104AF40047720E9461712E2B3F2B0E944772EA93EA
:104B04006CDAE03029F0E3E0E0932406E0E04CC006
:104B14000E944E720E9461712E2B3F2B0E944E7296
:104B2400EA935BDAE03029F0E3E0E0932406E0E086
:104B34003BC01F5FD2CF00E0053058F5A3E20A9FC7
:104B4400F0010E94827119F110E0133000F50E9407
:104B5400DB71DF010E948C710E945572AE0FBF1F82
:104B64001296EC910E9461714E2B5F2B0E94DB71B7
:104B7400DF010E948C710E945572AE0FBF1F139605
:104B8400EC910E9461714E2B5F2B1F5FDECF0F5F94
:104B9400D3CFF901E423F523309729F0E1E0E09342
:104BA4002406E0E001C0E1E00E94D37D269608954A
:104BB4001A93E091520CE03011F40C942F26E091FA
:104BC400E50BE13059F4A091520CA13311F4EFE05C
:104BD40001C0E0E0EA930E947C5E3FC0E23059F4F9
:104BE400A091520CA13311F4E6E001C0E5E1EA938F
:104BF4000E947C5E32C0E53061F4A091520CA13376
:104C040019F4E0919A0B01C0E0E0EA930E947C5E03
:104C140024C0E330B1F410E0173040F40E948C71EA
:104C2400E05CF64F0E945C721F5FF6CFA091520CBD
:104C3400A13311F4E1E301C0E0E3EA930E947C5E56
:104C44000CC00E946072E9E4EA930E94D662E0918B
:104C5400520C0E9467720E946C728FC422970E9449
:104C6400CC7D30E0A0911908A23029F0A83019F0C9
:104C7400A53009F021C1A985A03410F00C945D275A
:104C8400E0912F08E03009F417C1E9850E941870FB
:104C9400E03131F4E1E3E093520C8ADFE1E00CC14E
:104CA40021D9E03009F408C110E01530A0F4A3E2E2
:104CB4001A9FF001DF010E94827141F0FD01EB5562
:104CC400F94FE081AE2FE985EA1709F002C0E0E070
:104CD400F3C01F5FEACFF5DEE03011F40C945D27DA
:104CE40010E0A3E21A9FF001ED55F94FEE83FF8324
:104CF400AE81BF81EC91E03011F00C9456271396ED
:104D04000E94407100E0033010F00C942527A3E2C8
:104D14001A9FF001E855F94FDF010E94C46C0E940C
:104D2400E06DAF01DA0116960E9440710E94717223
:104D3400DA011296EC930E947872DA011396EC93DE
:104D4400A0919B0BEEEFEA23DA01EC930E947F72B1
:104D5400DA011196EC93B5D8E43139F0FA01A18166
:104D6400E2E0EA2BDA011196EC930A93D7D8E0300B
:104D740011F40C940727FA01A281AA9312D9E150E5
:104D84002E2F2F3F81F0A7E12A9FF001EF5CF94F0E
:104D9400A0E0A083A7E12A9FF001EE5BF94FA0E019
:104DA400B0E0A083B1830E9487720E940C6E0E94BF
:104DB400EA7BDA011496ED93FC93013040F00E94F3
:104DC40087720E940C6E0E94EA7B309709F00EC035
:104DD400AE81BF811596E02F0E94C56F0E94557267
:104DE400AE0FBF1F1196EC91E062EC93AE81BF81D0
:104DF4005A96EC91E062EC93023030F40E948A728D
:104E0400DA0116960E94307204C0DA0114960E94E8
:104E1400407157D8EC3019F4E0E0E0931D080E948B
:104E240091720E943270DA011896ED93FC93FA01A4
:104E3400A281A63030F0A181E4E0EA2BDA011196D8
:104E4400EC930F5F60CFA0911908A23011F0A53048
:104E540019F4A885AF3F08F007C0E0912F08EA9342
:104E6400EA85EA930E94C519E885AE81BF81EC9377
:104E7400E0912F08AE81BF811196EC93E985AE8154
:104E8400BF811296EC93A885A43138F4E8850E947A
:104E94005C71E15FFC4FA1E0A083AE81BF811696F7
:104EA400EC91ED7FEC9331E01F5F303011F415305D
:104EB40008F001C016CFE32F0E94D37D2A960895EF
:104EC4001A930A93A0911908A23011F0A53021F485
:104ED4000E9498720E94DC6EA0911908A830C9F44F
:104EE4000E949872E1E0EA930E940347E091E30B89
:104EF400E03069F4EA810E94A372E081EF771E2F0B
:104F0400ABE01A9FF001EA51FA4FA0E0A083689445
:104F140020F8198108812396089564970E94F86CFB
:104F2400A23039F4E0912F08EA93EB8DEA930E94C2
:104F3400C519A0911908A83011F00C9405280FEF99
:104F440020E0253050F4A7E12A9FF001EE5CF94FF0
:104F5400E081AE2FEA8DEA1709F402C02F5FF1CF8A
:104F6400A7E12A9FF001E15DF94FAF01DA0115963F
:104F74000C910F3F11F40C9405280E94A972108122
:104F84000E9414710E94C27DECF4ADE2BCE00E9468
:104F9400CB710E94AF720E94EB70A083B1831A930D
:104FA4000E94781EABE00A9FF001E252FA4F308172
:104FB4000A93FE0137960E94B5723A93FE01379622
:104FC4000E94B9720E94BF72F1F40E94A972AFEFFD
:104FD400A083DA011396EFEFEC93DA011596EC93C4
:104FE4000E94AF720E94C572E0E0F0E00E94F97086
:104FF400E0E0E0932A0C1A930E94781E0A930E9420
:105004007C10689420F80E94D37D6B9608951A93BF
:1050140010E01031B0F4A7E11A9FF001EC5BF94FF6
:10502400E081EF73AE2FE981EA1729F41A930E9405
:10503400EF1FE03009F403C0E1E01881E0C01F5F16
:10504400E8CFE0E01881DBC01A93E091550CF091B1
:10505400560CFA93EA93E4EFF1E00E940871F9F038
:105064000E94CA7210E01530D0F4A091590CAF5FC1
:10507400E5E00E94A07BE093590CEF5FEA93C7DF61
:10508400E03059F0E3E0E0932406E091590CF0E0BD
:10509400EF5FFF4EE093250670C21F5FE4CF6DC241
:1050A4001A93E0912306E093510CE8E7F0E0FA93B9
:1050B400EA93ECEDF0E0FA93EA930E94D24610E012
:1050C4001530D8F4E12FEF5FEA93A1DFE03099F0D7
:1050D4000E94566CE12FEA5FF0E00E941A6EEDEF39
:1050E400F6E10E94B86DA7EEBBE00E948C710E94AD
:1050F400E06D0E94E86D1F5FE3CF3FC2A5DFE09142
:105104002406E13029F4E5E0F7E10E94D1723CC0C5
:10511400E23029F4E2E1F7E10E94D17235C0E330D4
:1051240051F4EDEFF6E1FA93EA93E0912506F0E00D
:10513400E050F04F29C0E43019F4EAE1F7E11FC070
:10514400E53031F4E0912506EA930E94E31020C093
:10515400E63019F4E2E2F7E112C0E73029F4E8E2BC
:10516400F7E10E94D17210C0E83029F4E4E3F7E1DA
:105174000E94D17209C0E93059F4E3E4F7E1FA93EB
:10518400EA93E0912506F0E0FA93EA930E94001175
:10519400E0E0E09324060895A881B9811196E1E046
:1051A400EC930E941871A881B9811296ED93FC9337
:1051B4000E94681FA881B9811796EC930E941E6E05
:1051C400A881B98118960E943072E091C605A88121
:1051D400B981EC93E0912A0CA881B9811696EC93DD
:1051E400E0918A0BA881B9811A96EC93E091AD0BFA
:1051F400F091AE0BA881B9811496ED93FC9322969D
:10520400089564970E94CE7DA091E30BA230E1F44F
:10521400EB8DEA930E9494180E94681FADE2BCE0F3
:105224000E943072ABE2BCE0EB8D0E943072E091E0
:105234002F08E0932A0C0E941D70309721F00E94E1
:105244001D700E94037114C0AA8DAF3F09F4CAC037
:10525400EA8DEA930E94711EAB8DAF3F29F40E9440
:1052640018710E942270EB8FEB8DEA930E949418C0
:105274000E94681F0E2FA98DAF3F21F00E94741F5A
:10528400E03009F001C0AEC00E94EB700E94C46C13
:10529400AE17BF071CF015DCE13009F0A3C0A091E4
:1052A400D20BA03021F4A091E30BA23011F50E949F
:1052B4001E6EE13041F00E947133E03021F00E9413
:1052C4008733E03009F002C00E94D6720E941E6E3D
:1052D400E13021F40E947733E03009F409C00E94E0
:1052E400E272EE55F84FFA93EA9356DF0E94E872A1
:1052F40077C0EB8DEA93EA8DEA93B0DC1E2F113070
:1053040011F00C94F229A091D40BA13059F4E0913E
:105314002F08EA930E941871FA93EA93EFEFFFEFD4
:105324000E94EE720E94EB700E94C46C0E94D870BE
:105334000E94F970689420F8A091E30BA03019F44E
:10534400A88DAF3F09F437C00E94F272EE51FA4FB4
:105354000E94EB70A083B183E88D0E94C16D3081FF
:10536400E88DEA93FE0135960E94B572E88D0E949D
:10537400C16DE081EA93FE0135960E94B9720E94E4
:10538400631FE03131F00E94F272EA51FA4FA1E05A
:1053940005C00E94F272EA51FA4FA2E0A0830E9473
:1053A400F272EC51FA4FFF93EF930E948168AF9130
:1053B400BF91ED93FC930E94BF7219F4E0E0E09377
:1053C4002A0CEA8DEA930E94781EE0912F08EA9352
:1053D4000E941D700E94F772FA93EA930E94631C64
:1053E400E1E001C0E0E00E94D57D6C96089569DBA0
:1053F400E13041F40E947133E03021F00E948733A0
:10540400E03009F007C00E941D700E9403710E94E1
:10541400D6722FC337C30E94CE7D0E94FA721F3FFB
:1054240011F40C94642AE091520CE03011F00C94C5
:10543400632A1A930E949418E5E0E09324061093DB
:105444002506A0911908A23031F40E9403730E942A
:105454003521E03009F010C0A091530CA13331F490
:10546400E0912F08EA931A930E94C519E1E3E093AF
:10547400520C0E94D57DEBC2A0911908A830A1F46A
:105484000E941D700E9407730E2F0A930E94E93335
:105494003E2F1A930A93EFEFEA933A93B2DEE03089
:1054A40019F00E94D57DD3C2A0911908A53031F41A
:1054B4009EDFE03019F00E94D57DC9C2E0E3E0939D
:1054C400520C06C0E0E3E093520CE4E0E0932406BF
:1054D4000E94D57DBCC2E09140090E940B730895DF
:1054E4001A93E6E0EA930E947C5E0E946072A091A7
:1054F4004009A83539F4EFE4F7E10E941773E0E0BE
:105504000E946C72A0914009A33509F510E0A091A6
:105514001908A83021F0A23011F0A53009F411E3E4
:10552400E3E5EA930E94D6621A930E94D662E0E809
:10553400EA930E94D662E0E8EA930E94D662E0E829
:105544000E946772E093520CE0E00E946C72A0919A
:105554004009A93491F4A091E50BA43019F4E0E0DA
:10556400E093520C0E941B73E09325060E9425735E
:10557400EC91E093530C4FDF1BDB199108950E94CB
:10558400CE7DA0913F09A53411F00C94082B0E9404
:105594002A73E2E3F0E0E0934C0CF0934D0CA091FD
:1055A4004009A73741F4E4E4F9E00E9431730E9412
:1055B40036730E940B73A0914009A03310F0AA33F4
:1055C40008F023C02091270830912808E0E4F9E08E
:1055D4000E943173E2E0EA930E947D620E2F0E94E2
:1055E4003673E09325060E9436730E943A730E9434
:1055F400FA720A931A930E94C519209327083093CC
:105604002808E2E5EA930E947C5E1CC0E0914A0C03
:10561400F0914B0CFA93EA93E0914C0CF0914D0C01
:105624000E94087179F0E0E0E0933A09E5E4EA9336
:105634000E947C5E0E942A73E8ECF0E0E0934C0C3C
:10564400F0934D0C0E94D57D02C20E949A6D0E9477
:105654002E0E0E943F730E94566C0E94566C0E944C
:105664007A46A0911B08A23021F4E7E5F7E10E94F5
:10567400B86DA0911B08A13021F4EEE5F7E10E947A
:10568400B86DE0911B08E03021F4E5E6F7E10E94F3
:10569400B86D0E9449730E94826C0E947A460E94EF
:1056A4004C730E945173FA93EA93E0915F05F09171
:1056B40060050E9457730895E1E003C0E0E001C073
:1056C400E2E0E0931B08C1DF08950E94631FEC3100
:1056D40009F0D8C1E0919A0BE33631F4A09119088E
:1056E400A23009F4EBDF17C0E23631F4A0911908B7
:1056F400A23009F4E5DF0FC0A091C505A23011F076
:10570400A63021F4E0919A0BEA936FD9A091C505D4
:10571400A43009F4D1DFADC10E94EE6D0E94566C35
:105724000E94F26D0E94566C0E94566C0E947A464A
:10573400E8E7F5E00E94B86DE0911A080E945B73F7
:10574400E6E8F5E00E94B86DE2E0E0930E04089507
:105754000E944870E0ECF0E00E944F70E881E03075
:1057640009F406C0A0911A08AF5FE3E00E94A07B91
:10577400E0931A08E1E0E0934E0C0E9419206FC2F6
:105784000E94CE7D10E0103410F00C940F2C0E9477
:105794008C71ED55F94F30813F3FE9F11A930E9426
:1057A400941800E00E945F730E940C6E0E94EA7BD2
:1057B4003B9794F00E9462730F010E945F730E94F2
:1057C4000C6E0E9468730E946E730E941470EC91B8
:1057D400EE7FD001EC9301E00E9473730E940C6E83
:1057E4000E94EA7B759794F00E9462730F010E94F5
:1057F40073730E940C6E0E9468730E946E730E9401
:105804001470EC91E160D001EC9301E0013019F4E3
:105814001A930E94B4181F5FB6CF0E94D57D17C19A
:105824001A930A9323FE03C00E9476732CD70E9416
:10583400D542E030C1F1E0E00E947D73103820F5DC
:10584400113219F40E9476731ED71D3439F40E9464
:1058540084730E94F763E3E0E09318081B3271F449
:105864000E948973EAE2EA93E0E7F7E1FA93EA93A4
:10587400E0911A08E05DEA930E94F7631F3219F47D
:10588400E1E0EA93B2D848DF103868F00E948F73E1
:105894001A930E94F42019DFE03011F4103208F05A
:1058A40002C0E0E3F6E20E945E210E2F0038C8F148
:1058B4000F770034A8F5E0911F08E03031F00A9327
:1058C4000E945111E0E0E0931F08E0915A0CE017A8
:1058D40039F10A930E9494180E949971AC91A830EE
:1058E40028F40E949E71AC91A830A8F0E02FEF5FDD
:1058F400E093A2060A930E94F4200E949971EC910D
:10590400EA930E949E71EC91EA93E091A206EA93D5
:105914000E94F91E03C0E0E0E093A20600935A0C33
:105924000EC0A0915A0CAF3F51F0E091A206E030B6
:1059340019F0EA930E94161FEFEFE0935A0C0991B5
:1059440019910895A881A03310F0AA3308F01DC05E
:105954000E9493730E949873AAE0B0E00E94467B71
:10596400DF01E8810E949D73EA0FFB1FE093250885
:10597400F0932608E2E0E0930E040E9449730E942B
:10598400826C0E94F26D0E944C73A881A33451F47E
:105994000E943F730E9449730E94826C0E94F26DC0
:1059A4000E944C735CC11A930A93A0E023FCA1E00B
:1059B400A03019F0AA81A03009F016C0E89423F8A9
:1059C400E7E0E09318080E94BD45A0913108A0309B
:1059D40019F40E94A07309F407C0E7E0EA930E9457
:1059E400A57351D6E89424F824FE24C00E94A87319
:1059F400EAE5F0E00E94AF7319F0AA81A130C9F47E
:105A04006ED6E030B1F00E94B5730FEF1FEF0E9425
:105A140003730E940C21E03021F4009127081091B7
:105A24002808EB81EA93E0912F08EA931A930A93EA
:105A34002AD60BC00E94A873ECE2F1E00E94AF7377
:105A440021F40E94BC73E0933008198108812496E4
:105A54000895E091C80BF091C90B0E94C07311F432
:105A6400E2E00895E091C60BF091C70B0E94C07369
:105A740011F4E1E00895E091CC0BF091CD0B0E947C
:105A8400C07311F4E0E00895EFEF0895E0E0E093CF
:105A94001B08A0911908A23021F40E94A1460E947B
:105AA4008F0EA0911908A83009F44CD6A0911908BA
:105AB400A53009F443D10895E2E0EA930E94A1409D
:105AC400E2E0E0930E04E881EA933CDFA881AF377B
:105AD40021F4E0912B06E37009F403C0E2E0E093C3
:105AE4001808A881A13239F0A33421F40E949373D9
:105AF400109709F004C0A0911908A23009F00FC052
:105B0400A0911B08A33009F4DBDDA0911B08A2308F
:105B140009F4BCDFE0911B08E03009F4CFDDA88173
:105B2400AD3311F00C94ED2D0E94BD45E0911B089E
:105B3400E030A1F4E0912508F0912608FA93EA9365
:105B44000E943521E03041F4E0912508F0912608C7
:105B54000E943A739BDF01C0B1DD3DC0E13069F4BE
:105B640078DFEF3F41F0E3E00E94C4730E94847346
:105B74000E94CA7301C08ADF2EC0E230F1F40E9491
:105B84009373A034E0E0BE07B4F4E0912508EA93EF
:105B94000E94D173E2E0E0930E040E94566C0E94CE
:105BA400566C0E947A460E94AB6D0E94E40FE3E0BB
:105BB400E0931B0801C084DD0EC0E33061F4E09182
:105BC4002508EA930E949418E0912508EA93EEEFE1
:105BD400EA9344D875DDA881AD3409F46DDDA8815C
:105BE400A43521F4A0911908A23009F001C066DDA2
:105BF400A881AB3221F4EEEFEA930E94F724A88146
:105C0400AD3221F4EFEFEA930E94F724A881A73480
:105C140021F4E1E0EA930E94F724A881AB3421F453
:105C2400ECEFEA930E94F7241AC00E9491200E948C
:105C3400A146E0E0E0931B08A881A13039F40E945A
:105C4400A07321F0A091CB0BA03009F402C036DD83
:105C540006C00E948F0E0E9403730E940C2121969D
:105C640008951A930A930E94D5730E94431F0E94B9
:105C7400D542E03091F10E94DE7378F10E948F7377
:105C840024DDE03051F50E94E6730E94CA20EF3F04
:105C940009F0F6C40E9403730E943521E03021F418
:105CA4000E94741FE13009F018C00E94631FE8319C
:105CB40019F40E94EB7309F001C0E2C40E94E67378
:105CC4000E9430260E2F013021F4A0919A0BA030AF
:105CD40009F403C01A930E94E310A0912E06AF3F6B
:105CE40061F110912E06EFEFE0932E061A930E94B5
:105CF40094180E9403730E943521E03021F40E941D
:105D0400741FE13009F019C00E94631FE83119F4CF
:105D14000E94EB7309F001C0B3C41A93EEEFEA9347
:105D24000E9430260E2F013021F4A0919A0BA0304E
:105D340009F403C01A930E94E310A2C40E949120A4
:105D44000E941920E89421F8E0E0E0931E080E94E4
:105D5400F2730E94A1460E94566C0E94566C0E94E7
:105D64007A46E09132060E942F6EE09133060E943B
:105D74002F6E0E94566C0E94B36D0E947A46E09189
:105D84003F060E942F6EE0913906F0913A060E9478
:105D9400056E08950E94CE7D0E94D5730E94D5425F
:105DA400E03049F00E94DE7330F00E948F738DDC86
:105DB400E03009F41CDBE091570CF091580C0E9480
:105DC400E06E11F40C94462F0E94F2730E94566CFC
:105DD400E2E0F0E00E94F973E0913706F0913806B2
:105DE4000E94056EE0913B06F0913C060E94056E10
:105DF40000E0053010F00C94462FA7E10A9FF00153
:105E0400E15DF94F9F01F901A381AF3FD9F1D901B8
:105E14001A960E94116E7F936F93FF93EF930E94E3
:105E2400FC73AF91BF918F919F910E94087B0E9458
:105E34004B7BDF01CB010E940174D9011C96ED93C9
:105E4400FC93F90104841584D9011E960E94EA7B0F
:105E5400E015F105B9F0F90104841584A685B78528
:105E6400F001EA1BFB0BE093AD0BF093AE0BBFDA32
:105E7400E13041F4D9011C960E94EA7BD9011E96B7
:105E8400ED93FC930F5FB5CF0E94D57D1AC40E9499
:105E9400CE7D0E94D5730E94431F0E94D542E030FC
:105EA40011F40C94DF2F0E94D8420E2F0A9304DEC3
:105EB400003820F0A091C605A03808F429C00F7757
:105EC4000A930E9408740E9407731E2FA091E30B8B
:105ED400A03011F41F3F09F416C030E0353098F4B7
:105EE400ABE03A9FF001E452FA4FE081E11749F444
:105EF4003A9FF001E252FA4FE081EF5FE093C6056A
:105F0400232F3F5FEBCF0A930E94E6732A9354C07A
:105F1400A091E30BA03021F4003810F0053808F00C
:105F24000AC00F770E94A9721081EFEFEA930E94D2
:105F3400E6730A9366D9A091E30BA03011F0003800
:105F440008F43BC00F770A930E949418BEDBE0303C
:105F5400A1F50E940B740E94CA20EF3F19F00E9421
:105F6400D57DAFC30E94741FE13039F50E94681FCC
:105F7400E03049F40E940B740E943026E03011F0A6
:105F84000E9410741AC00E94631FE83141F40E94F9
:105F9400EB7321F00E940B740E9430260EC0A09176
:105FA4001E08E02F0E947E6DAE0FBF1F1C910A9346
:105FB4000E94E673EFEFEA9324D9A0912E06AF3F37
:105FC400F9F000912E06EFEFE0932E060A930E945B
:105FD40008740E9407731E2F0A931A93EEEFEA9334
:105FE400EFEFEA930ED91F3F41F4A0919E0BA0302E
:105FF40021F4A091A10BA03009F002C00E941074FA
:1060040020FE0AC0E89420F8E091E30BE03019F494
:10601400F1D342D501C0A1D530E0353080F5ABE0F5
:106024003A9FF001DF01EA51FA4FE081E03049F094
:10603400AC51BA4F0E941674E8EEF3E00E94087166
:1060440099F4ABE03A9FF001EA51FA4FE081E23073
:1060540051F43A9FF001EC51FA4FDF010E94EA7BC0
:106064000E94E06E09F409C0ABE03A9FF001EA51E6
:10607400FA4FA0E0A083689420F83F5FCECF0E943F
:10608400D57D1FC30E94F86CA33011F40C94FD312C
:10609400E0913A08ED3411F00C942631E0913B087C
:1060A400EA3511F00C94DB3024FC83C0E0913C0809
:1060B400E0532E2FE0913D08E0533E2FEEE3F8E04D
:1060C4000E9431730E942573AC91AB3429F40E9471
:1060D4001B740E9409620E2F0E942573AC91A43593
:1060E40029F40E941B740E940962AF01E091CE0B57
:1060F400E31731F5E0E0E093500C0E94B573409350
:10610400270850932808A09130080A1759F0E7E0AF
:10611400E09318080093300820934F0CE0E0E093DC
:106124002F080DC0A0914F0C2A1721F0A0912E0822
:10613400A03009F004C02093180820934F0C35C0F8
:10614400A0913008A03049F4A091CF0B0E94DC6CE0
:10615400E255FF4FE491EA2309F40CC0E7E0E09331
:10616400180820934F0CE0E0E0932F08E0913908E1
:10617400E093500CE0913908A091500CEA17A9F46F
:106184004093270850932808009330080E94B57361
:10619400A0914F0C2A1721F0A0912E08A03009F0ED
:1061A40004C02093180820934F0C273011F40E9448
:1061B4002D71E0913B08E93439F4E7E00E94C4739F
:1061C4000E94BC73E0932F08E0913B08E23439F459
:1061D400E4E00E94C4730E94BC73E0932F08E09132
:1061E4003B08E03519F4E1E0E0931808E0913B083E
:1061F400EC3449F4E4E0E0931808E0913C08E053FF
:10620400EA930E94B915E0913B08E334E9F4A091C4
:106214003C08A13320F0A0913C08A93308F014C035
:106224000E941E74E0912208EA930E94E01AE09111
:106234003908EA93E3E7F7E1FA93EA930E9453708B
:106244000E94FD7B0E94EA63E0913A08E03521F464
:10625400A0911908A13009F003C00E9489735CDA87
:10626400E0913A08EF3459F4E0913B08EE3439F404
:10627400E0913908EA93E6E7F7E10E942474E0919B
:106284003A08E33569F5E0913B08EF3349F5A0910D
:106294003C08A03320F0A0913D08A03308F420C0AE
:1062A4000E941E74E0913D08E0531E2FA091220825
:1062B400A63010F41A3008F013C0103011F40E9404
:1062C4002A1AE0913908EA93E9E7F7E1FA93EA93A5
:1062D4000E9486700E9469700E94FD7B0E94EA639E
:1062E400E0913A08E33411F00C94C531E0913B0895
:1062F400EF3311F00C94C531E0913D08E03319F40B
:10630400EFEFE0932308A0913C08A033F8F00E943B
:106314001E74A0912208A630C8F4E0912308EF5F10
:10632400E0932308E0912208EA93E0912308EA939A
:106334000E94A61AA0911F0CB091200C109721F472
:10634400A0912308A03408F001C0E7CFE09123080E
:10635400EA930E9494180E942A74ECE7F7E10E94E1
:1063640017730E94236F0E942F740E9434740E943A
:10637400286F0E94FD7B0E9434740E94906F0E94DB
:106384006F630E94BC63E0913A08E434A1F5E091A4
:106394003B08E43481F514E0E1E0E0933909103579
:1063A40038F40E948C71E85CF74FE081E03208F425
:1063B4001AC00E948C71E85CF74FE081E33259F413
:1063C4000E948C71E75CF74FE081E053EA930E94EE
:1063D4007C5E1F5F06C00E948C71E85CF74F0E94D0
:1063E4005C721F5FDCCF0E942A74EFE7F7E10E9422
:1063F40017730E94BC630E94D37D269608951A9356
:106404000A930E943A7211F40C946F32E0E0E09324
:106414005C0CE0911808EF770E2F009318080E9487
:10642400A1460E94B36D0E94B56C0E947A46013069
:1064340021F0A0911908A13009F00DC0EEE8F5E0B3
:106444000E94B86D9DD9E4EFF1E0FA93EA930E94BB
:10645400F3420E94A146073049F40E949120E0E0F3
:10646400E0931B080E9484110E945228043031F4E6
:10647400E2E8F7E10E94B86D0E94440D083019F477
:106484000E943A745FD1053019F40E943A7456DCC4
:10649400013039F40E944774009319083DD90E94D1
:1064A4008F0E093059F40E9447740E948F0E0A938C
:1064B400E1E0EA9378DAE1E0E0935C0C023029F45D
:1064C4000E943A74E1E0EA93B0DB033011F40E94D5
:1064D4005340009319080E94431FA0911908A73044
:1064E40011F00C941B33E091550CF091560C0E9462
:1064F400E06E21F0A0911B08A03009F00AC00E94B0
:10650400CA72E091510CA0912306EA1711F00E947F
:1065140052280E94D542E030E9F0E2E00E947D7307
:106524001A9310DA1D3409F4C7D81D3399F40E9464
:10653400BD458FDAEF3F41F0E3E0E09318080E9495
:1065440084730E94CA7306C0E7E8E0931808E0E089
:10655400E0931B08A0912F08A03031F0E0912F08A0
:10656400A0912E08EA1709F455C0E0912F08E150D4
:10657400EA930E94E918A091350CE1E0EA23E130A6
:1065840021F4E0912B06EF7C09F429C0E0E0E093CC
:106594002E08E0914F0CE03019F0E09318081EC06B
:1065A40012E0E0912B06EC7009F018E0E091C50BC5
:1065B400A0912F08EA1781F0E0912B06E07439F0DE
:1065C40011E0EAE2EA93E7E8F7E10E942474E0913B
:1065D4002B06E07809F019E0109318081BC00E94FC
:1065E400A1460E9484110E94B36D0E94B56C0E9462
:1065F4007A46EBE4EA930E941446E0912F08EA936A
:106604000E944241EAE8F7E10E94B86DE0912F0848
:10661400E0932E08A0912F08A03021F4A0912E0819
:10662400A03009F406C0E0E0E0932E08E7E8E09328
:106634001808A0911908A33011F40E94553EA091A6
:106644001908A13009F4ECD8A0911908A23009F472
:1066540008DBA0911908A83009F419DCA0911908E5
:10666400A53009F497DBA0911908A93049F4E0E0BA
:10667400E0932008E0911908EA93E0E0EA9393D9C3
:106684000991199108950E945274E652F84FA6E0B8
:10669400A0830E945274E752F84FAB81A0830E94FA
:1066A4005274E152F84FAA81A0830E945274E552B9
:1066B400F84FA881B981A083B1830E9434720E94EB
:1066C400DA50249608950E945874A881B981AC9137
:1066D400A53020F0A881B981E0E0EC9389C0A091B5
:1066E4001308BB27E091120805C0A0911108BB272D
:1066F400E0911008F0E031960E94D8703596DF01E1
:10670400E5E0F0E00E94A37B08951A93109113082A
:10671400E0911208E117A1F0ABE01A9FF001E652F4
:10672400F84FE081E13011F0E23011F4E1E04DC0C6
:10673400EDB7FEB7FA93EA931F93C5DF1F91E8CF35
:10674400E0E043C01A930E949120ECEDF5E00E9432
:106754009D700E94246D0E940B6910E0153068F44E
:106764000E940E71AFEFA083ABE01A9FF001EE51CF
:10677400FA4F0E94C5721F5FF1CF10E0153048F444
:10678400A7E11A9FF001EC5CF94FAFEFA0831F5F04
:10679400F5CFE0912B06E37019F00E94A07309F481
:1067A40002C0689401C0E89421F8EFEFE0932D084B
:1067B400E091E30BE03029F41DD06ED1E89420F889
:1067C40004C00E94A1460E94160F199108951A93BD
:1067D40010E0153058F40E940E71E081AE2FE9816B
:1067E400EA1711F4E12F03C01F5FF3CFEFEF188115
:1067F4002296089522970E94CC7D00E0053058F43B
:106804000E945E74A0E00E946474E152FA4FA0E01A
:10681400A0830F5FF3CF00E00530C0F50E94A9729A
:10682400E081EF3F89F10E94A972E0810E941D710D
:10683400B9F00E94AF72DF010E94EA7B0E94EB7004
:10684400EA17FB0751F00E94AF720E94EB70A0831D
:10685400B1830E946974A1E0A0830E945E7412C097
:10686400ABE00A9FF001EA51FA4FE081E03061F4B5
:106874000E94A972AFEFA0830E94AF720E94C572FA
:106884000E946974A1E0A0830F5FC6CF0E94631EBB
:106894001E2F1F3F11F0E1E001C0E0E0E0935C0C2B
:1068A4001F3F11F40C94A83450E000E0053048F484
:1068B4000E94A972E0811E1711F451E002C00F5F1B
:1068C400F5CF5030E1F500E00530C8F50E94A9721B
:1068D400E081EF3F91F50E94A97210830E94AF728C
:1068E4000E94EB70A083B183ABE00A9FF001E052F9
:1068F400FA4FA0912A0C0E946474EF51FA4FFF934F
:10690400EF930E9418710E942270AF91BF91EC9393
:106914000E946974A1E0A0830E945E74A1E00E94B9
:106924006474EC51FA4FFF93EF930E948168AF9126
:10693400BF91ED93FC9351E002C00F5FC5CF50307F
:1069440029F01A930E946A1E1E2FAACF30E0353018
:1069540010F00C94EE34A7E13A9FF001E15DF94F99
:10696400EE83FF8350E000E0053048F5503029F510
:10697400ABE00A9FF001EF51FA4F20812A930E9465
:1069840094180E945E74E081E13059F42A930E94C5
:10699400841FE13031F4A32FAF5FE0919E0BEA171F
:1069A40009F00BC0E22FAE81BF811396EC93E02F68
:1069B400AE81BF811596EC9351E00F5FD5CF503077
:1069C40049F4AE81BF811396EFEFEC93AE81BF81A2
:1069D4001596EC933F5FBBCF0E94D37D0C94963702
:1069E4000E94CE7DAC81BD81EBE4EC93EC81FD8112
:1069F4003196FA93EA930E946F74E052FA4FE08161
:106A04000E949C6C00E00E947874EC91E03011F0DC
:106A14000F5FF9CF0E947874E0E2EC930F5F0E945D
:106A24007E740E94526D0E946F74EE51FA4FDF0122
:106A34000E94116E0E948374EE81ABE0EA9FF00124
:106A4400EF51FA4F10811A930E94941800E00E94AB
:106A54007874EC91E03011F00F5FF9CF0E947874F4
:106A6400E8E7EC930F5F0E947874E0E2EC930F5F29
:106A740030E03A3060F40E947E74EA0FFB1F0F018D
:106A8400ABE8BBE00E948A740F5F3F5FF2CF0E94C5
:106A94007874EC930C94DB3764970E94CE7D00E00D
:106AA40010E0153040F40E940E71E081EF3F09F4CC
:106AB4000F5F1F5FF6CF053021F0A0912D08A030A5
:106AC40009F406C0E0E0E0932D08EA930E94311037
:106AD40010E0153088F5ABE01A9FF001E152FA4F4F
:106AE400E081E03039F11A9FF001E352FA4FE0817E
:106AF400E030B1F01A93FE0135960E94B572ABE016
:106B04001A9FF001EF51FA4F30813A930E94941882
:106B14001A93FE013596FA93EA930E948C100AC0E8
:106B24001A930E947C10ABE01A9FF001E152FA4FD5
:106B3400A0E0A0831F5FCDCF053021F4A0912D08E4
:106B4400A13009F406C0E1E0E0932D08EA930E9425
:106B540031100E94D57D689608950E94CC7DA09145
:106B6400E30BA23011F40C94753930E0343168F43D
:106B74000E9491740E949574DA011296E0E0EC93FD
:106B8400DA01EFEFEC933F5FF1CF0E94631E0E2F0B
:106B94000F3F11F0E1E001C0E0E0E0935C0C0F3F37
:106BA400A1F10E941871FA93EA930E9444181E2FCF
:106BB4001F3F31F1A0911E08E12FEA1B3E2F343113
:106BC400F8F40E9491740E949574FA0132960F01B0
:106BD400E081AE2F0E949B74B0E0EA0FFB1FD0014E
:106BE400EC93FA01A281A43620F0DA011296E3E6CE
:106BF400EC93DA01AC91AF3F19F4E02FDA01EC9396
:106C04000A930E946A1E0E2FCACF0E94C81430E055
:106C1400343110F00C9494360E9491740E9495744F
:106C2400FA01A381AF3F11F40C9492360E94A07430
:106C34000E941870E83139F40E94A074EA930E940B
:106C44008D17E03009F408C00E94A074EA930E94F2
:106C54008D17DA011296EC93A0919B0BA07839F46E
:106C6400FA010280DA011196EC91E01509F458C09A
:106C7400DA0113962C91ADE02A9FF001EF5EFC4FF0
:106C84000F01DA011296EC91D001EC930E94A074EA
:106C9400EA930E94A720EF3F29F0ADE02A9FF0017C
:106CA4000E94576DDA011296EC91E03089F00E944F
:106CB400A574DF010E94796DEC93ADE02A9FF00189
:106CC400E25FFC4FDF01E091990BEF70EC9313C08E
:106CD4000E94796DE03021F40E94A574A0E003C005
:106CE4000E94A574A8E0A083ADE02A9FF001E25FB2
:106CF400FC4FA7E0A0830E94A074EA930E94A720FF
:106D0400EF3F19F0ECE0E0930F04DA011296EC91F6
:106D1400DA011196EC932A93E1E0EA930E94034787
:106D24003F5F76CF0C947539E7E0E09318080E9432
:106D3400CF17A8950E94271CA8950E947F1EA8958E
:106D4400EFEFE093B30BE0938A0BE093340CE09302
:106D54002F0CE0932E060E94AB74EC7F29F0A8E080
:106D6400B0E0E0E00E942C7C089524970E94CE7D40
:106D74000E94F041E8E9F7E10E949D700E947C4284
:106D84000E941842E0912208E03061F0E3EAF7E162
:106D94000E949D700E947C42E09122080E94B0747F
:106DA4000E94B4740E9418420E942A1A00E00A3019
:106DB400A0F40A930E94C3180E94B66FEFE0EA930E
:106DC4000E945642E02FA3EAB6E00E94B8740E94E3
:106DD40069700E94BC740F5FEACF0E942A42ECEAF9
:106DE400F7E1FA93EA93EFE0EA930E947C420E946F
:106DF400F06E0E94BC740E942C420E94184210E063
:106E0400103110F00C9492370E941E6EE117E1F5D8
:106E1400E2EBF7E10E949D700E947C420E949F6D0C
:106E24000E94B474E0E0E0931E08A0911E08A03410
:106E340048F5E0912208EA93E0911E08EA930E9443
:106E4400A61A0E94236F3097B9F0E0911E08EA93C6
:106E54000E9494180E94236FFA93EA930E94C274CA
:106E64000E947C420E94906FEAE0EA930E9456429C
:106E74000E94286F0E94BC74E0911E08EF5FE093AB
:106E84001E08D3CF0E94C7740E948C710E946E703A
:106E940011F00C949037E2EBF7E10E949D700E9490
:106EA4007C420E949F6D0E94B4740E94CB74E0E304
:106EB4000E947A7029F40E947F700E9409629F01E7
:106EC40000240216030644F50E941B740E943362D8
:106ED4000E94936E0E941B740E94D3743A932A9367
:106EE4000E94C2740E947C420E94D774EAE0EA9332
:106EF4000E945642EC81FD816E817F810E94BC74A8
:106F04000E94CB74E1E30E947A7029F40E947F709E
:106F14000E9409629F01D4CF0E94C7741F5F70CF83
:106F24000E94F1410E94D57D289608950E94CE7D4D
:106F3400AD81BE812C910E94DC740E949F6D0E94E1
:106F4400C46C0E941A6EECE3EA930E941446EC812E
:106F5400EA930E946C462A93ED81EA930E94E240F0
:106F6400EEE3EA930E9414460E9451730E94F77262
:106F74000E9457730E94E174333409F431E23133CF
:106F840020F0EC81E05DE31708F407C0E32F0E94D2
:106F94009D73E255FF4FE4912E273D3311F03132BA
:106FA40009F401C0CACF3D3319F4AD81BE812C93DD
:106FB400E32F0E94D57D279608950E94CC7D20E082
:106FC400AF81B8855C910E94DC740E949F6D0E9421
:106FD400C46C0E941A6EE2E0EA930E946C465A93D3
:106FE4000E9442410E9451730E94F7720E9457739B
:106FF4000E94E174303310F03A3308F00EC02030B0
:1070040009F450E021E0A52FEAE00E94A07BAAE069
:10701400EA9FF001E30FE0535E2F3B3211F4533645
:1070240008F001C05F5F3D3211F4513008F401C033
:107034005150333429F4203009F431E250E020E097
:107044003D3319F4EE81E51708F005C0AF81B8852A
:107054005C9130E020E03D3311F0313209F401C09D
:10706400B4CF3D3319F4AF81B8855C93D0C00E948E
:10707400CC7D20E0AF81B8854D915C910E94DC7499
:107084000E949F6D0E94C46C0E941A6EAE81A23051
:1070940051F4E6E0EA930E946C46FA010E942F74D0
:1070A4000E94214108C0E5E0EA930E946C465A938D
:1070B4004A930E942C410E9451730E94F7720E94CD
:1070C40057730E94E174303310F03A3308F01EC055
:1070D400203011F440E050E021E04031E7E25E0767
:1070E40034F0DA01E0E1F7E20E94A37BAF01493B0F
:1070F400EBE05E0724F0DA010E949873AF01DA0135
:107104000E94E6740E94EB74D097AD013B3221F4E7
:107114004033E5E75E070CF002C04F5F5F4F3D323E
:1071240021F40024041605060CF002C0415050401E
:10713400333431F4203009F431E240E050E020E00F
:107144003D3311F0313209F401C09ACF3D3321F4BB
:10715400AF81B8854D935C935AC00E94CC7D0E9448
:10716400DC7420E050E04FEF0E949F6D0E94C46CDD
:107174000E94F9730E94F074E885EA930E944246E3
:10718400E52FE10FF0E00E94F7720E9457730E940E
:10719400E174303310F03A3308F021C03053431710
:1071A40029F04F3F09F05F5F20E005C0A22FAF5FD9
:1071B400EA2FE3702E2FE52FAF81B8850E94F57476
:1071C4000F01E32FACEBB6E00E94B874AE0FBF1F03
:1071D400E22F0E94F574E491D001EC93432F3B32EB
:1071E40019F4EE815E1708F002C05F5F4FEF3D3285
:1071F40011F4513008F402C051504FEFEE815E1784
:1072040020F4313211F03D3309F401C0ADCFE32F46
:107214000E94D37D299608951A930A93A0919B0BFB
:10722400ECEDEA231E2F00E00D3040F40E94F974C7
:107234000E94FD74E11711F00F5FF6CF0E94F974FC
:10724400EA0FFB1F0E94F97B0E94B86DE02F45C432
:10725400ABE9BBE00E94096EAE0FBF1FEC91E17079
:1072640011F4E3E701C0E9E4EA930E94144621968D
:1072740008950E94CC7D0E94DC740E949F6D0E9440
:10728400C46C0E94F973C8DF5E2F0E9451730E9480
:10729400F7720E9457730E94E1743D3211F0363345
:1072A40011F4503009F401C051503B3211F0333322
:1072B40011F45C3008F001C05F5FA0919B0BE1E02A
:1072C400EA232E2FE52FA0E0B2E00E94B8740E94BA
:1072D400FD74E20FE0939B0B3D3311F0313209F45E
:1072E40001C0CBCFE32F0E94D37D269608950E9440
:1072F400CE7D0E94DC740E949F6D0E94C46C0E942B
:10730400F973ABE9BBE0EC810E941470EC91E1707D
:1073140019F4EFEBF7E102C0E3ECF7E1FA93EA9337
:107324000E942B460E9451730E94F7720E94577369
:107334000E94E174303310F03A3308F00FC0ABE927
:10734400BBE00E9438700F01ABE9BBE0EC810E9406
:107354001470AC91E1E0EA27D001EC933D3311F0D5
:10736400313209F401C0C7CFE32F0E94D57D2596A1
:1073740008950E94AC6CE1E0EA930E942E0E0E94F4
:10738400566C0E94566C0E947A460E94906FEAE006
:10739400EA93E3DEE13209F469C40E94566C0E9468
:1073A400566C0E94F26DE7ECF7E10E94B86DE6E9D5
:1073B400FBE00E949D705BDEE13209F457C40E9439
:1073C400566C0E94566C0E94F26DEDECF7E10E943F
:1073D400B86DE091980BEF5F0E2FEDB7FEB7FA93FF
:1073E400EA930F93EAE0EA93E8DD0F91E13209F4BE
:1073F4003DC400240216030624F4E02FE150E09378
:10740400980B0E94566C0E94566C0E94F26DE6ED39
:10741400F7E10E94B86DEDEAFBE00E94027509F401
:1074240025C40E94566C0E94566C0E94F26DECEDCD
:10743400F7E10E94B86DEFEAFBE00E94027509F4DF
:1074440015C40E94566C0E94566C0E94F26DE2EEC6
:10745400F7E10E94B86DEAE9FBE0FA93EA93E3E608
:107464000E940B7509F402C40E94566C0E94566C6B
:107474000E94F26DEBEEF7E10E94B86DFADEE132A4
:1074840009F4F4C310E0133010F00C94003B0E9494
:10749400566C0E94566C0E94F26DE12F0E945B7341
:1074A400E1EFF7E10E94B86D0E9410750E947A46E0
:1074B400AEE9BBE00E948C710E94526DE0E10E9433
:1074C4000B7509F4D3C3E9E0F0E00E94826C0E94DA
:1074D4007A46A1EABBE00E948C710E94526DE0E101
:1074E4000E940B7509F4C2C30E94566C0E94566C2C
:1074F4000E94F26DE12F0E945B73ECEFF7E10E94B2
:10750400B86D1A93F4DEE13209F4B0C30E94107529
:107514000E94147551F40E9444720E941E75E2E0A8
:107524000E94227509F4A2C309C00E9444720E94F9
:107534001E75E0E00E94227509F498C30E94566CFF
:107544000E94566C0E94F26DE12F0E945B73EEEF75
:10755400F7E10E94B86D0E9410750E947A46AAEA6B
:10756400BBE0EE27A10FBE1F2C913327EDB7FEB76A
:107574003197FA93EA933F932F93E0E0EA9377DD10
:107584002F913F91E13209F471C3AAEABBE00E9452
:107594008C71EA0FFB1F2083123070F50E94566C29
:1075A4000E94566C0E94F26DE12F0E945B73E5E02D
:1075B400F8E10E94B86D0E9410750E947A46A1EB12
:1075C400BBE0EE27A10FBE1F2C913327EDB7FEB70A
:1075D4003197FA93EA933F932F93E0E0EA9347DDE0
:1075E4002F913F91E13209F441C3A1EBBBE00E942A
:1075F4008C71EA0FFB1F20831F5F45CF37C30E94A6
:10760400CE7D10E01A930E94D1730E9427750E94C8
:10761400566C0E947A460E942A6E0E942B750E9424
:10762400AB6D0E941D700E94056E0E94566C0E94F4
:10763400B36D0E947A460E942B700E94166EE7E09A
:10764400F0E0FA93EA930E94B36D0E947A46E091C7
:10765400AF0BF091B00B0E94087B0E94166E0E9443
:10766400566CE2E0F0E00E941A6EECE0F8E10E9451
:10767400B86DE091980BEF5FEA930E944241E7E016
:10768400F0E00E94A46D0E947A46C6DD0E94F66D69
:10769400E0919A0BE03029F0E0919A0BEA930E9472
:1076A400424100E00330D8F50E94566CE02FED5FB4
:1076B400F0E00E941A6E0E947172EA930E944241A5
:1076C400EBE2EA930E9414460E947872EA930E94C5
:1076D40042410E94F66D0E947F7251F40E948772AB
:1076E4000E940C6E0E94116E0E942F75E3E709C080
:1076F4000E9487720E940C6E0E94EA7B0E94056EB3
:10770400E9E4EA930E9414460E94F66D0E94917285
:10771400EA930E9448410E9433750F5FC3CF0E94D1
:10772400D8423E2F3B3211F4103408F001C01F5FE1
:107734003D3211F4113008F401C011503D3439F4D4
:107744001A930E94941815DE1A930E94B4183132C9
:1077540009F058CF8BC20E94CE7D10E00E94A14652
:10776400012F0E94566C0E94566C0E947A46E0E1FA
:10777400F8E10E94B86D31E03C3018F51038F8F4A7
:107784000E94566C0E94DC6C0E941A6E1A930E942E
:10779400E9180E942A6E0E94F66DA091350CE3E070
:1077A4000E943775A091360CE7E00E943775E0918E
:1077B4002B06EA93E8E0EA930E94E24013953F5FC8
:1077C400DBCF0E94440D0E94D8423E2F3D3411F07D
:1077D4000C942B3C0E949A6D0E942E0E102F103890
:1077E400C0F51A930E94E9180E94566C0E94566CC8
:1077F4000E94F26DE4E2F8E10E94B86D0E942A6EE4
:107804000E942B750E94316E0E947A46E7E2F8E1ED
:107814000E94B86DE5E3FCE0FA93EA93E3E00E948A
:107824000B7509F423C20E94316E0E94F26DEDE2E1
:10783400F8E10E94B86DE6E3FCE0FA93EA93E7E02E
:107844000E940B7509F412C21A930E941B191F5F40
:10785400C6CF313211F0103808F001C07FCF06C214
:107864000E94AC6C0E9427750E94566C0E947A4656
:10787400E3E3F8E10E94B86D10E01530F0F41A93D8
:107884000E9427190E94566C0E94066F0E942A6E5D
:107894000E942B75E091300C0E943C75E091330CF2
:1078A4000E943C75E091310C0E943C75E091320CD1
:1078B400EA930E9448411F5FE0CF0E94D8420E2FF6
:1078C4000D3411F00C94A53C0E949A6D0E942E0E6A
:1078D40010E01530C0F51A930E9427190E94566CC7
:1078E4000E94566C0E94F26DE6E4F8E10E94B86DC5
:1078F4000E942A6E0E942B7530E03430F8F40E9406
:10790400316E0E94F26D0E94DC6C0E94FB7AE45698
:10791400F94F0E94F97B0E94B86D0E94DC6C0E94B2
:10792400FB7AE456F94F0E944075FD013596E491C7
:107934000E940B7509F49AC13F5FDFCF1A930E942E
:1079440047191F5FC6CF92C11A930A930E94A1469A
:10795400E1E0EA930E942E0E00E0083210F00C944D
:107964006F3D0E94100D0E94566C0E94566C0E943E
:107974007A460E94C46C0E9443750E94F97B31963A
:107984000E94B86D0E94F66D0E94C46C0E944375FB
:107994003496E491E038A9F40E941E6E1E2FEDB7D0
:1079A400FEB7FA93EA931F93E0E1EA9306DB1F9193
:1079B400E13209F492C0E12FA9E0B0E00E942C7CEE
:1079C40088C0E238A9F40E94A2701E2FEDB7FEB75A
:1079D400FA93EA931F93E0E1EA93EFDA1F91E1321D
:1079E40009F47BC0E12FAAE0B0E00E942C7C71C0B6
:1079F400E138E1F40E94AB741E2FEDB7FEB7FA93A1
:107A0400EA931F93E3E0EA93D8DA1F91E13209F491
:107A140064C00E94100D0E94AB74E11731F0E12F95
:107A2400A8E0B0E00E942C7CFFCF53C0E03069F4A2
:107A34000E94C46C0E94437532960E94BC6DE1E0C2
:107A44000E940B7509F449C044C0E13069F40E94F6
:107A5400C46C0E9443750E944075FD013596E49103
:107A64000E940B75D1F135C0E23061F40E94C46C00
:107A74000E94437532960E94BC6DEFE00E9422750D
:107A840061F127C0E33071F40E94C46C0E94437515
:107A94000E944075FD013596E491EA9347DAE1329C
:107AA400E1F017C0E430A9F40E94C46C0E9443754D
:107AB40032960E94F97BE0935D0CF0935E0C0E9479
:107AC400F7720E9443753596E491EA9346DBE132FE
:107AD40021F00E94D2170F5F40CF099119910895A8
:107AE400E8810E945B73EAECF7E10E94B86D0C94A4
:107AF400EE411A930E949A6D0E942E0E10E01330EC
:107B040010F00C94D63D0E94566C0E94566C0E9454
:107B1400F26D1A93E5DFECE0F0E00E94826C0E94C3
:107B24007A461A9395DB0E9410750E94147551F4DD
:107B34000E9444720E941E75E2E00E94227509F4BC
:107B4400FCC209C00E9444720E941E75E0E00E94BB
:107B5400227509F4F2C2123028F50E94566C0E9474
:107B6400566C0E94F26D1A93BBDFE9E4F8E10E94BF
:107B7400B86DECE0F0E00E94826C0E947A460E94AC
:107B84003375EAE0F0E00E94826C0E947A46A1EB31
:107B9400BBE00E948C710E94526DE3E60E940B755B
:107BA40009F4CBC21F5FABCFC8C20E94CE7D10E0E8
:107BB4001A930E94D1730E9427750E94566C0E94EA
:107BC4007A460E942A6E0E942B750E94AB6D21E0BA
:107BD40000E0033080F5E3E0F0E00E94F36C0E94E3
:107BE4001A6E0A937DDF0E947F7249F40E948772A5
:107BF4000E940C6E0E94116E0E942F7508C00E9494
:107C040087720E940C6E0E94EA7B0E94056E0A93A2
:107C14001FDB2F5F023068F4E7E0F0E00E94F36CB2
:107C24000E941A6E0E948A720E942F6E0E943375FF
:107C34002F5F0F5FCECF0E94D8423E2F3B3211F40C
:107C4400103408F001C01F5F3D3211F4113008F404
:107C540001C011503D3439F41A930E94941849DF3D
:107C64001A930E94B418313209F0A2CF0E94D57D34
:107C7400249608950E949A6D0E942E0E0E94566CBE
:107C84000E94566C0E947A46EFE4F8E10E94B86DB7
:107C9400E1E0E0932208E2E2F8E0FA93EA93E5E017
:107CA400EA938BD9089522970E94CC7D0E94D842F2
:107CB4000E2FE0911B08E03011F00C9401400132CA
:107CC400D1F4E2E4F6E0A0913B0CB0913C0CEA174D
:107CD400FB0761F4E7E0E0931808EAE2EA93E8E5D9
:107CE400F8E10E949D700E94F763A9C0E0E0E09370
:107CF400C0050E9448750D3331F4E091C005F0E0F1
:107D04000E94E26C04910D3441F4EAE2EA93EBE55B
:107D1400F8E10E949D700E94F763063449F4EAE694
:107D2400F6E0E0933B0CF0933C0CE0E0E093C005FC
:107D3400003311F00B3229F4E091C005EF5FE093BA
:107D4400C0050D3229F4E091C005E150E093C0056F
:107D5400013329F48FDFED3311F40E944F7503339F
:107D640029F488DFED3311F40E94B736063329F481
:107D7400E0E0E09322080E94B736043329F4E0E0FF
:107D8400E09322080E944F75A0912408A13010F4BA
:107D94000C949B3F023301F56DDFED33E9F40E944F
:107DA4005C75D1F4E0912208EA930E94E01A30E075
:107DB400303190F40E94DC6C0E946E7059F4E32F11
:107DC400E05DEA93EEE5F8E10E947370E0E3EA9384
:107DD4000E9419643F5FECCF053331F5E0E0E09396
:107DE40022080E945C7501F511E01630E8F41A933C
:107DF4000E94E01A30E03031A8F40E94DC6C0E944A
:107E04006E7071F4E32FE05DEA93EEE5F8E1FA9326
:107E1400EA93E12FE05DEA93E0E3EA930E941964B8
:107E24003F5FE9CF1F5FE1CF013469F4EAE2EA93EF
:107E3400E1E6F8E10E942474E1E0E09318080E946E
:107E4400D37D289608950A3409F4AFDE073311F080
:107E54000C949B3F0E949A6D0E94720DE1E0E093A6
:107E64001C08E0E0F0E0E0931408F0931508EFE25A
:107E7400F6E00E949D70E3E7F0E00E944F700E94DC
:107E84008168EE83FF830E946575E8E2F0E00E945A
:107E94000871B9F00E94C7110E948168EE83FF83C4
:107EA400A0911A0CA03021F00E947133E03009F443
:107EB40008C00E945274E652F84FAEE0A0830E94BC
:107EC40034720E946A750E94F34240E050E00E94BE
:107ED4005E21E03868F00E945E21EF573E2F31307A
:107EE40010F0313108F004C0E32F0E946171AF013A
:107EF4005A934A930E941D1F4093140850931508E7
:107F04000091DB05E0E0E093DB05013211F00B3278
:107F140009F401C0B8CF0B3221F4E1E0EA930E94E6
:107F2400720D013209F0A3CFE0E0E0931C08E09366
:107F3400DB05A0912408A23011F00C94FA3F093318
:107F440009F402DD053409F48BDC083309F457DB4A
:107F5400023409F400DC0334B1F510913A0C0E94A8
:107F6400A14600E0E091390CE11711F00C3008F063
:107F74001DC00E94566C0E94C46C0E941A6E1A9313
:107F84000E94711E1A937CD10E94F66DE0912A0C16
:107F94000E943C75E0912D0C0E943C750E94187162
:107FA4000E94056E0E94FE700395DCCF0E94440D72
:107FB4000E94D8420E2F013221F0E091390CE117D2
:107FC40009F401C0CCCF043499F40E945C7581F4A7
:107FD400A091D40BA03021F4A091D20BA03031F0A9
:107FE4000E94A5730E94566C0E940A530E94BA1CF8
:107FF400E0911B08E03011F40E94CB0D49C0E13040
:10800400D1F4A0912108AB3010F4013209F405C079
:108014000E9469150E94440D0DC0E0E0E0931E0823
:108024000E946F750E942474E0E00E947475E2E07F
:10803400E0931B082DC0E23059F5013269F4E0E009
:10804400E0931B080E94A146EAE2EA93EBE5F8E11B
:108054000E9424740E94CB0D0B3211F00D3359F49D
:108064000E946F75FA93EA93E1E3EA930E94F7633F
:10807400E1E00E9474750D3259F40E946F75FA9311
:10808400EA93E2E3EA930E94F763E2E00E947475E4
:10809400A0911808A33009F409CE0E94D37D0C9452
:1080A40047451A93E3E0E09319080E94A1460E9411
:1080B400566C0E94566C0E947A46E7E6F8E10E94EC
:1080C400B86D0E94566C0E94B36D0E947A46E3E13B
:1080D400F6E00E949D70E0E1F0E00E944F7010E035
:1080E400E091CA0B1E1700F50E941E6EE117D1F035
:1080F400E12FE05DEA93EFE6F8E1FA93EA93E0E337
:10810400EA93E0E00E947A7049F40E948C71ED5E7B
:10811400F94FA1E0A083E12FE05D01C0EEE2EA9314
:108124000E9414461F5FDCCF0E944875E0E0E09394
:10813400C005E0931B080E94CB0D19910895E881B6
:10814400E03021F4EAEEF6E00E947975A881A130CE
:1081540021F4E4EEF6E00E947975A881A23021F4BE
:10816400E0EFF6E00E947975A881A33021F4EEEFE8
:10817400F6E00E947975A881A43021F4E4E0F7E0E8
:108184000E94797529C11A930A93E0E0E0937D0572
:10819400E0937E0510E0143190F400E0033068F4BD
:1081A400A3E01A9FF001EC57FA4FDF01EE27A00F6E
:1081B400BE1FE0E2EC930F5FF1CF1F5FECCFECC387
:1081C4001A9311E0E981E11780F00E948C71E25565
:1081D400FF4FE491AA81EA2319F0E12FE05D01C089
:1081E400E0E2EA931FD51F5FEDCF30C51A9311E08B
:1081F400E981E11778F00E948C71E255FF4FE49118
:10820400AA81EA2311F0E1E301C0E0E3EA930AD58D
:108214001F5FEECF1BC52A97A0911C0CA13038F02C
:10822400EA85FB856C857D850E942F7507C00E94B9
:108234007E750E9482750E947E75FCD426C12A97A1
:108244000E947E750E948B750E9494750E947E75B3
:10825400F1D41BC12A970E947E750E94A7750E94C3
:10826400AE75E8D41FC12A970E947E75EDE8F8E147
:108274000E94B3750E942F740E94AE75DBD412C1A4
:108284002A970E947E75E0E9F8E105C02A970E94CA
:108294007E75E4E9F8E1FA93EA93EE850E949C6C1A
:1082A4000E947E75C7D42B9608950E94CE7D10E05F
:1082B400E1E3E0933809E89431F8EA930E94A1637A
:1082C400E8E9F8E10E94177300E0E09182050E17D7
:1082D400E0F40E94C46CEC57FA4FE081E03258F4A9
:1082E400E3E2EA930E94D6620E94C46CEC57FA4F10
:1082F400E081E05D05C00E94C46CEC57FA4FE08158
:10830400EA930E94D6620F5FE0CF0E94B8759F0186
:108314000E94D1143A932A93E8ECF0E0FA93EA939A
:108324000E948D680E2FA0E031FCA1E0A03011F472
:10833400003009F001C0ECCF31FE09C0E0E0E09369
:108344008205E89431F8E1E00E94D57DF6C41F5F10
:10835400123008F4ADCFE0E0E09382050E94D57DB1
:10836400ECC4E0918105E03021F4E881EA930E94B5
:108374007C5EA0918105A13069F4A0E09299A1E00E
:10838400A13021F4A8950E94346FF7CFE881EA93D5
:108394000E942061A0918105A230F1F4E091820550
:1083A400F0E0EC57FA4FA881A083E0918205EF5FDB
:1083B400E0938205E0918305EF5FE0938305A032AB
:1083C40018F4EF5FE0938305A0918305A83320F0B0
:1083D4006CDFE0E0E09383052196089508950E9400
:1083E400C7740E94C77422D0EBE1EA93BADFE9E6CE
:1083F400EA93B7DFA0918105A13061F4E8ECF0E0E5
:108404000E949C6EE0919A00E069E0939A00E9E191
:10841400E0939900A0918105A23021F446DFE0E0C9
:10842400E0938305E0E0E09381050895EDE0EA93AD
:1084340098DFEAE0EA9395DF08951A9310E0E98162
:108444001E1728F4EA81EA938CDF1F5FF8CFFEC37E
:10845400EDE201C0EDE3EA93E8E2EA93EEDFE6DF62
:1084640008952A97A0911C0CA13038F00E947E75C3
:108474000E948B750E94947504C00E947E750E94B0
:108484008275FE010E949D700FD02E9608952A9742
:108494000E947E750E94A7750E94BC75FE010E9411
:1084A4009D7002D02C9608951A930A9310E0EA81E5
:1084B400E03011F408E201C00A81AB81BC81EE27EF
:1084C400A10FBE1FAC91A03011F0101708F007C027
:1084D400AB81BC810E94C1750E94C675EECFEA8152
:1084E400E03039F0EA811E1720F4E0E20E94C675FC
:1084F400F9CF27C01A930A9310E0EA81E03011F40F
:1085040008E201C00A81E12FAB81BC810E94F574AD
:10851400E491E03011F0101708F009C0E12FAB81AD
:10852400BC810E94F574E4910E94C675ECCFEA8187
:10853400E03039F0EA811E1720F4E0E20E94C675AB
:10854400F9CF1981088125960895E091C405A09179
:10855400C305EA17B1F00E94CB750E940C6EEC9132
:10856400E093C6050E94CB750E94A671E181E09359
:10857400C505A091C4050E94D175E093C405E1E04E
:108584000895E0E008950E94D675A981A0830E9411
:10859400D6753196A881A083A091C3050E94D17598
:1085A400E093C305C2C0E091DB0508951A93E091FE
:1085B400DB05E03059F40E94D1140E943A7221F490
:1085C400A091DB05A03009F001C0F5CF1091DB05C7
:1085D400E0E0E093DB050E943A7209F011E2E12F3A
:1085E400DDC30E94CE7D0E9481688F010E94D11458
:1085F400EC81FD81E00FF11FFF93EF930E948168EE
:10860400AF91BF91AE1BBF0B9D0100240216030660
:108614001CF40E943A7209F001C0E8CFE0E00E9425
:10862400D57D269608951A93E9810E94A3720E942B
:10863400DC75E05FFC4F108117FF05C0E12F0E943D
:10864400E375A0E0A08316FF05C0E12F0E94EA7540
:10865400A0E0A083E981ADE0EA9FF001E05FFC4F78
:108664000E94DC75E15FFC4FA0E0A08318815DC02F
:108674000E94CE7D30E0EE81ADE0EA9FF001E05F44
:10868400FC4F108116FF17C0E12FEF730E2F0E94CD
:10869400F17511F03A3008F009C00E94F975DF0154
:1086A4000E94DC6C0E94FF753F5FF1CF0E94F97558
:1086B4000E94EB74EC9317FF17C0E12FEF730E2F9A
:1086C4000E94F17511F0343108F009C00E9405765A
:1086D400DF010E94DC6C0E94FF753F5FF1CF0E94B6
:1086E40005760E94EB74EC930E94D57D42C2E8812A
:1086F400F9810E94BC6DEA81FB8132960E94BC6DB7
:10870400EC81FD8134960E94BC6DEE81FF8136962A
:108714000E94BC6DE885F9853896E491EA93E98571
:10872400FA8539960E94C16C02D022960895A097CA
:108734000E94CC7DEDA5FEA5A9A9BAA9EA0FFB1F4D
:10874400AF01E5E0F3E0EE83FF8310E01431C0F500
:10875400AE81BF81AC91A03049F1EE81FF81A3814C
:10876400B481EFA5F8A9EA17FB0701F5EE81FF81B3
:10877400A181B281E9A9FAA9AE17BF07BCF0EE81C5
:10878400FF81A181B2814A175B0784F00E940B76B6
:10879400AE0FBF1FE9A9FAA9AE17BF073CF00E94AC
:1087A4000B76AE0FBF1F4A175B070CF402C01A9377
:1087B4003ADFEE81FF813D96EE83FF831F5FC6CFD4
:1087C400E5E0F3E0EE83FF8310E0143110F00C9445
:1087D4008E44AE81BF81EC91E03011F00C9487445B
:1087E400EAA5EC93E9A9FAA9AE81BF811196ED93AC
:1087F400FC93EFA5F8A9AE81BF811396ED93FC938A
:10880400EDA5FEA5AE81BF811596ED93FC93EBA576
:10881400AE81BF811796EC93E0910904A0910F04F7
:10882400EA27AE81BF811896EC93E0911004AE81E3
:10883400BF811996EC93E0911104AE81BF811A9621
:10884400EC93AE81BF811B960E945F6D1C96E0E0A5
:10885400EC93E887E8A5F9A5309741F00E941676D5
:108864000E941B76E4E1EA930E946A69EEA1FFA1EB
:10887400309751F00E941676E8A5F9A5FA93EA9389
:10888400E4E1EA930E945669E0E0EC8F0E941676D8
:108894000E9441693E2F3B30C8F000E00E940576FB
:1088A400E081E03011F0053008F002C00F5FF6CF30
:1088B4000E940576E081E03049F40E9405760E942A
:1088C4002076E058AE81BF811B96EC93E0E0EA8B02
:1088D4003130C8F000E00E94F975E081E03011F019
:1088E400043108F002C00F5FF6CF0E94F975E081F1
:1088F400E03049F40E94F9750E942076E05CAE8174
:10890400BF811B96EC93E12F08C0EE81FF813D9659
:10891400EE83FF831F5F59CFEFEF0E94D37DE39671
:1089240008951A930A930E942B763097A9F1E09147
:108934006205E03061F50E942B7604900092620596
:10894400E0916205E03031F4E0E0F0E00E947975F6
:10895400E0E01AC00E9430760E942B760E94F97BD8
:10896400F595E7958F01D801E0E0F1E00E94717B75
:10897400E0938700D801E0E0F1E00E94A37BE0935C
:1089840086000E943076E0E4E0938B0005C0E0911D
:108994006205E150E09362050991199108950E94DE
:1089A400CE7D00E025E033E010E01431B8F5D901C4
:1089B400EC91E03079F111960E94EA7B0E943876BE
:1089C40024F5D90113960E94EA7BAC81BD81EA1794
:1089D400FB07DCF4F90101801280D90115960E948D
:1089E400EA7BE00DF11DAE81BF81AE17BF076CF4C9
:1089F400F90103801480D9011796EC910E9440720A
:108A0400AC81BD81AE17BF070CF004C0E12FEF5F4E
:108A14000E2F04C0235F3F4F1F5FC7CF003049F0C4
:108A2400E0916305E01721F0A0916305A03009F4FB
:108A340001C022C0A0916405A53079F40A93E1E055
:108A4400EA93A1DD0093630500936505D901EC91D8
:108A5400E0936605E3E0E0936105A0916405AE311F
:108A640019F4E4E0E0936105A0916105A33018F0E6
:108A7400E5E0E093680507C0E0E0E0936405E09377
:108A840061050E943D760E94D57D28960895E09167
:108A94006305E03091F0A0916405A93220F4EA93D3
:108AA400E2E0EA9370DDA0916405AD3330F0E0912B
:108AB4006305EA93E4E0EA9366DDE0E0E0936105B0
:108AC400E09364050E943D76E0E0E0936305E09363
:108AD4006705089534D157DB0895EA81E0937F0553
:108AE400E881E0938005E0910A04E061E0930A04E0
:108AF40024C10E94CC7DA0917F05A43120F4A091D3
:108B04008005A33008F033C0E0917F05F0E0ACE0CD
:108B1400B0E00E94467B8F01E0918005F0E0A4E183
:108B2400B0E00E94467B9F010E944376ECE0F0E0B7
:108B34000E944876F0E00E94F97A0E94606CEE810F
:108B4400E030A9F0E0917F05A3E0EA9FF001EC5743
:108B5400FA4FDF01E09180050E9414704C91552773
:108B64000E9443764A93EFE0EA930E943E4D0E94AE
:108B7400D37D27960895E0910A04E07141F0E2E084
:108B8400EA93B7DFE0910A04EF7EE0930A040895C4
:108B94000E944D76AF3EE0E0BE0744F4A09102038C
:108BA400B0910303AF33E1E0BE070CF039C00E947B
:108BB40052760E9426700E943E4DA0915D05B091B0
:108BC4005E05549734F4A0915F05B0916005139746
:108BD4000CF012C0E0915D05F0915E05A3E0B0E0F9
:108BE4000E941E7BEC57FA4FA0915F05B09160057F
:108BF400EA0FFB1FA981A083E0910D04ACE0EA9F7A
:108C0400F0010E944D760E94F5740E945F76E09117
:108C14005D05F0915E053196E0935D05F0935E0588
:108C24000C947D4AE881EA93E0911004EA93B0DF62
:108C34000C944C4A1A9310E00E946476E03031F0B0
:108C44000E946476EA93EEDF1F5FF6CF18812396C5
:108C540008951A930A9300E010E00E946776E030CA
:108C640021F00832E0E01E070CF007C00E9467768E
:108C7400EA93D8DF0F5F1F4FF0CF198108815DC0E1
:108C84001A930A9300E010E0F801AB81BC810E94C2
:108C94006E7621F0EA810E9473760CF009C0F80127
:108CA400AB81BC810E947876BDDF0F5F1F4FECCF94
:108CB400198108810EC30E94CE7D0E944D760E94C8
:108CC4007D7631978F010E9482760E9443760E94BE
:108CD4008A7633C00E94CE7DAC810E9491760E2F9D
:108CE40011270E9482760E9443760E948A76F1C2FE
:108CF400EA81FB81E0935D05F0935E05E881F981EB
:108D0400E0935F05F0936005AA81BB81ECE0F0E09D
:108D14000E94467B0E945F76A881B981E4E1F0E07D
:108D24000E94467B06C0EA81FB810E945F76E8814F
:108D3400F981E0930203F0930303249608950E94BB
:108D44009976143120F41A936EDC1F5FFACF0E94D7
:108D5400566C0E94566C0E945B6CEFE3F1E00E943B
:108D6400606C10E0153048F4A5E11A9FF001E05161
:108D7400FB4FA0E0A0831F5FF5CF10E0143148F44F
:108D8400ABE01A9FF001EC5EFB4FA0E0A0831F5FF5
:108D9400F5CFE0910A04EF7EE0930A041991089557
:108DA4000E949976143100F5ADE01A9FF001BF01DD
:108DB400E85FFC4FDF010E94EA7B0F01DF01EB81DA
:108DC400FC81AE17BF075CF0E981FA81E015F1057B
:108DD40034F0FB01E05FFC4FE081E03009F402C0B5
:108DE4001A9321DC1F5FDECF0E94566C0E94A1768D
:108DF4000E945B6CA985BA850E94A6760E94606C6D
:108E040067C2A2970E94CC7DE9A50E94A3728F013C
:108E1400D8011B96EC91E03009F415C2D8011B96D9
:108E2400EC91E9A3E07859F0FE013696FA93EA93BF
:108E3400EBA10E94E375FA93EA930E942B69E9A1DE
:108E4400E07459F0FE013696FA93EA93EBA10E947E
:108E5400EA75FA93EA930E942B69FE013696FA9317
:108E6400EA930E944169E8A3E0910D04EB8FE0913D
:108E74000E04EA8F0E94EA6ED80111962D913C915E
:108E8400D80113964D915C91D80115960E94EA7B06
:108E9400EEA3FFA3D8011796EC91F0E0ECA3FDA399
:108EA400D8011896EC91EC8FE0910E04A0E10E9499
:108EB400AB76EAA3FBA30E94AF760E941B760E94C6
:108EC4001B76ECA1EA930E94904BD8011996EC9181
:108ED400EC8FE03011F4E8E0EC8F0E94AF760E9452
:108EE400B4765A934A930E94BB760E94BF760E943E
:108EF400C6760E94C9760E94AF763A932A930E945E
:108F0400C976EEA1FFA10E94D0765A934A930E949B
:108F1400B4760E94C976A8A5A130B1F43A932A93F5
:108F2400FA0131960E94C676FA013196FA93EA93D1
:108F34000E94BB76F90131960E94D576F9013196EB
:108F4400FA93EA930E94C976A8A5A230F1F40E948C
:108F5400BF7631970E94C676EAA5FBA5E40FF51FFC
:108F64003197FA93EA930E94BB76EEA1FFA1E20F38
:108F7400F31F31970E94D576EAA5FBA5E20FF31FF4
:108F84003197FA93EA930E94C976E8A5E03011F488
:108F94000C94F548D8011996EC91EC8FE0910D04EE
:108FA400ACE00E94DA760E94717BED8FA8A1EA17EB
:108FB40010F40C942448E1E0E0930E04E03021F036
:108FC400ECA1FDA1B5970CF402C00E94E076AAA121
:108FD400BBA1ECA1FDA1EA1BFB0BDF010E948F7179
:108FE400EAA3FBA3ABA1AA231AF4E0E0EAA3EBA350
:108FF400A8A10E949176AEA1BFA1F0E00E94E876FC
:10900400EE8FA8A5A13021F40E94EB760E94EE76A3
:10901400A8A5A23031F40E94EB760E94D0760E947B
:10902400FA76E0E0E9A30E940077AE0FBF1FEC914F
:10903400E03039F00E9400770E9478760E9405772C
:10904400F2CFD1C0E1E0E0930E04E03031F0ECA1C6
:10905400FDA1E734A0E0FA070CF402C00E94E07618
:10906400E8A1EF8FEAA1FBA1EE0FFF1FACA1BDA108
:10907400AE1BBF0BE3E0F0E00E94717BEAA3FBA30D
:10908400ABA1AA2322F4E1E0F0E0EAA3FBA3EF8D75
:10909400E150EF8FEF8DF0E0DE011696AE0FBF1FAB
:1090A400AC91A03219F0AF8DA13008F404C0EF8D5B
:1090B400E150EF8FEFCFAF8D0E949176AE2FEEA1EE
:1090C400FFA1B0E0EA17FB0714F3EF8DE03011F4D1
:1090D400ED8DEF8FAF8DECE00E94DA760E94E8769A
:1090E400EE8FA8A5A13021F40E94EB760E94EE76C3
:1090F400A8A5A23031F40E94EB760E94D0760E949B
:10910400FA76E0E0E9A30E9400770E946E7621F0EF
:10911400EF8DA9A1AE1708F007C00E9400770E9446
:1091240078760E940577EFCFAF8DE8A1EA1BAE2FCA
:10913400ED8DEA1768F0AF8DE8A1EA1BACE0EA9F79
:10914400F001A0910D040E94DA760E94E87601C035
:10915400E0E0EE8FA8A5A130A1F40E94EB76E20F27
:10916400F31F31960E944876AFE00E94AB76E40F7D
:10917400F51FDF01ECA1FDA10E94A67131960E94AA
:10918400986EA8A5A23089F40E94EB76E20FF31F33
:109194000E944876AFE00E94AB76E40FF51FDF0132
:1091A400ECA1FDA10E941E75BEDD0E940077AE0FEA
:1091B400BF1FAC91A03219F4E9A1EF5FE9A30E94AB
:1091C40000770E946E7639F0AF8DE9A1EA1BAE2FCD
:1091D400ED8DEA1708F407C00E9400770E947876A4
:1091E4000E940577ECCFD8011C96EC91E03029F170
:1091F4000E94EA6E0E94AF7696DDF801A485A4363B
:1092040098F4EFE0E0931004F801A485AA3028F064
:10921400A485AA930E94424106C0D8011C96EC91F1
:10922400E05DEA93FFDC09C0ECE0E0931004E2E5C2
:10923400EA93F8DCEDE4EA93F5DCEB8DE0930D04BE
:10924400EA8DE0930E040E94D37DAA9608951A93A2
:1092540010E0E89427F8143170F40E94C76EE030EF
:1092640011F00E94CE6E1F5FA895E12FE37011F4F8
:109274000E94C814F0CFEFE0E09310040E94C814D9
:109284000C94D94D1A9310E01431F8F40E94D36E63
:10929400B1F0A85FBC4F0E94EA7BDF01EB81FC8147
:1092A400EA17FB0764F4F001E85FFC4FDF010E945A
:1092B400EA7BDF01E981FA81AE17BF070CF002C037
:1092C4000E94CE6E1F5FA895DFCFEFE0E0931004FD
:1092D4001881259608951A9310E0143190F40E9491
:1092E400D36E31F0FD01E15FFC4FE081E17009F4E0
:1092F40006C01A93E0910A04E170EA9382DD1F5FCD
:10930400ECCF0C94D94D2C970E94CC7DAD89BE89AD
:109314000E948F710E940D77EB8BFC8BED89FE8987
:109324000E941277EB89FC89E017F107FCF00E9498
:1093340045772E2F33270E9469770E9470770E9409
:1093440077770E947C770E946977F801A98DBA8D9E
:109354000E94526D0E947777F8010E948677EA8D09
:10936400EA930E94F34B0F5F1F4FDCCF48C02C974A
:109374000E94CC7DAD89BE89E4E0F0E00E94717B5F
:109384000E940D77EB8BFC8BED89FE89EE0FFF1F9E
:109394000E941277EB89FC89E017F10784F10E949F
:1093A4004577AE2FED89FE89B0E0EA0FFB1F9F01E0
:1093B4000E9469770E947077E98DFA8DEE0FFF1F86
:1093C4000E9486770E947C77ED89FE89EE0FFF1F4D
:1093D400A98DBA8DAE1BBF0BBA93AA93F801A98DC0
:1093E400BA8D0E94526D0E947777F8010E948677A9
:1093F400EA8DEA930E94F34B0F5F1F4FCBCF0E947D
:10940400D37D6B960895EA81F0E0EBBBF5BBF7E101
:10941400F09365001F98E6E1E0936500F093650022
:109424001F9AE881F981EBBBF5BB1F98FFE1F0932C
:109434006500EEE1E0936500F09365001F9A0C94DB
:109444004C4EE2E2EBBBE0E0E5BBE7E1E093650014
:109454001F98E6E1E0936500E7E1E0936500089575
:109464001F9A0895A0910403A23021F4E881AEE389
:10947400B3E10BC0A0910403A43021F4E881AEE36E
:10948400B3E103C0E881AEE1B3E1F0E00E94A6716C
:109494000E94F97B21960895E0910403E23011F4CF
:1094A400EEE40AC0E43039F4E0E2EA93A981BA8137
:1094B4000E947D7604C0E0E2EA93E981FA81FA939E
:1094C400EA930E94054A17C0E0910403E23011F4C4
:1094D400EFE40AC0E43039F4E1E2EA93A981BA8105
:1094E4000E948A7704C0E1E2EA93E981FA81FA935F
:1094F400EA930E94054A22960895E0910403E2301B
:10950400B9F4E4E4EA930E948F77AE0FBF1FFD0124
:10951400FE2FE0E0AF81B8850E94526D0E94054A9B
:10952400E5E4EA930E94A1760E94054AE6E453C06A
:10953400E33089F4E7E3EA93FF81E0E00F010E945E
:109544008F77EA0FFB1F0E9494770E94A1760E94F6
:10955400054AE6E340C0E43049F5E7E3EA93AF8126
:10956400B8850E947D76DF01EB81FC81AE1BBF0BC9
:10957400FD01FE2FE0E00F01AF81B8850E947D76EA
:109584000E949477AD81BE810E948A77DF01E981D0
:10959400FA81AE1BBF0BBA93AA930E94054AE6E375
:1095A400EA93AD81BE810E948A771CC0E0E5EA930C
:1095B4000E94F0740E94054AE1E5EA930E948F77C5
:1095C4000E94526D0E94054AE2E5EA930E94A17648
:1095D4000E94054AE3E5EA93E981FA81AD81BE81FF
:1095E400EA0FFB1FFA93EA930E94054A289608950E
:1095F400E0910403E33029F4E3E0EA93E0E1F1E0ED
:109604000BC0E43029F4E3E0EA93E0E2F1E004C0C3
:10961400E3E0EA93E0E3F0E1FA93EA930E94054A77
:109624000895E0910403E33029F4E3E0EA93E1E2EE
:10963400F1E00BC0E43029F4E3E0EA93E1E1F1E086
:1096440004C0E3E0EA93E8E3F0E1FA93EA930E94CA
:10965400054A08951A930A93EFE10E949D77EBE17E
:109664000E949D77EFE10E949D77E8EFFFEFE09382
:109674005F0CF093600CE491EF3F39F0E0915F0CE4
:10968400F091600C049000920403ECEBF3E18F0181
:10969400A0910403A23019F4EEE9F3E18F01A09143
:1096A4000403A43019F4EEE5F3E18F01F801E49129
:1096B400ED3F39F4F80131960E94BC6D0E94CB7ADB
:1096C40019C0EE3F71F4F80131960E94F97BDF0175
:1096D400E0910403F0E0EA17FB0711F00D5F1F4F60
:1096E40009C0F801E491EA93F80131960E94BC6D37
:1096F4000E94054A0D5F1F4FF801E491EF3FB1F658
:109704000E946F6DE1E0E0930E04E0930D04E4E148
:10971400E09313046DDF0991199108950E94A177D4
:10972400AE85AA2362F0AD85BE85A03FE0E0BE070A
:1097340034F4AB85BC85AF33E1E0BE070CF050C018
:109744000E94A977AE0FBF1FA03FE0E0BE0734F030
:10975400AD85BE850E947D76E987FA87EF81F8851D
:10976400AB85BC85AE0FBF1FA034E1E0BE0734F06B
:10977400AB85BC850E948A77EF83F8870E94C76D0A
:109784000E94C76D0E94C76D0E94C76DB6DE0E941D
:10979400C76D0E94AE77498554DE0BBB15BB2EE125
:1097A4003FE100E010E0EF81F885E017F10764F095
:1097B40050E0451730F020936500309365005F5FFB
:1097C400F8CF0F5F1F4FEFCF4BDE0E94566C0E9405
:1097D400566C0E945B6CEFE3F1E0FA93EA938DDE42
:1097E400C9C00E94A1770E94A977EA17FB0741F03C
:1097F400EF81F885AB85BC85EA17FB0709F03EC00D
:109804000E94B6771CF00E94BD7784F42D853E85B6
:10981400ED85FE85E987FA872D873E872B853C8574
:10982400EB85FC85EF83F8872B873C870E94C76D07
:109834000E94AE770E94A977EA17FB0749F4F1DE8C
:10984400EB85FC85ED87FE87EF81F885E987FA874C
:10985400F8DD0BBB15BB2EE13FE10D851E85E985C7
:10986400FA85E017F1073CF020936500309365001A
:109874000F5F1F4FF4CFF4DDBBDE7CC000930B04FD
:1098840010930C040E94C4770E94CB77FF93EF934C
:109894000E94CF770E94CB77AF91BF91EA17FB0765
:1098A40080F10E94BD77B4F420E030E00E94D277CA
:1098B400E217F30774F00E94C4770E94D9770E94DC
:1098C400D2770E94DE770E94E77758D02F5F3F4F10
:1098D400EDCF16C020E030E00E94CF77E217F30707
:1098E4007CF00E94C4770E94D9770E94CF770E94AF
:1098F400DE77F9010E94EE7741D02F5F3F4FECCF26
:1099040039C00E94B677DCF420E030E00E94F277A0
:10991400E217F3079CF00E94CF770E94D9770E9448
:10992400F277D0010E94717BAF010E94E777FA01C0
:109934000E94EE7723D02F5F3F4FE8CF1BC020E07B
:1099440030E00E94C477E217F307A4F00E94CF77B7
:109954000E94D9770E94C477D0010E94717BAF0125
:10996400F9010E94EE77FA010E94EE7707D02F5F8B
:109974003F4FE7CF0E94D37D2F960895EA81FB8164
:10998400FA93EA9389DD0E94F9779EDDE2E2EA9395
:10999400E0910B04F0910C04FA93EA930E94054AB7
:1099A400249608950E94CC7DEC85FD85309711F4B2
:1099B4000C94764D00910D0410E0E0910E041E17F6
:1099C40010F00C943D4DE885F985FA93EA937CDD1B
:1099D4002C853D854A855B85022E032A11F40C945F
:1099E400354D37FF36C05A934A9356DDE2E2EBBB5E
:1099F400E0E0E5BBE7E1E09365001F98F6E1F09352
:109A04006500E0936500EE81EBBBEF81E5BBEFE120
:109A1400FEE1E0936500F0936500E093650001FFCB
:109A240004C0F0936500E093650036FF11C0F09325
:109A34006500E093650001FF06C0F0936500E093C4
:109A440065004F5F5F4F220F331F4F5F5F4FEDCFB6
:109A54001F9A220F331F01FF02C04F5F5F4F4F5FFA
:109A64005F4F0C94EE4CE885F9853196E887F987C9
:109A74001F5F0C94DF4C38C022970E94CC7DE88590
:109A8400EA930E94344AEE83FF83E985A8E1EA9FC2
:109A9400F001E25EF84F8F0130E0383028F5F8012C
:109AA400E4915E2F0F5F1F4FF801E4914E2F407F2A
:109AB4000E94FE770E940378EA87FB87F801E4910D
:109AC4004E2F440F440F440F440F0F5F1F4FF801F4
:109AD400E4915E2F0F5F1F4F0E94FE770E94037870
:109AE400EA87FB873F5FD9CF0E94D37D2E960895E6
:109AF40024970E94CC7DEA85EA930E94344AEE833F
:109B0400FF8300E010E0EB850E947376C4F5EF85D7
:109B1400F889E887F98720E030E0EC850E94107826
:109B24001CF5E989FA89449155273196E98BFA8B1A
:109B34005A934A930E942F6DE989FA89FA93EA931A
:109B4400EC85FD85FA93EA930E94D44CE0910D04D0
:109B5400EE0FEE0FEE0FA885B9850E94F574E88725
:109B6400F9872F5F3F4FD9CFE0910E04AD85BE85B5
:109B74000E94F574ED87FE870F5F1F4FC4CF0E94CC
:109B8400D37D639608951A93EFEF0E946772E09372
:109B9400390910E00E948C71E05CF54FE081EF3FE1
:109BA40031F00E948C710E9415781F5FF3CF1991D8
:109BB40008951A930A930091D00BAA81A53411F445
:109BC400E0E066C0AA81A23539F4A0913508A1303D
:109BD40019F40E94187809F405C00E94141CE0E0EE
:109BE400E0933508AA81AB3411F0A33599F4E02F42
:109BF400E470E43011F414E001C013E0E02FE270EB
:109C0400E23009F41C5FE02FE170E13009F41F5FDA
:109C1400E12F3EC0AA81A13511F0A13799F4E02FBC
:109C2400E470E43011F417E001C016E0E02FE270B4
:109C3400E23009F41C5FE02FE170E13009F41F5FAA
:109C4400E12F26C0AA81A33421F0A13411F0A2345B
:109C540041F413E0E02FE170E13009F41F5FE12FDC
:109C640017C0AA81A73741F417E0E02FE170E13073
:109C740009F41F5FE12F0CC0AA81A03441F415E060
:109C8400E02FE170E13009F41F5FE12F01C0EFEF35
:109C9400198108812396089524970E94CC7D2091F0
:109CA400D00BA0914009A53411F00C94184FE0E0BA
:109CB400E09335080E946072E0E0E0935D0BE09170
:109CC400D40BE03089F5E0911008A0911108EA174F
:109CD40039F00E941E78ED55F84FE081E13009F02B
:109CE40023C0E7E7EA930E94D6620E941E78E855F3
:109CF400F84F0E94AB71FA93EA930E942478EC55D2
:109D0400F84FDF010E9416740E942478E755F84F3B
:109D14000E942978E2E0E09335080E941E78ED5510
:109D2400F84FA2E0A0832FDFE0913508E03011F076
:109D34000C94184F0E94187811F40C94F24E0E945F
:109D4400091CE1E0E0933508E22FE870E83081F483
:109D54000E942E78E8EEF3E00E94717BDF010E94FE
:109D6400C27D14F4E1E301C0E0E3EA930E94D66209
:109D7400E22FE074E03411F413E001C012E0E0914A
:109D8400250C0E94B0741A930E944263E22FE4707F
:109D9400E43049F40E942E78E0E1F7E20E94A37BCC
:109DA400AF0114E006C00E942E780E949873AF01A0
:109DB40013E0E22FE071E03111F4415050405A9326
:109DC4004A931A930E944263E22FE072E03211F444
:109DD40014E001C013E0E091280CF091290C17C0A5
:109DE40018E0E22FE470E43009F41F5FE22FE8701A
:109DF400E83009F41F5FE22FE072E03209F41F5FDC
:109E0400E22FE074E03409F41F5FE0E0F0E0FA933D
:109E1400EA931A930E944263E22FE170E13029F43D
:109E2400E0915D0BEA930E94D662ADDEA0914009F9
:109E3400A73729F4E2E0E0933508E03009F473C071
:109E44000E9460720E9433780E941B731E2F0E942E
:109E54003673AF01E1E0EA930E947D620E2FE09138
:109E64001008A0911108EA1739F00E941E78ED55E8
:109E7400F84FE081E23009F053C00E941E78EC559F
:109E8400F84FDF010E94EA7B4E175F0711F00C9434
:109E94008E4F0E941E78E655F84F008011800E9474
:109EA4001E6E0E94F571EA17FB0769F10E941E7885
:109EB400E655F84FDF010E94EA7B0E9439780E9440
:109EC4001E78E655F84FDF010E94EA7BEB59F44F08
:109ED400E0810E9441780E9448780E949F6D0E9410
:109EE4004B78EFE9F8E10E941773003029F05A9398
:109EF4004A930E94096302C00E9451780E945578D7
:109F04000E94BC6309C0003039F00E94597820F4E3
:109F14000E940B740E943026E1E1F8E00E94607810
:109F2400E0E0E0933508A0914009A33421F40E94B5
:109F34007133E03009F40BC00E9460720E943378E0
:109F44000E94A5730E94566C63D30E94BA1CA09110
:109F54004009A13411F0A23421F40E9460720E94DD
:109F64003378A0914009A03421F40E947133E03089
:109F740009F420C00E941B73E887F987E2E0EA93A2
:109F84000E947D621E2F0E9464780E94E8170E943E
:109F940052740E946A78E152F84F10830E945274FE
:109FA400E652F84FA7E0A0830E9434720E946072C8
:109FB4000E943378A0914009AB3439F0A33529F0DD
:109FC400A13519F0A13709F076C00E947133E03051
:109FD40011F40C9457500E9460720E947178E1E46D
:109FE400F9E00E943173E22FE270E23029F4E4E0F8
:109FF400EA930E947D6202C0E1E0F0E0E887F9871D
:10A00400A0914009A13511F0A13721F40E943673C3
:10A014001E2F02C01091E60BE22FE470E43011F41D
:10A02400E4E001C0E3E0EA930E947D62AF01A09105
:10A034004009A33511F0A13731F4E885F9850E9470
:10A04400E57AE887F9870E94597820F0A091D40B2B
:10A05400A13011F51A935A934A93EB85FC85FA9330
:10A06400EA930E94D91C0E94CB77EE83FF83AE81D2
:10A07400BF810E94C27D84F40E946072E6E6EA9386
:10A084000E94D662EE81FF813197EE83FF83AE8119
:10A09400BF810E94C27D94F31A935A934A93EB852D
:10A0A400FC850E94EE726FDD06C00E94A5730E94BB
:10A0B400566C0E94D91C0E94D37D2A9608950E9452
:10A0C4007578E89422F80E942A74E2E7EA930E94E1
:10A0D400D662E0913B08EA930E94D662EFE0EA93ED
:10A0E4000E94D662A0913808AA3219F41A9363D355
:10A0F4001AC0A0913B080E948C71EB59F44FE08187
:10A10400EA1721F4E0913B08E03349F40E94DF6C44
:10A11400AB59B44FE0913B08EC931A934CD322FC17
:10A1240002C00E94BC63C0C20E947578E0913B08E3
:10A13400E053AE2F0E948C71EA58F44FE081EA1785
:10A1440041F51A9338D3A0913608A23019F40E942D
:10A154007D7809F402C00E948378A0913608A33068
:10A1640019F40E947D7809F402C00E948378E0E02B
:10A17400E0933608E093630C0E948C71EA58F44F24
:10A18400BF01E081EF5FAE2FEAE00E94A07BDB011C
:10A19400EC938AC2E881E03019F40E94517806C039
:10A1A400E881E8500E94B0740E94096321960895E2
:10A1B4000E94CC7D25FC28C20E947D7811F40C9469
:10A1C4005A520E948678E752F84F9F01D90111969E
:10A1D400EC91E43071F50E948C780E948F780E9493
:10A1E4009678F901A681A03021F4A281B381109759
:10A1F40009F007C0E2EAF8E10E9417730E9455785B
:10A2040015C00E9448780E949A780E944B78E5EA2B
:10A21400F8E10E9417730E949E780E94A478F901C5
:10A22400A085B185BA93AA930E9409630E94AA7873
:10A23400EBC1E730C9F40E948C780E948F780E94A9
:10A244009678E8EAF8E10E9417730E949E780E94CB
:10A254004B78EBEAF8E10E9417730E949A780E9407
:10A2640009630E94AA78D0C1E93089F40E948C78ED
:10A274000E948F780E949678EEEAF8E10E941773A4
:10A284000E94B1780E944B780E94AA78BDC1E63042
:10A2940029F5EAE2EA930E94A163E1EBF8E10E9466
:10A2A4001773D901EC910E94B478E091CE0B0E940F
:10A2B400B478EBE4EA930E94D6620E949A780E94F2
:10A2C4000963E4E5EA930E94D6620E949E780E94A4
:10A2D40009630E94BC630E94837896C1E530C9F487
:10A2E4000E94FC730E943978D901EC910E94417854
:10A2F4000E9448780E949A780E944B78EFE9F8E12E
:10A304000E9417730E949E780E9409630E94AA7893
:10A314007BC1E83039F50E948C780E948F780E94C6
:10A324009678E4EBF8E10E941773F901A681AA93E9
:10A334000E940874309719F00E941D7004C0D9015E
:10A344001696EC91F0E0FA93EA930E9409630E9456
:10A3540055780E94BC63D9011196E0E0EC930E9409
:10A36400837852C1E130C9F5A0911908A53029F4C8
:10A37400E091CE0BE65F1E2F01C011E0E12F0E9499
:10A38400B8780E948C710E94BD780E94C0780E94A7
:10A3940048780E949A780E944B78E7EBF8E10E9493
:10A3A40017730E949E780E94A478D9011796EC91A5
:10A3B4000E94B0740E940963A0911908A53041F469
:10A3C4000E94C478A481B581BA93AA930E94786349
:10A3D4000E94B8750E94CA7817C1E330B1F40E9494
:10A3E400FC73F0960E94D5780E94FC730E94BD789D
:10A3F4000E94C078EAEBF8E10E9417730E949E78ED
:10A404000E94D9780E94CA78FFC0EB3069F50E9497
:10A41400DC780E94DF780E94C078EDEBF8E10E94BE
:10A424001773F901A681AA93B5DE0E94C478A781A7
:10A43400AA93B0DE0E94C478A085B185BA93AA938A
:10A444000E94A4780E949E780E94A478F901A481B5
:10A45400B581BA93AA930E94A4780E94B1780E940D
:10A46400D9780E94CA78D0C0EC3089F40E94DC7894
:10A474000E94DF780E94C078E0ECF8E10E94177334
:10A484000E94B1780E94D9780E94CA78BDC0EE308B
:10A4940079F40E94DC780E94DF780E94C078E3ECB3
:10A4A400F8E10E9417730E94B8750E94CA78ACC084
:10A4B4000E94187861F0A0913608A03041F4A09170
:10A4C400D30BA13021F40E941E6EE13009F426C0A2
:10A4D400A091860BA03059F0E091880BF091890B84
:10A4E400FA93EA93E8EEF3E00E94AF73B9F4E1E380
:10A4F4000E94D578E091770BE05D0E9441780E943C
:10A504001E6EEA930ED1E09336080E94B875E0936C
:10A51400610CF093620CE0E0E093860BA0913608A6
:10A52400A03059F0E091610CF091620CFA93EA9337
:10A53400E4E6F0E00E94AF7309F025C0A09136086C
:10A54400A23019F40E947D7809F402C00E94837835
:10A55400A0913608A33019F40E947D7809F410C044
:10A56400A091630CA33030F00E948378E0E0E09384
:10A57400630C06C00E948678E652F84FA8E0A083D8
:10A58400E0E0E0933608A091870BA130E9F5E09173
:10A594003A0CA091390CEA1791F1EAE20E94D578BD
:10A5A400E091750BE05D0E944178E0913A0CEA93EA
:10A5B4000E94711E0E944878E0912A0C0E94B07497
:10A5C4000E944B78E6ECF8E10E9417730E94187120
:10A5D400FA93EA930E94A4780E949B740E94E37801
:10A5E4000E94BC63E0913A0CEA930E94B31CE09190
:10A5F4003A0CEA930E94821CE0933A0C05C0E0E016
:10A60400E093870B689420F80E94D37D26960895E2
:10A614001A930A930E947133E030D9F00E94527465
:10A62400E752F84F8F01EC81FD81D8011296ED932A
:10A63400FC93EA81FB81D8011896ED93FC93EE819B
:10A64400D8011696EC93D8011196E4E0EC930E949D
:10A6540034721981088127960895E091420BEA9398
:10A664000E94D662E091430BEA930E94D662089559
:10A67400F4DF0E94F9770E94E6780E94E6780E944F
:10A684004B7897C01A930E9409621E2F103021F054
:10A69400E12FE150E093400BE0DFE091400BEF5FEE
:10A6A4000E94B0740E944B78199108950E94CE7D47
:10A6B40031E00E94ED7828F00E942573AC91A43318
:10A6C40008F02AC030E00E942573EC91E270E69510
:10A6D4001E2F0E942573EC91E1700E2FA0915A0B4E
:10A6E4001A1729F4E1E0EA27E0935A0B31E0A0912C
:10A6F4005B0B0A1729F0E1E0EA27E0935B0B31E0FA
:10A70400E0915B0BEE0FE05DA0915A0BEA0FEA9328
:10A714000E94D6620E941B74E32F0E94D57D24966A
:10A7240008951A9310E00E94187811F40C94D953E8
:10A734000E94091CEAECF8E10E941773E091250CD1
:10A744000E94B0740E944B78EDECF8E10E941773FC
:10A75400E091280CF091290C0E94E3780E942E7855
:10A76400A031E7E2BE074CF4E0EDF8E10E94177374
:10A77400E091260CF091270C13C0E3EDF8E10E9460
:10A784001773E9810E9432700E942E78EA0FFB1F32
:10A794000E94D370E091260CF091270CE051F7420F
:10A7A400FA93EA930E9409630E94557811E0E12F1D
:10A7B40018812296089524970E94CC7D0E94F178F6
:10A7C400E0E0EC930E94B061E13010F40C94C056C8
:10A7D400E091420BEB3441F4E091430BE33219F482
:10A7E4000E9409621E2FC7C2E435A9F4E091430B0D
:10A7F400E33221F40E940962EE83FF83E091430B6C
:10A80400EF3441F40E9409621E2F1A930E94F074DF
:10A814000E94E817B0C2E23411F00C945855E0914C
:10A82400430BE13251F4AA85AF3F29F40E94A5738A
:10A834000E94566CEDDE0E94BA1CE091430BE13499
:10A84400E1F40E9409621E2F113071F4A0913608C0
:10A85400A13019F40E94187809F402C00E94141C53
:10A86400E0E0E093860B09C0E1E0E093860B0E94F0
:10A874008168E093880BF093890BE091430BE534F6
:10A88400A9F4E6EDF8E10E9417730E94F11BF39717
:10A894003CF00E9409620E94D3700E94F67801C0C5
:10A8A400E0E3EA930E94D6620E945578E091430B5C
:10A8B400E63409F50E94027919F40E940962AF0195
:10A8C400E885F9850E9422700E2FE091E60BE030B6
:10A8D40011F01091E60B003420F0A091D40BA130BC
:10A8E40021F40E940E790E94D91CAA85AF3F19F465
:10A8F4000E940E798DDEE091430BE23511F00C9449
:10A9040015550E94027919F40E940962AF0130E0E2
:10A91400A091D40BA03021F40E941E6EE13009F006
:10A9240027C00E947733E03011F10E94E272EC55A7
:10A93400F84FA885B985A083B1830E94E272E655D9
:10A94400F84FDF01EA850E9430720E94E272E855F6
:10A95400F84F10830E94E272E755F84F40830E943B
:10A96400E272ED55F84FA1E0A0830E94E87259C04D
:10A974000E947133E23010F40C9413550E946478F1
:10A984000E94EB1D3E2F3F3F29F00E94EB70A4175D
:10A99400B5070CF412C00E949B74E41BF50B0E94D3
:10A9A400F9700E94BF7219F4E0E0E0932A0C3A9324
:10A9B4000E94781E689420F803C0E0E0E887E987E5
:10A9C4000E945274E752F84FDF01EA85F0E0EB5938
:10A9D400F44FE081EC930E9452740E946A78EF5124
:10A9E400F84FDF01EA850E9430720E945274E152EE
:10A9F400F84F10830E945274E652F84FA5E0A083EA
:10AA04000E943472E885F985309759F00E94647881
:10AA1400FA010E94E57A0E94EE720E940E790E9469
:10AA2400631C689422F8E091430BE335F1F50E942E
:10AA34000962E887F9870E948678DF01E652F84FB9
:10AA4400E081E23081F4FD01EF51F84F0080118084
:10AA54000E941E6E0E94F571EA17FB0721F4A09173
:10AA64003608A23009F01FC00E948678E552F84FDC
:10AA7400DF010E94EA7BDF01E885F985EA17FB071D
:10AA840079F40E948678DF01ED51F84FE081EA9372
:10AA9400FD01E752F84FE081EA930E94302603C09B
:10AAA400E7E0E0932406689422F865C1E43411F0E9
:10AAB4000C94C055E091430BE33559F4E9EDF8E10A
:10AAC4000E9417730E94A15E0E94B478E1E0E093B3
:10AAD4003909E091430BE03511F00C94BF550E9405
:10AAE400127911F40C94BF5520E00E94187940F0BB
:10AAF4000E942573AC91A23219F00E941C7909F4CA
:10AB04003CC0E22FE03061F40E942573AC91A33283
:10AB140011F421E004C00E9420790E947C5E2AC0C6
:10AB2400E13051F40E942573AC91A43211F422E077
:10AB340001C020E010E01EC0E23011F0E330D1F497
:10AB44000E9420790E945968EF3F99F0E12FE29525
:10AB5400E07FEF930E9420790E945968AF91EA0F39
:10AB64001E2F2F5F243021F41A930E947C5E20E074
:10AB740001C020E00E941B74B8CFFDC0E33411F083
:10AB84000C943056E091430BE534B9F4E6EDF8E16A
:10AB94000E9417730E94F11BF3974CF00E94096204
:10ABA400E05FF84D0E94D3700E94F67801C0E0E3A4
:10ABB400EA930E94D6620E945578E091430BE634F2
:10ABC400D9F441E050E00E9409620E2F0E942479DA
:10ABD400E13019F40E940962AF01E091E60BE03024
:10ABE40011F01091E60B1A930E94C46CE05FF84DCB
:10ABF4000E94D5760E94D91CE091430BE335A1F461
:10AC04000E9428790E941870E83141F4E0918A0B7F
:10AC1400EA930E949717689420F806C0E885EA939F
:10AC2400EFEFEA930E943026E091430BE134A9F45C
:10AC3400ECEDF8E10E9417730E942879EA930E94D0
:10AC440094180E946325E03011F0E1E301C0E0E3D1
:10AC5400EA930E94D6620E9455788DC0E63511F0C1
:10AC64000C949556E091430BE33411F00C949456F4
:10AC74000E9409621E2F113010F40C949456A09176
:10AC84001908A13091F50E942479E03021F0A091B7
:10AC9400A2061A1709F028C011500E940962AF01D8
:10ACA4001A930E94F4203E2F0E945F730E94A671A3
:10ACB4000F010E945F730E940C6E0E942F790E9404
:10ACC4002479E03071F00E940962AF010E9473732D
:10ACD4000E94A6710F010E9473730E940C6E0E9461
:10ACE4002F791A930E9451111DC01630D8F41150B7
:10ACF400A12FEAE00E94507BA3E2EA9FF001E8550D
:10AD0400F94FBF01A12FEAE00E94A07BF0E0BB0154
:10AD1400AAE0B0E00E941E7BDB01AE0FBF1F1496B9
:10AD24000E94407128C0E93431F5E091430BE035CD
:10AD340051F40E9409621E2FE0E0EA931A930E94E4
:10AD44006718E0932E06E091430BEC34A1F40E94C3
:10AD5400CB61E09328060E942479E03021F00E9420
:10AD6400CB61E09329060E942479E03021F00E940F
:10AD7400CB61E0932A060E946C6124CD0E94D37DAE
:10AD84002B960895A091580BA03521F4A091590B4E
:10AD9400A03408F005C0E091590BEA930E94B4185E
:10ADA400A091580BA33521F4A091590BAA3008F0B7
:10ADB40005C0E091590BEA930E94DF18A091580B4B
:10ADC400AB3421F4A091590BA03808F005C0E091F0
:10ADD400590BEA930E941B19A091580BA63521F434
:10ADE400A091590BA03108F005C0E091590BEA93EA
:10ADF4000E944719A091580BA43511F40E94D21750
:10AE0400E1D60895E3EAF6E0FA93EA93E091420B7F
:10AE1400EA93E0E8F0E00E944F7008950E943779C9
:10AE2400A0E0A083E091400BE093590BE091420B2A
:10AE3400E093580B08950E94CC7D0E94B061E130EC
:10AE440010F40C94385AE091580BA091420BEA1775
:10AE540009F098DFE091420BE33239F5E091430BBE
:10AE6400EC3431F4CFDFE4E0E09318080E943D793C
:10AE7400E091430BE435C1F4C5DFE091660CE030AA
:10AE840029F0EF77A9E0B0E00E942C7CE091670CF8
:10AE9400E03029F0EF77AAE0B0E00E942C7C0E9419
:10AEA4003D79E7E0E0931808DEC2E934E9F4E09183
:10AEB400430BE434C1F40E941279A9F010E010E0CD
:10AEC400183178F4A3E2B7E00E948C71EA0FFB1FFB
:10AED400FF93EF930E94CB61AF91BF91EC931F5FFF
:10AEE400EFCF0E94FE0CBFC2EB34E1F5E091430BBF
:10AEF400E13211F487DF35C0E53211F443DF31C0AC
:10AF0400E33299F40E94437921F00E944E790E9421
:10AF1400E9180E943779E081EB3429F4E0E0E0930A
:10AF2400350CE093360C7ADF1CC0E134D1F40E9476
:10AF340009629F012093350C0E94547991F00E947C
:10AF440009629F01A091350CF901E270F070EA2BBF
:10AF5400E093350C0E94547921F00E940962E09339
:10AF6400360C81C2E33581F5E091430BE13211F4F3
:10AF740049DF29C0E33299F40E94437921F00E9409
:10AF84004E790E94C3180E943779E081E33529F491
:10AF9400E091400BEA930E94041B40DF14C0EE349E
:10AFA40091F40E94D37410E01A3068F4A4EBBBE06F
:10AFB400EE27A10FBE1F0E948C71EC5BF44FE08161
:10AFC400EC931F5FF1CF4FC2E63511F00C94325869
:10AFD400E091430BE13211F415DF41C0E33299F4FF
:10AFE4000E94437921F00E944E790E9427190E9401
:10AFF4003779E081E63529F4E091400BEA930E9429
:10B004005A190CDF2CC0E63531F40E9409629F0105
:10B014002093310C24C0E53471F40E9409629F012D
:10B024002093300C0E94547929F00E9409629F01F8
:10B034002093330C14C0E43591F440E050E00E94B6
:10B0440009629F01022E032A11F042E050E00E949F
:10B05400547919F00E940962AF014093320C03C283
:10B06400E43511F00C94EC58E091430BE33231F4E5
:10B074000E9409623197E093400BABC0E03511F0B8
:10B084000C94EB5810E00E94187950F00E9425733C
:10B09400AC91AD3329F00E941C7911F01E3008F0F8
:10B0A40005C00E948C710E945A79EDCF0E948C7168
:10B0B4000E946379EDE30E94687911F00C94EB58D7
:10B0C400E4E5E093580B10E00E94B1703496E491EB
:10B0D400EF3F11F40C94EB580E94D7740E94B170A6
:10B0E4000E94BC6D0E941969E03011F00C94E9587B
:10B0F4000E94B1703496E491E03851F40E940962E0
:10B10400E058FF4FE093660CE0E8E093670C5FC003
:10B11400E23839F40E940962E058FF4FE093670C6B
:10B1240056C0E13839F40E940962A8E0B0E00E94F8
:10B134002C7C4DC0E03011F0E13051F40E94A77036
:10B14400FF93EF930E940962AF91BF91EC933FC0CC
:10B15400E23059F40E94A770FF93EF930E940962B2
:10B16400AF91BF91ED93FC9332C0E33051F40E9450
:10B17400A770FF93EF930E94E861AF91BF91EC93A6
:10B1840026C0E43021F50E94B1703596E491EA932B
:10B194000E94B7620E94A770E093640CF093650C60
:10B1A40000E00E94B1703596E4910E1780F40E947D
:10B1B400C46CEC5BF44FE081A091640CB091650C1D
:10B1C400EC93A4E6BCE00E94C16E0F5FEACF1F5F60
:10B1D4007BCF49C1E03511F00C94355AE091430B13
:10B1E400E33299F40E94437921F00E944E790E943F
:10B1F40094180E943779E081E03529F4E091400BFE
:10B20400EA930E94191B0ADE2EC1E13211F4FADD21
:10B214002AC1E134D1F40E9409621E2F00E00D30EE
:10B2240098F40E94F974EA0FFB1F3396E491E11736
:10B2340049F40E94F9740E94FD74A0919B0BEA2BBF
:10B24400E0939B0B0F5FEBCF0EC1E63559F5E0E0C1
:10B25400E093410BAEE9BBE00E946D79FF93EF935D
:10B264000E940962AF91BF91EC93EBE2EA930E94D2
:10B274007C61E03059F0A1EABBE00E946D79FF9354
:10B28400EF930E940962AF91BF91EC930E94707991
:10B29400A091410BA33018F40E94547909F401C021
:10B2A400D9CFE1C0ED34D1F4E0E0E093410BAAEA58
:10B2B400BBE00E946D79FF93EF930E940962AF9106
:10B2C400BF91EC930E947079A091410BA33018F4C4
:10B2D4000E94547909F401C0EACFC5C0E735D1F41E
:10B2E400E0E0E093410BA1EBBBE00E946D79FF939A
:10B2F400EF930E940962AF91BF91EC930E94707921
:10B30400A091410BA23018F40E94547909F401C0B1
:10B31400EACFA9C0E434C9F5E0E0E093410B0E9410
:10B3240009629F01E2E0EA930E948961AF01E3E7C9
:10B334000E94687959F40E947679BF01D9010E946C
:10B344002B72E40FF51FDB01ED93FC93E9E40E94FB
:10B35400687979F40E94767920833183ABE9BBE084
:10B364000E946D790F010E947D79EC91E160D0011A
:10B37400EC930E947079A091410BA33018F40E94C1
:10B38400547909F401C0CBCF6EC0EE3499F40E9415
:10B39400D37410E01A3068F4ABE8BBE0EE27A10FD9
:10B3A400BE1F0E948C71EC5BF44FE081EC931F5F35
:10B3B400F1CF59C0E33459F4E2E2EA930E947C618C
:10B3C4000E940962E093960BF093970B4CC0E3350F
:10B3D40089F40E9409629F0100240216030624F4E2
:10B3E4002B30E0E03E070CF004C0F9013197E09304
:10B3F400980B39C0E53529F40E940962E0939A0B51
:10B4040032C0EF3491F40E9409621E2FECE2EA93F9
:10B414000E947C61E12FE295E07FEF930E94096234
:10B42400AF91EA0FE093990B1EC0E035E1F4E0E040
:10B43400E093410BADEABBE00E9483790E94A671C0
:10B44400FF93EF930E949762AF91BF91ED93FC93AA
:10B454000E947079A091410BA23018F40E94547993
:10B4640009F401C0E7CF0E946C61E7CC0E94D37D50
:10B47400269608950E94CE7D0E94B061E13010F4BA
:10B484000C940D5DE091420BE332A9F4E091430B7F
:10B49400E03519F4EFEDF8E109C0E83419F4E0E01F
:10B4A400F9E104C0E33531F4EBE1F9E1FA93EA930D
:10B4B4000E94E762ADC2E934C1F4E091430BE43485
:10B4C40099F40E94F30CC9D80E94877910E01831CE
:10B4D40048F4A3E2B7E00E94C175EA930E9417639F
:10B4E4001F5FF5CF0E94877993C2E43511F00C9465
:10B4F400135BE091430BE43229F4E8E2F0E00E94AC
:10B504008B798EC0E33211F4BDD88AC0E03511F0D6
:10B514000C94125BA2D8A091400BA83210F00C94AA
:10B52400125B0E948F790E94BC6D0E94E762EDE37A
:10B53400EA930E94D6620E948F793496E491E038AF
:10B5440039F40E941E6E0E94B0740E94096368C0A0
:10B55400E23839F40E94A2700E94B0740E94096318
:10B564005FC0E13839F40E94AB740E94B0740E9449
:10B57400096356C0E03011F0E13051F40E948F7934
:10B5840032960E94F97B0E94AB710E94937948C065
:10B59400E23059F40E948F7932960E94F97BDF01E0
:10B5A4000E9416740E9409633BC0E33051F40E9468
:10B5B4008F7932960E94F97BE081EA930E94266398
:10B5C4002FC0E43069F50E948F7932960E94F97B8E
:10B5D400E093640CF093650C10E00E948F7935962B
:10B5E400E4911E1790F40E948C71EC5BF44F0F01F0
:10B5F400A091640CB091650CEC91D001EC93A4E69D
:10B60400BCE00E94C16E1F5FE8CF0E948F7935961F
:10B61400E491F0E00E9463790E94D7740E946F6302
:10B62400F7C1E33581F5E091400BEA930E94C3181A
:10B63400E091430BE43229F4EAE0F0E00E948B79D4
:10B6440021C0E33211F41ED81DC0EE34D9F40E9497
:10B654002F5310E01A3068F40E948C71EC5BF44FA5
:10B664000F01A4EBBBE00E94C175D001EC931F5FF6
:10B67400F1CFE0E0E0934E0B0E94D7740E946F6319
:10B684000E945578C5C1E63511F00C94865BE091B3
:10B69400400BEA930E942719E091430BE43229F40A
:10B6A4000E946A750E943A532EC0E33219F40E9434
:10B6B400445329C0E53459F40E942F53E091300CCF
:10B6C4000E94B0740E949779E091330C19C0E6355A
:10B6D40029F40E942F53E091310C12C0E43599F4FF
:10B6E4000E942F53E091320CE03011F0E1E301C0ED
:10B6F400E0E3EA930E94D6620E949D79E091320CC5
:10B70400F0E00E94E37884C1E03511F00C94D75C3A
:10B71400E091400BEA930E949418E091430BE432C9
:10B7240029F4E0E4F0E00E948B793EC1E33219F49D
:10B734000E94445339C1E13411F00C94E35B0E943C
:10B744002F5312E0A0919B0BECEDEA233E2F00E077
:10B754000D3078F40E94F9740E94FD74E31739F4F3
:10B764000E94F974EA0FFB1F3396149102C00F5F15
:10B77400EFCF0E949F6D0E944B78E091990BE030CF
:10B7840089F0E6E3F9E10E9417730E94796D0E9443
:10B79400B0740E949779E091990BEF700E94B07495
:10B7A4000E944B78E0919A0BE03051F0E9E3F9E123
:10B7B4000E941773E0919A0B0E94B0740E944B7818
:10B7C400F3C0E43479F50E94A179A091410BA33030
:10B7D40040F5E091410BE03011F00E949D790E9408
:10B7E4007D79EC91E17061F4A4EABBE00E94837975
:10B7F4000E940C6E0E9416740E947863E3E70BC0EB
:10B80400A4EABBE00E9483790E940C6E0E94167425
:10B814000E940963E9E4EA930E94D6620E94707967
:10B82400D4CFBEC0ED34C9F40E94A179A091410BDC
:10B83400A33090F4E091410BE03011F00E949D7927
:10B84400AAEABBE00E94A779EC910E94B0740E941E
:10B8540009630E947079EACFA3C0E735C9F40E9456
:10B86400A179A091410BA23090F4E091410BE0301A
:10B8740011F00E949D79A1EBBBE00E94A779EC91A5
:10B884000E94B0740E9409630E947079EACF88C054
:10B89400E63531F50E94A179A091410BA330F8F46B
:10B8A400E091410BE03011F00E949D79AEE9BBE0DC
:10B8B4000E94A779EC910E94B0740E940963EBE2A4
:10B8C400EA930E94D662A1EABBE00E94A779EC91B8
:10B8D4000E94B0740E9409630E947079DDCF60C039
:10B8E400EE34D1F40E942F5310E01A3068F40E9411
:10B8F4008C71EC5BF44F0F01ABE8BBE00E94C175A7
:10B90400D001EC931F5FF1CFE0E0E0934E0B0E9477
:10B91400D7740E946F6344C0E33499F40E942F5398
:10B924000E94D774E1E4F9E1FA93EA930E941D704E
:10B934000E942F740E94BC750E94D7740E946F638A
:10B944002FC0E035A9F40E942F53E091AD0BF09184
:10B95400AE0BFA93EA930E9490630E949D79E09162
:10B96400AF0BF091B00BFA93EA930E94906318C066
:10B97400E33531F40E942F53E091980BEF5F0DC033
:10B98400EF3491F40E942F530E94796D0E94B07499
:10B994000E949779E091990BEF70F0E00E949379FF
:10B9A400EBE3EA930E94D66233C0EB3489F5E0916D
:10B9B400400BEA930E94E918E091430BE43229F426
:10B9C400E0E8F0E00E948B7923C0E33219F40E948E
:10B9D40044531EC0E134E1F40E942F53A091350C6E
:10B9E400E1E0EA230E94B0740E949779A091350C9B
:10B9F400E3E0EA230E94B0740E949779E091360C48
:10BA04000E94B0740E940963E4E4F9E10E94177390
:10BA14000E946C6131CD0E94D57D249608951A93BD
:10BA24000E946072E0E4F9E00E9431730E94AB79F5
:10BA3400E181E43471F40E94AB7902800E941E6EAD
:10BA4400E05DE01529F00E94AB79E281EA3209F465
:10BA540001C05BC00E94B0790E94AB79E1810E9471
:10BA6400B4790E94AB79E2810E94B4790E94257373
:10BA74001C910E94AB7933960E943173E12FE2311D
:10BA840039F40E94F1781397E6E0EC93D4D93DC0E1
:10BA9400E13139F40E94F1781397E2E1EC93EADCA6
:10BAA40034C0EF30B1F40E94F1781397EEE0EC93D8
:10BAB4000E945853E13039F4A0913508A03019F0B0
:10BAC4000E94187809F402C00E94141C0E94B779DD
:10BAD4001CC0EE30D1F40E94F1781397EFE0EC93A0
:10BAE4000E945853E13089F4A0913508A03019F030
:10BAF4000E94187809F402C00E94141CE0E0E0934C
:10BB04003508EFEFEA930E94DD530E94F178E0E0FC
:10BB1400EC936BC21A930E942A740E947F70EAE726
:10BB2400EA930E94D6620E94257311971C91E12F1B
:10BB3400E23131F4E6E0EA930E94D6627CD937C060
:10BB4400E13131F4E2E1EA930E94D66293DC2FC042
:10BB5400EF3099F40E94C0780E945853E13039F4D0
:10BB6400A0913508A03019F00E94187809F402C099
:10BB74000E94141C0E94B7791AC0EE30C1F4EFE0A1
:10BB8400EA930E94D6620E945853E13081F4A09156
:10BB94003508A03019F00E94187809F402C00E94F8
:10BBA400141CE0E0E0933508EA930E94DD530E9400
:10BBB400F178E0E0EC93A0913808AA3211F00E94E9
:10BBC400BC6313C2EFEFE093580BE093590B089555
:10BBD400AC81A03310F0AA3308F006C00E94BE79ED
:10BBE400E0530E94C6799FC4AC81A13410F0A734FD
:10BBF40008F006C00E94BE79E7530E94C67993C438
:10BC0400A881B981E0E0EC938EC4AA93EA93FA93F5
:10BC1400EFB7EA931A930A931BB10CB1E091A00C0D
:10BC2400F0E0E259F34F0083A091A00CAF5FA09322
:10BC3400A00CA23319F4E0E0E093A00C099119914F
:10BC4400F7C21A93E091A10CA091A00CEA17D1F3CA
:10BC5400F0E0E259F34F1081A091A10CAF5FA093E3
:10BC6400A10CA23319F4E0E0E093A10CBDC1A091B2
:10BC7400A00CAE5CE091A10CAE1BE2E30E94A07BA1
:10BC840008950A921A92FA926A937A938A939A93EB
:10BC9400AA93BA93EA93FA93EFB7EA930E94CB7903
:10BCA40049F0A0913909A03021F00E94ED0CE13057
:10BCB40009F401C011C0E091070DF0E0EE55F34F17
:10BCC400E081ECB9A091070DAF5FA093070DA436F6
:10BCD40019F4E0E0E093070DE991EFBFF991E991E0
:10BCE400B991A9919991899179916991F990199052
:10BCF400099018951A930E94CB7959F45D9B09C059
:10BD0400A0913909A13021F40E94ED0CE03009F032
:10BD140013C01091060D0E948C71EE55F34FA9814A
:10BD2400A0831F5F143609F410E0E091070DE117BA
:10BD3400E1F31093060D02C0E981ECB9A5C20E949B
:10BD4400CB7921F40E94ED0CE13009F001C01DC350
:10BD540054C10E94CE7D8BDFE03011F40C94AD5FB2
:10BD640070DF1E2FA0916B0CA53618F0E0E0E09375
:10BD74003A0930913A09E0913A09E03011F00C9413
:10BD8400145FA091E50BA13041F0A091E50BA23026
:10BD940021F0A091E50BA53031F4E12FEF77E0938A
:10BDA4004009EBE4CEC01A3521F4E1E0E0933A090E
:10BDB400CAC0123049F4E4E1E0933A09E0E0E093C8
:10BDC4003B09E0933D09BFC0A091E50BA33069F4A2
:10BDD400173729F01A3310F4103308F402C0E7E0DF
:10BDE40001C0E0E0E0933C0905C01A930E94DB4DDA
:10BDF400E0933C09A0913C09AF3F99F010934009AE
:10BE0400E1E0E0933B0910933D09E0913C09E03007
:10BE140011F4E5E404C0EAE0E0933A09E0E0E093D9
:10BE24003F0991C0E13069F4103039F4E2E0E09365
:10BE34003A09E0E0E0933F0903C0E0E0E0933A0907
:10BE440082C0E23059F410933C0910933D09E0E0BC
:10BE5400E0933B09E3E0E0933A0975C0E330F1F481
:10BE64000E94D1790E94D779EA0F0E94E179A9F45E
:10BE7400E0913D09E03071F4E4E0E0933A09E091A7
:10BE84003B090E94C56F0E94EA790E94D179A0E023
:10BE9400A08303C0E0E0E0933A0955C0E43049F4DC
:10BEA4001D3019F4EAE5E0933F09E0E0E0933A0934
:10BEB4004AC0EA3079F40E94D1790E94D779EA27FE
:10BEC4000E94E17931F4E0E0E0933A09E5E4E0939B
:10BED4003F0939C0E431B9F40E94D1791083E12FCC
:10BEE400A0913D09EA27E0933D09E0913B09EF5F0A
:10BEF400E0933B09E0E0E0936A0C133019F4E5E1C8
:10BF0400E0933A0920C0E53111F0E63159F41A936F
:10BF1400EAE6FCE0FA93EA93EAE3F9E0FA93EA93B7
:10BF240057DE11C0E73179F4E0E0E0933A091731C4
:10BF340031F4E0916A0CA0913D09EA1709F003C0BD
:10BF4400E3E4E0933F09A0913A093A1719F0E0E0DD
:10BF5400E0936B0C00CF0E94D57D50C4AA93BA9392
:10BF6400EA93FA93EFB7EA931A930A9310919B001A
:10BF740000919C00E12FEC71A9F4E091D00DF091B7
:10BF8400D10DE85FF24F0083A0EDBDE00E94C16EC9
:10BF9400E83CA0E0FA0731F4E0E0F0E0E093D00DF3
:10BFA400F093D10D09911991E991EFBFF991E991BC
:10BFB400B991A99118951A930E94EF790E94F47986
:10BFC400D9F30E94EF79E85FF24F1081A2EDBDE052
:10BFD4000E94C16EE83CA0E0FA0731F4E0E0F0E032
:10BFE400E093D20DF093D30DE12F199108950E949F
:10BFF400EF790E94F47909F0C8C1E0E008950E9445
:10C00400CE7DF5DFE03021F0A091690CA03009F07D
:10C01400E5C0D1DF1E2FA091DC0DA53618F0E0E0BD
:10C02400E093D60D3091D60DE091D60DE03059F461
:10C03400113019F4E4E0E093D60D1A3519F4EAE06E
:10C04400E093D60DC3C0E430C1F4E0E0E093D60D34
:10C054001A3229F00E941E6EE05DE11769F4109314
:10C0640038081093D70DE5E0E093D60DE0E0E093B7
:10C07400690CE1E0E093D90DA9C0E530A9F4E0E052
:10C08400E093D60D0E941E6EE05DE11761F00E9400
:10C09400FB790E94047AE091D90DEF5FE093D90D0A
:10C0A400E6E0E093D60D92C0E63091F4E091D90D2C
:10C0B4000E94047A0E94FB79EF5FE093D90DE0E0DF
:10C0C400E093DA0D133019F4E7E0E093D60D7EC067
:10C0D400E73011F0E83059F41A93EAEDFDE0FA93F1
:10C0E400EA93E6EDFDE0FA93EA9372DD6FC0E9307E
:10C0F40081F4E0E0E093D60D173131F4E091DA0DEC
:10C10400A091D70DEA1709F003C0E4E5E093690CA8
:10C114005DC0EA3041F4103011F4EBE001C0E0E01E
:10C12400E093D60D53C0EB3071F4E0E0E093D90D09
:10C134001093D80D1093D70DECE0E093D60DE0E00A
:10C14400E093690C43C0EC30A1F5E091D90DF0E027
:10C15400E05CF64F10830E94FB79EF5FE093D90D0A
:10C16400E091D80DE150E093D80DA091D80DA03006
:10C1740021F4A091D70DA03009F00EC0EDE0E093BA
:10C18400D60DE091D90D0E94C56F0E94EA79E09125
:10C19400D90DF0E00E94EA79A091D80DA03021F4E5
:10C1A400A091D70DA03009F403C0E0E0E093D60DD0
:10C1B4000DC0ED3059F4E0E0E093D60D1D3031F4BC
:10C1C400EAE5E093690CEFEFE093680CE091D60D9B
:10C1D400E31719F0E0E0E093DC0D13CF0E94D57D66
:10C1E4000DC3AA93EA93FA93EFB7EA93E091DE0EB4
:10C1F400A091DD0EEA1791F0E0913708E03019F0D4
:10C20400E89426F80AC00E94097AF0E0E030A1E040
:10C21400FA0719F4E0E0E093DE0E03C0E89425F891
:10C2240026F8E091680CE03019F0E0E0E093D60DD8
:10C23400E991EFBFF991E991A99118951A93E091C9
:10C24400DE0EA091DD0EEA1721F4E0919B00E0726E
:10C25400C1F4E091DD0EF0E0E352F24FA981A08336
:10C264001091DD0E1F5F0E94DF6CA030E1E0BE077D
:10C2740009F410E0E091DE0EE117E1F31093DD0E16
:10C2840003C0E981E0939C00188122960895E0E0C0
:10C29400E093DE0EA091DD0EA13020F00E94097A19
:10C2A400689426F80895AA93BA93EA93EFB7EA93A9
:10C2B400E091680CE03041F4E0E0E093DE0E0E948F
:10C2C4001E6EEF5FE0933708E991EFBFE991B991F2
:10C2D400A99118950E94187918F00E941C7909F404
:10C2E40003C00E941B74F6CF0E941C7911F40E94B3
:10C2F4001B7408950E942573AC91E881EA1729F410
:10C304000E941B743197E1E05EC1E0E05CC10E94D1
:10C31400CE7D00E010E0EEE20E946879E9F420E0CE
:10C3240030E0EC810E941078BCF4D8010E94E674DD
:10C334008F010E94ED7818F00E94177A08F009C066
:10C344000E942573EC910E949D730E0F1F1F0E9483
:10C354001B742F5F3F4FE5CFF801E3C00E941879AB
:10C3640028F00E94AB79E181E03208F410C00E9409
:10C374002573EC91E093420B0E941B740E94257379
:10C38400EC91E093430B0E941B74E1E008950C943C
:10C39400BB661A930A9300E010E01230A8F40E94DE
:10C3A40020790E945968EF3F69F0E02FE295E07F21
:10C3B400EF930E9420790E945968AF91EA0F0E2FE3
:10C3C4000E941B741F5FE9CFE02F1EC01A930A93CB
:10C3D40010E00E9425730C910B3311F0003208F425
:10C3E40012C0013310F0093308F007C0E02F0E9497
:10C3F4009D73E255FF4FE4911E2B0E941B740E9413
:10C4040025730C91E9CFE12F0991199108950E94A8
:10C41400CE7D00E010E00E942573AC91AD3221F492
:10C424000E941B7431E001C030E00E94ED7818F0E6
:10C434000E94177A08F009C0D8010E94E6740E948D
:10C444001B7A8F010E941B74F0CF303021F4F80165
:10C454000E94D57DD3C1F8010E94E57A0E94D57D62
:10C46400CDC124971A93E0E0E983EA83EB83EC835C
:10C474000E942573AC91AD3221F40E941B7411E02B
:10C4840001C010E00E94ED7818F00E94177A08F0BD
:10C4940022C0A981BA818B819C81EAE0F0E060E04E
:10C4A40070E00E944B7B7F936F93FF93EF930E9406
:10C4B4002573EC91E053AF91BF918F919F91FF272A
:10C4C400662777270E94DB7AE983FA836B837C8370
:10C4D4000E941B74D7CF103031F4E981FA816B814B
:10C4E4007C81188120C0E981FA816B817C810E9462
:10C4F400E97A188118C00E94CE7D20E030E000E087
:10C5040010E0EC810E9473765CF4D9010E94E67419
:10C514000E941B7A9F010E941B740F5F1F4FF1CF73
:10C52400F9010E94D57D259608950E94CE7D6FDF86
:10C534008F0120E030E0EEE20E94687911F467DFB9
:10C544009F01112322F4F9010E94E57A9F01A09131
:10C554001C0CA13030F0D8010E942B72E20FF31FA3
:10C564008F01F8010E94D57D49C11A9310E00E9401
:10C574001279A1F00E94187958F00E942573AC91A9
:10C58400A23231F00E941C7919F0E9811E1708F0DB
:10C5940005C00E948C710E945A79ECCF0E948C7164
:10C5A4000E9463790C941767E8810E94B479E8814A
:10C5B400A0915C0BEA0FE0935C0BE881A0915D0B0A
:10C5C400EA27E0935D0B219608951A9310E0E12F7A
:10C5D400A981BA810E94F574E491E03049F0E12F19
:10C5E400A981BA810E94F574E4910E94217AEFCF67
:10C5F4000BC01A9310E00E946476E03029F00E9488
:10C6040064760E94217AF7CF18812396089564975F
:10C614000E947E750E94267AE88DF98D0E942F74FF
:10C624000E94AE75E6DF6696089564970E947E7553
:10C63400EDE4F9E1FA93EA93E88D0E949C6C0E9480
:10C644007E75D7DF659608951A93ECE3EA93ACDF21
:10C6540011E0193080F40E948C71E255FF4FE4918F
:10C66400A981EA2319F0E12FE05D01C0E0E2EA9339
:10C674009BDF1F5FEECFEEE3EA9396DF0C94176720
:10C6840064971A930E942B7A0E94267AEA8DFB8D76
:10C694000E942F740E94BC750E942B7A0E944169EB
:10C6A4001E2FED891E1720F40E9451781F5FF9CFC9
:10C6B4000E942B7A9EDF18810EC064970E947E75BB
:10C6C4000E94267AE88DF98D6A8D7B8D0E94837491
:10C6D4000E947E758EDF689608950E9487790E9475
:10C6E400F97787DF0E9487790C941867A881B9814C
:10C6F400E4E6F0E00E94717B0E949379EEE2EA9313
:10C7040053DFA881B981E4E6F0E00E94A37BFA93A9
:10C71400EA93E2E0EA93B4DF0C941867A0911C0C4E
:10C72400A13020F00E94F977E1DF07C00E94F97779
:10C734006EDFE2E5F9E10E9417730C94186725FE99
:10C7440006C0E5E0F0E00E949C6EA895F8CFEDED00
:10C75400FDE0E0935E0BF0935F0BE1E00E946772F3
:10C76400E0935C0B0E94307A0E941E6E0E94B478A3
:10C774000C9482691A930A93E091680CE03011F0EA
:10C784000C948A68E3E0EA930FDFE0915C0BE29596
:10C79400EF70EA930E9470681E2FE0915C0BEF70BB
:10C7A400EA930E9470680E2F1A93FEDE0A93FCDE51
:10C7B400E7E1EA93F9DEEDEDFDE00E94F1780E94F5
:10C7C4000D7CEA1BE093DD0E689425F80C948A68CE
:10C7D400EE81EA93B4DFEC81FD810E9417730E941D
:10C7E400347A6BDFC7DF0C94A969EB81EA93A7DF86
:10C7F4000E948771EADE0E94307ABCDF2496089595
:10C80400ED81EA939CDFEB81FC810E941773EA813E
:10C81400EA93CADEE981E03011F0EA93C5DEE881EB
:10C82400E03011F00E94307AA5DF269608950E9428
:10C83400CC7D10E0E6E5F9E1A885B985EA17FB07A8
:10C8440019F444E150E002C048EC50E0EA85E0937A
:10C854003809E89431F8EA93E985FA85FA93EA937A
:10C86400EA85EA93EA85EA93E0E0EA93C9DF0E9465
:10C8740081689F010E94D1140E94AF760E948D6846
:10C884000E2F31FC02C0003009F001C0F3CF31FE9D
:10C8940004C0E89431F8E1E004C01F5F1230B0F244
:10C8A400E0E00E94D37D2B9608951A930A93E091B9
:10C8B400400AE03011F40C948A68E0E0E09339090E
:10C8C400E2E0EA9317DA10E003E00E948C710E9420
:10C8D4003B7A61F00E948C710E9415780E948C71E1
:10C8E400E05CF54FE0810E271F5FEFCFE3E0EA93B2
:10C8F40001DAE02FE295EF700E94407AE02FEF70AA
:10C904000E94407AE7E1EA93F5D90C948A681A9375
:10C914000A93E091400AE03011F40C948A680E9472
:10C92400A270E03021F0E091420AEA3209F405C035
:10C934000E94A270E05DE093420AE0E0E0933909CE
:10C94400EAE5EA93D7D9E0E0EA93D4D910E00E946B
:10C954008C710E943B7A11F01F5FF9CF1F5F012F8A
:10C964000A93C8D910E00E948C710E943B7A61F04E
:10C974000E948C710E9415780E948C71E05CF54FC6
:10C98400E0810E0F1F5FEFCFE02FE195EA93B2D95C
:10C99400EDE0EA93AFD90C948A681A930A93F89459
:10C9A400E0E0E0933708E091DE0EE093DD0E78944A
:10C9B400E091400AE03011F40C948A68EAE5EA93C5
:10C9C4003DDCE0E0EA933ADC10E00E948C710E94C6
:10C9D4003B7A11F01F5FF9CF1F5F012F0A932EDC02
:10C9E40010E00E948C710E943B7A79F00E948C7155
:10C9F400E05CF54FE081EA9321DC0E948C71E05CFD
:10CA0400F54FE0810E0F1F5FECCFE02FE195EA9325
:10CA140015DCEDE0EA9312DC0C948A68E881EA9371
:10CA24008EDEEAE5EA93C0DDE0914009EA93BCDDDD
:10CA34000E942573EC91E03031F00E942079B4DD3E
:10CA44000E941B74F5CF96DE0C9482691A930E949F
:10CA54006072E0913B08EA93A7DDE4E4EA93A4DD85
:10CA6400E0913908EA93A0DD14E00E948C71E85C3F
:10CA7400F74FE081E43040F00E948C71E85CF74F9E
:10CA8400E0810E94217AF1CFE0E0EA938DDD3FDF7F
:10CA94006BC11A930A935DD9E0913F09E03011F418
:10CAA4000C94C865A0913F09AA3541F4A0913B09B3
:10CAB400A33020F0E0914109E43409F04BC00E9416
:10CAC400A270E03021F0E0914209EA32C1F40E9400
:10CAD4001E6EE05DA0914209EA1721F0E09142093F
:10CAE400EA3221F40E94115D12DF08C0E3E4F9E0A8
:10CAF4000E943173E09142090E94467A2BC00E9441
:10CB0400A270E05DA0914209EA1721F50E941E6E11
:10CB14001E2FE0914309ED3421F4E0914409E332FE
:10CB240009F007C0E5E4F9E00E94317370DC1E2FC0
:10CB3400D1DB0E941E6EE11729F0E12FE05D0E9417
:10CB4400467A08C00E941E6EE05DE09342090E948E
:10CB5400115DDDDEA0913F09A53449F4A091E50BF8
:10CB6400A33019F40E94C12A02C00E944E4EA09123
:10CB74003F09A33411F40E94722AA0913F09AB34F7
:10CB840011F40E946D2AE0E0E0933F09A091E50BC7
:10CB9400A33011F40E94C12AE0E00C948A682FDAD1
:10CBA400A091690CA43529F4A0E025FCA1E0A030F3
:10CBB40009F03AC0E0913A08E03581F4E0913B088D
:10CBC400EA93E6E0EA930E94C542A0913B08A038AC
:10CBD40020F0E0913B08E093650523C0E03721F4A1
:10CBE400E0E0E09365051DC0EA3519F40E948C5D10
:10CBF40018C0EA3711F42ADF14C0E23519F40E9490
:10CC040061500FC0E23719F40E9496500AC00E9486
:10CC14004430E0913908A0913809EA1711F4689476
:10CC240031F8E0E0E093690CA091690CAA3531F485
:10CC34000E94115DB2DEE0E0E093690C9AC0A0911D
:10CC44006C0CA13050F0E0916C0CE150E0936C0C52
:10CC5400E03019F4E1E0E0936D0CA0E025FCA1E0E4
:10CC6400A13049F4A0E026FCA1E0A03021F4A09179
:10CC74003708A03009F001C00ADBE0913708E03042
:10CC840019F0E150E09337080895E091DC0DEF5F6F
:10CC9400E093DC0DE0916B0CEF5FE0936B0CE091A3
:10CCA400680CE03019F0E150E093680C0895A0910D
:10CCB400E50BA13041F0A091E50BA23021F0A09149
:10CCC400E50BA53029F4E3E0E0939000E8E3E9B94B
:10CCD4000895E091620BE0937100E0E0E09374004A
:10CCE400E2B3E360E2BBE1B3E360E1BB85E38A95D1
:10CCF400F1F7E1B3EC7FE1BBE4E4E093740088EC8A
:10CD040090E00197F1F70895E2E001C0E0E0E093DC
:10CD1400620BDFDF08951A931FEFF6DF16D0E030C1
:10CD240089F4E9810E944D7A41F4EDB7FEB7FA9394
:10CD3400EA931F930E94527A1F9118D080E991E0E0
:10CD44000197F1F7E3DFE12F70C01A9314EAE4EAE4
:10CD54000E94567A41F40E945B7A183011F0103127
:10CD640011F4E0E001C0E2E019910895E4E9E093F0
:10CD74007400E0E008951A93E981E1600E94607A0A
:10CD840031F40E945B7A103411F4E0E04EC04CC0E0
:10CD94001A93E9810E94607A31F40E945B7A183117
:10CDA40011F4E0E042C040C01A93E9810E94607A25
:10CDB40031F40E945B7A183211F4E0E036C034C0DA
:10CDC4001A93E981E03011F0E4EC01C0E4E80E9438
:10CDD400567A79F40E945B7AE0917300AA81BB8150
:10CDE400EC93103511F0183521F4E0E018810C941F
:10CDF400FF6BE1E018810C94FF6B1A93E981E093D7
:10CE0400740010E0E0917400E07811F4163908F031
:10CE140005C08BE18A95F1F71F5FF4CFE0917400B0
:10CE2400E07811F0E0E001C0E1E018812296089575
:10CE34000E94CE7D3D810C8120E087DFE03011F53A
:10CE4400EE810E944F6FF1F43A93AEDFE030D1F4FB
:10CE54000E94647AB9F479DFE030A1F4EE810E9493
:10CE64004D7A81F4EDB7FEB7FA93EA931F930E94CB
:10CE7400527A1F91E03031F479DFE12F0E94D57DA1
:10CE84000C94A96926DFD9CF0E94CE7D30E00E81B3
:10CE94001D815BDFE03099F4EF810E944F6F79F4DC
:10CEA4000E94647A61F41A937FDFE03041F4EC81EC
:10CEB400EA937ADFE03019F459DFE0E002C009DFD9
:10CEC400E8CF0E94D57D2896089522970E94CC7DB4
:10CED40050E02B853A85A89538DFE03011F00C94AA
:10CEE400C967EE850E944F6F11F00C94C9672A93AD
:10CEF4005BDFE03011F00C94C9673A9355DFE03002
:10CF040011F00C94C96721DFE03011F00C94C9676B
:10CF1400EE850E944D7AD9F5E0E0EE83EF83EC854F
:10CF2400FD8531970E94387649F4EDB7FEB7FA9340
:10CF3400EA931F930E94527A1F9109C0EDB7FEB77E
:10CF4400FA93EA931F93E1E0EA933ADF1F910E2FDD
:10CF5400EE81FF81A885B985EA0FFB1F1083EE815E
:10CF6400FF813196EE83FF83003039F4EC85FD8533
:10CF7400AE81BF81AE17BF0708F001C0D0CFEC85EA
:10CF8400FD850E94387619F4F1DEE0E002C0A1DEEE
:10CF9400A3CF0E94D37D2F96089568970E94CC7DDD
:10CFA40020E0E0E0EC8FED8F31E0A895E9A1FAA153
:10CFB400662777270E94A37CEA87FB876C877D8797
:10CFC400EE8D0E94697AEE83FF8368877987AA854C
:10CFD400BB858C859D850E94797DEA8BFB8B6C8B50
:10CFE4007D8B0E94FD7BFE017296FA93EA930E9468
:10CFF400016CEE8BFF8B688F798F0E946F7A0E9491
:10D004006A7CAF010E946F7AAE8DBB27882799276F
:10D014000E94047C0E94827ADE015A960E946A7CF5
:10D02400ED93FC930AA119A190DEE030D1F5EDA1B6
:10D034000E944F6FB1F50E94647A99F51A93B4DE99
:10D04400E03079F5303051F14F5F5F4FEC8DFD8D5D
:10D054003196EC8FFD8FAC8DBD8D1197EBA1FCA1AA
:10D06400EA17FB0711F430E018C0EC8DFD8D319701
:10D07400AF8DB8A10E94787697DEEE8DDA01F0E0EC
:10D08400EA17FB0751F472DEEA8DFB8DA9A1BAA160
:10D09400EA0FFB1FE9A3FAA389CFD4CF67DEE0E050
:10D0A40002C017DEC1CF0E94D37DA6960895A88141
:10D0B400A03310F0AA3308F004C0E881E0530C94C4
:10D0C4008269A881A13410F0A73408F004C0E88173
:10D0D400E7530C948269EFEF0C948269A881AA301B
:10D0E40020F4E881E05D0C948269A881AA3020F0E4
:10D0F400E881E95C0C948269E8E50C9482691A93EE
:10D104000A93F8940091630B1091640B7894F801DE
:10D114000991199108951A930A93F1DF8F01EA8115
:10D12400FB81AC81BD81EA0FFB1FE01BF10BDF012A
:10D134000E94C27D2CF4E0E0198108810C942D6CCE
:10D14400E1E0198108810C942D6CE2E9F4E1FA9391
:10D15400EA93EAEBF0E0FA93EA930E946A75E4E05A
:10D16400EA93E6E2EA93EEE0EA930E947A4DEAE279
:10D17400F5E1FA93EA93EAEAF0E00E94877AE8E0BC
:10D18400EA93E0E2EA93E1E0EA930E947A4DEAE26C
:10D19400F6E1FA93EA93E2EDF0E00E947D6CFA93F3
:10D1A400EA93E2E0EA93E2E1EA93E1E0EA930E949F
:10D1B4007A4D0E94566C0E94AD6EEFEAF0E00E9438
:10D1C400877AE3E0EA930E94904BEAE0F0E0FA9376
:10D1D400EA93E4E3F0E00E94986EE0E0E093100448
:10D1E400EAE5F9E10E94B86DEFE0E09310040895D8
:10D1F400089599818881009641F0BD81AC81FB81BD
:10D20400EA8105900D920197E1F7FD81EC810C9480
:10D214002D6CB981A881109631F0FC81EB816A8173
:10D2240061931197E9F7EB81FC8125960895E991C3
:10D23400F991A991B9911D900590011421F4002050
:10D24400D1F7EE2708951018E1F3E1E008F4E25075
:10D254000895E991F991A991B991CD0161916D93E5
:10D264006623E1F7FC010895E991F991A991B99137
:10D27400CD0105900D920020E1F7FC010895A991DC
:10D28400B991EE27FF276D91662311F03196FBCFFC
:10D294000895AA27BB27E991F9910590002011F080
:10D2A4001196FBCFFD0108957991E991F991A99126
:10D2B400B991CD01772351F07A9561916D936623ED
:10D2C400C9F7772319F07A956D93FBCFFC01089584
:10D2D4006991E991F991A991B991CD01662351F030
:10D2E4006A9505900D920020C9F7662319F06A9596
:10D2F4000D92FBCFFC0108955D9BFECFE881ECB954
:10D30400219608951A930A93AC81BD810E94EA7B09
:10D314003097C1F0AA81BB810E94EA7B8F013097CC
:10D3240049F00230E0E01E0760F0F80131978F0108
:10D33400ED93FC93AC81BD810E94C16E3197AE81A7
:10D34400A08303C0EE81EA93D7DF19810881279671
:10D3540008952C970E94CC7D10E0E88DF98D3196CC
:10D36400E88FF98F3197E4912E2FE03011F40C946B
:10D37400696BE12FE03039F4253211F411E002C079
:10D384000E948E7AA3C1E130C1F4253219F40E94BF
:10D394008E7A9BC112E0E0E0E98B00E02D3211F4BB
:10D3A40001E094C12B3219F4EBE2E98B8FC12032F6
:10D3B40019F4E0E2E98B8AC102C0E23039F450E0AA
:10D3C40013E0203311F4006881C102C0E330A1F4FA
:10D3D400203310F02A3308F009C0A52FEAE0EA9FB1
:10D3E400F0015E2FE22FE0535E0F70C140E02E3259
:10D3F40011F414E06BC110C0E430A1F4203310F038
:10D404002A3308F009C0A42FEAE0EA9FF0014E2F66
:10D41400E22FE0534E0F5AC12C3619F4026015E086
:10D4240055C104C0E53011F00C94686BE22FE3366B
:10D4340049F40E94997AEE89FF89A481AA930E94F3
:10D444009F7A43C1E33741F40E94997A0E94A97AF2
:10D454000E9441691E2F0AC0E037A1F40E94997A04
:10D464000E94A97A0E944B691E2F08600F774030F2
:10D4740011F0411708F001C0142F40E0E0E0E88B00
:10D4840030E076C0E43611F0E93611F4046002C0ED
:10D49400E537A1F4EAE0E88B01FF08C0E0E0FAEC2C
:10D4A4006AE97BE30E947B6E1AE023C0E0E1F7E2C5
:10D4B40060E070E00E947B6E15E01BC0E83511F45B
:10D4C400086004C0E83711F00C94676BE0E1E88B66
:10D4D40001FF08C0E0E0F0E060E070E10E947B6ED4
:10D4E40018E007C0E0E0F0E160E070E00E947B6ECD
:10D4F40014E0403011F00F7701C041E001FF08C093
:10D504000E94997AAE89BF8914960E94EE7B13C05B
:10D5140002FF08C00E94997AAE89BF8914960E94BE
:10D52400116E09C00E94997AAE89BF8914960E942F
:10D53400EA7B66277727EC87FD876E877F8702FF64
:10D5440016C0AF85AA2362F4EC85FD856E857F85C0
:10D554000E94E97AEC87FD876E877F87EDE2E98B8D
:10D56400E989E03019F01F5F4F5F01C00B7F342F52
:10D5740000FD14C0151710F4351708F00FC007FF8D
:10D5840008C002FF04C00B7F2989115001C020E3A9
:10D5940001C020E20E948E7A5150ECCF1417B0F4EF
:10D5A400006102FF0AC00B7FE989EA930E949F7A17
:10D5B400503009F0515011504150E0E3EA930E9479
:10D5C4009F7A503009F051504150E8CF312FE8890B
:10D5D400E030D1F43030B9F003FF08C0EE81FF81B0
:10D5E4003196EE83FF833197E49105C0AE81BF810C
:10D5F400ED91AE83BF83EA930E949F7A503009F085
:10D6040051503150E7CF57C00E94B17A0E94767BC7
:10D614002E2F2A3030F003FF02C0295C01C0295AA2
:10D6240001C0205D04FD25C0213360F4A885B985BF
:10D634008A859B85A130E0E0BE07E0E08E07E0E04C
:10D644009E0709F40BC0431740F4531710F000FF72
:10D6540001C014C020E207FF0CC020E3006102FFF8
:10D6640008C00B7FE989EA930E949F7A503009F041
:10D6740051500E948E7A503009F0515031500E941E
:10D68400B17A0E94B17BEC87FD876E877F87E8893A
:10D69400A885B9858A859B85FF27662777270E94F9
:10D6A400767B0E947B6EE885F9856A857B850E947E
:10D6B400BE7D09F0A9CF00FF08C0503031F05150B1
:10D6C400E0E2EA930E949F7AF8CF10E046CE0E94EF
:10D6D400D37D6A960895FF92F82E22971A930A939F
:10D6E400DE010E94D77A8D01DE0116960E94D77A58
:10D6F4000E94EA7BEA83FB83DE0114960E94D77AB8
:10D704000E9416741A930A93FE0136960E94826C44
:10D7140020DEAA81BB81E0E0EC9319810881249684
:10D72400FF900895A991B991EE27002460E8E89448
:10D73400162E169407941E2A1EF0A015B10518F093
:10D74400A019B109E62BB7FBAA0FBB1F669580F79A
:10D7540008957B816A81F981E88177FB770F67FD02
:10D764007160972F9E5781F078F0983190F4AA2732
:10D77400BB27882708948795B795A7959A95D1F7DD
:10D78400EA23FB23682305C0E8947727EE27FF27C5
:10D7940066276F77769508F4606877F9A991B9914F
:10D7A40089919991EA17FB076807790797FB089510
:10D7B4000E94347A0E94BA7A19F40E94C17A1DC078
:10D7C400E6F7A881B9818A819B81E0E0F0E060E816
:10D7D4007FE30E94827A11C00E94347A0E94BA7A4E
:10D7E40019F40E94C17A09C0E6F30E94C17AA0E04C
:10D7F400B0E080E89FE30E94DD7C249608950E94B7
:10D80400C67A0E94BE7D39F4A881B9810E94537002
:10D814000E94F47B20C0AA81BB818C819D810E94DF
:10D82400C67D34F40E94C67A0E94FD7BC1DF05C028
:10D834000E94C67A0E94FD7BCFDFA881B9810E9435
:10D84400F47BA881B9810E94EE7BAA81BB818C8183
:10D854009D810E94827A26960895E991F9913097E4
:10D864001AF4E095F095319608950E948666E0EBEF
:10D87400EA93E8E1F0E0FA93EA93E1E0F0E0FA9366
:10D88400EA93E3E2F7E0FA93EA930895E0EBEA938C
:10D89400E0E0F0E0FA93EA930E941A670C94886639
:10D8A400E0E2EA930C94CF67E0E0F0E0FA93EA93C5
:10D8B4000895EFEEF0E0FA93EA930895FA93EA9369
:10D8C400E0E0EA930C94904BFA93EA930C94794336
:10D8D400E12FA0E4B2E0F0E00E94FD7AEA0FFB1F22
:10D8E4000895A12FB0E0ECE3F0E00E94467B389667
:10D8F400FA93EA930895FA93EA93E2E3F0E0089541
:10D90400FA93EA93D1CFE0911004E0930F040895C1
:10D914000E941B0D0C942949E32FF0E0E05BFD4FBE
:10D92400E4910895EA930E94310DFE013696FA932C
:10D93400EA930895FF27662777270E94FD7B84E0FA
:10D944000E946D6B28960895FE017196FA93EA93EE
:10D954000C9499430E94CE7D0C94A146E8E0F0E03B
:10D96400FA93EA930895E4E0F0E0FA93EA930895D1
:10D97400FA93EA93E8E3F0E0FA93EA9308950E94B5
:10D98400F97BBECFE02FF0E00895A0913B0CB0915D
:10D994003C0CBD01A3E0B0E00E941E7BE60FF71F24
:10D9A400E491E0300895E091C005EE0FEE0FEF5FD3
:10D9B4003E2F0895E32FF0E00895A12FB0E00895DD
:10D9C400A0913B0CB0913C0CBD01A3E0B0E00E94DF
:10D9D4001E7BE60FF71F08950E94FB7AE05AFD4F65
:10D9E4000895FA93EA93E22FF0E008950E94CC7D23
:10D9F400A09119080895E091C30BF0E00895AFE3F6
:10DA0400B1E00E94717B089530911E08E1E0E0933B
:10DA14000D04E2E0E0930E043A930E949418E0911E
:10DA2400990BE295EF70E0930F04E091990BEF707E
:10DA3400E09310040895FA93EA93E52FF0E0FA9343
:10DA4400EA930895E7E3F0E0FA93EA930895E22F66
:10DA5400E450F0E0FA93EA930895EA85FB85FA939B
:10DA6400EA930895E32FE058EA931ECFEBE8FBE036
:10DA7400FA93EA930C9499433A930E949418A091D0
:10DA84008B0BAD320895E091990BE295EF70E09322
:10DA94000F04E091990BEF700895E52FF0E00895DD
:10DAA400EA0FFB1FFA93EA930895EF5EFC4FBF0160
:10DAB400E081E058DB01EC930895E0E0EC93AE8163
:10DAC400BF810895E3E0F0E0FA93EA930895E52F27
:10DAD400E450F0E0FA93EA930895E0E0E0930F0451
:10DAE400EFE0E09310040895E550F0E00895E0912C
:10DAF400990BE295EF700895EA1BA2E5B7E0F0E018
:10DB04000E94FD7A0895F0E0EE0FFF1FEA5CFD4FDE
:10DB14000895A4E3B2E0F0E0EE0FFF1FEA0FFB1F4D
:10DB24000895FA93EA93E12FF0E0FA93EA930895C3
:10DB34000E94A146E0E0EA930895E12FF0E0FA9311
:10DB4400EA930895FA93EA93E2E0F0E0FA93EA9311
:10DB54000895EBE8FBE0FA93EA93EAE0EA930C9485
:10DB64004246E1E0F0E0FA93EA930895FA93EA93E7
:10DB74000C942B460E94F97BFA93EA930895ABE048
:10DB8400EA9FF001E252FA4F0895ED85FE85FA937B
:10DB9400EA9308951A930A932ECF1A930A93E0E016
:10DBA400EA930E94904BDDCFE1E0E0933D0C0E94AC
:10DBB4008168E0933F0CF093400C0895BD01AAE006
:10DBC400B0E00E941E7BE60FF71F0895FA93EA93D4
:10DBD400EAE0EA930C944246E1E0E0930E0464CE5A
:10DBE4000E947A460C945D46E0E2EA930C94144653
:10DBF400A3E2B7E0E881F0E0EE0FFF1FAE0FBF1F16
:10DC04000E94EA7B0895FA93EA930C942C41E881EC
:10DC1400F0E00895EE0FFF1FAE0FBF1F08950E949E
:10DC2400EA7B0E94087B08950E94FD7B0C940D41C1
:10DC3400FA93EA930C947A46A9E0B0E00E94187C27
:10DC44000895A7E11A9FF001EF5CF94FE081089570
:10DC5400E12FEF5FEA930C944241F0E0D4CFE8E087
:10DC6400F0E04ECEEA93E6E0EA930E94F84076CEE6
:10DC7400E093620088EC90E00197F1F70895E09357
:10DC8400610088EC90E00197F1F70895E0916D054B
:10DC9400F0916E050895E0916905F0916A05089583
:10DCA400AE0FBF1FE3E0F0E00E94717B0895FA938A
:10DCB400EA931A930A930C945212FA93EA933A93BE
:10DCC4002A930C945212A0917105B0917205089593
:10DCD400A0917305B09174050895A0E0B0E00E948E
:10DCE400147C08950E940D7CEA1BFB0B0E94087BA8
:10DCF4000895E887F9876A877B870895A885B98599
:10DD04008A859B85EFEEF0E060E070E008950E9464
:10DD1400087B0E949B7B0895A4E0B0E00E94147CE1
:10DD24000895EC83FD836E837F830895FA93EA93C9
:10DD34000C949546FA93EA930C94CB7AA9E01A9F33
:10DD4400F001E058FC4F089537960E94F97BDF01FB
:10DD54000E94EA7B0895E2E3F0E0FA93EA930895DF
:10DD64000A921A92FA926A937A938A939A93AA934A
:10DD7400BA93EA93FA93EFB7EA931A930895ED915D
:10DD8400FD913196FE93EE930895ADE01A9FF00154
:10DD9400EB5FFC4FE08108951A93E1E0EA930C9461
:10DDA4000347ADE01A9FF001DF01EB5FFC4FE08118
:10DDB400E0300895E2E0EA930C940347FA93EA937F
:10DDC400E4E6F0E0FA93EA930E948D68E030089567
:10DDD400E1E0E0930D04E0930E040895E091290836
:10DDE400F0912A0860912B0870912C080895E09115
:10DDF4002108E150A3EAB6E0F0E00E94FD7AAE0FFC
:10DE0400BF1F0E94EE7B0895E12FEF5FF0E010CF7B
:10DE1400E0912208EA93E0911E08EA930E94A61A70
:10DE2400A0911F0CB091200C10970895A091210C83
:10DE3400B091220C8091230C9091240C0E94C67DF9
:10DE44000895E0911F0CF091200C0895E091210CAD
:10DE5400F091220C6091230C7091240C0895EAE057
:10DE6400F0E068CFE2E3F0E065CF1A93E0EAEA93EA
:10DE7400EA81F0E0E054F14FFA93EA930E941A67C2
:10DE84001E2F0895E0EAEA93EA81F0E0E054F14FAE
:10DE9400FA93EA931A930C944667EA930E94CA662B
:10DEA400E0300895E0EAEA93EEE5F0E0FA93EA93CD
:10DEB400E0E0FFE0FA93EA93EFEBFBE00895FA93D6
:10DEC400EA93EECCE0EAEA93E981FA81E050FE4E6F
:10DED400FA93EA930895EA81F0E0A8E2B0E00E94A0
:10DEE400467B0895E0EAEA93E2E0F0E0FA93EA93ED
:10DEF4001A930A930895FA93EA930C946767FA9332
:10DF0400EA930C941A67E0EAEA93E8E2F0E0FA9301
:10DF1400EA931A930A93EBE8FBE00895EBE8FBE03D
:10DF2400FA93EA930895EDE2EA93EAE0F0E0FA93D3
:10DF3400EA930E940B69E0E00895EA81F0E0ABE027
:10DF4400B0E00E94467BE050F24F8F01AA81AA30D4
:10DF54000895E0EAEA93EBE0F0E0FA93EA931A9387
:10DF64000A93E3EBFBE00895E4EBFBE0FA93EA9316
:10DF74000895EA81F0E0EE0FFF1FE050F04F8F01AB
:10DF8400AA81A0380895E150F0E00895EA81F0E014
:10DF94000E94FD7AE058F14F8F01AA81A5300895BF
:10DFA400E0E3FCE0FA93EA93E0E0EA93DCCCEDE111
:10DFB400FCE0FA93EA93E0E0EA93D0CC0E94FD7A85
:10DFC4000E94F97ADF01EA85F0E0AE0FBF1FE8E0B6
:10DFD400F0E00E94467BE050FA4E8F01E0EAEA93BB
:10DFE400BDCC1A930A93EDE1FCE085CFAE81BF81ED
:10DFF400888599850E94DB7AEE83FF836887798719
:10E00400089540931F0C5093200CEE81FF81688586
:10E014007985E093210CF093220C6093230C709388
:10E02400240C0895F0E0AE0FBF1F0895EA930E94F8
:10E0340094180C94631FE091960BF091970B08953C
:10E04400FA93EA930C943318ED81EA93ED81EA9301
:10E054000895E091AD0BF091AE0B0E94087B0895FA
:10E06400F0E0A4E6B0E00E94467B0895EC81F0E085
:10E07400EA0FFB1F0895E0912708F09128080895FE
:10E08400E093280CF093290C0C94F71BE3EAF6E0D8
:10E09400FA93EA93E0E0EA930895FA93EA930C94EE
:10E0A4000B69E0E0F0E060E070E00895E093290897
:10E0B400F0932A0860932B0870932C080895E0913C
:10E0C400980BA3EAB6E0F0E00E94FD7A0895AE0F43
:10E0D400BF1F0E94EE7B0895ED5EF94FE081E130B1
:10E0E4000895FA93EA93E0912208E05DEA93089593
:10E0F400EA930E941964E1300895ECE3F8E0E093B8
:10E10400600BF093610B0895E12FA3EAB6E0F0E011
:10E114000E94FD7A08950E94FB68A881AF5FEAE03F
:10E124000E94507BE05D0895A881AF5FEAE00E9401
:10E13400A07BE05D0895FA93EA93E0E0EA93089502
:10E14400AAE0B0E00E94187C0895E12FF0E00E945C
:10E15400FB7AE854FF4F32960E94F97B0895E12F31
:10E16400F0E00E94FB7AE854FF4F08953696E4915C
:10E17400D901EC930895E0EAEA93E5E0F0E0FA933C
:10E18400EA930895EA930E94E81BFA93EA93E5E27E
:10E19400FCE00895FA93EA93EFEFEA93E5E0F0E008
:10E1A4007CCFE093260CF093270C08950E940D7CFD
:10E1B400EA1BFB0B0895EAE2FCE0ECCFA0912B0CE8
:10E1C400B0912C0C0895E0E0E093390CE0933A0C04
:10E1D4000895A0912D0CB0912E0C0895E0912D0C72
:10E1E400F0912E0CAC81BD81EA0FFB1F0895E093E2
:10E1F4002D0CF0932E0C08951A930E94821C1E2F4E
:10E204000895E0932B0CF0932C0C0895FA93EA9361
:10E214000E948D68E0300895ABE01A9FF001E4524B
:10E22400FA4F08951A930E94711ED3CFE0912B0CDC
:10E23400F0912C0C0895EA930E94711E0E940E1E08
:10E24400E0300895EB81EA930E94A91CFA93EA93C3
:10E25400EAE2FCE00895E0E0E093500CE0934F0C18
:10E2640008951A930A93E0911208ABE0EA9FF00133
:10E27400E752F84F8F01D80111960895E0E0F0E0DD
:10E28400ED93FC930895EA81D801EC93E2E1F8E080
:10E29400FA93EA930E946533198108810895E12F66
:10E2A400ACE8B0E0F0E0EE0FFF1FEA0FFB1F0E94A6
:10E2B400F97B0895E150ADE0EA9FF0010895ACE8E0
:10E2C400B0E0F0E0EE0FFF1FEA0FFB1F0E94F97BA6
:10E2D4000895A0911608B0911708EA2BFB2BE09340
:10E2E4001608F09317080895E150A7E1EA9FF0019A
:10E2F4000895A7E10A9FF001E15DF94FAF01089588
:10E30400ED55F94FE081E0300895E981FA81FA93FF
:10E31400EA930895E12FF0E00895E2E0F0E00E942E
:10E32400717B0895ABE9BBE0E0911A080895AEE96A
:10E33400BBE0E0911A0876CEA1EABBE0E0911A08AE
:10E3440071CEA3E2B7E0A9CBEE0FFF1FEA0FFB1FCC
:10E354000895E081F0E00895A7E11A9FF001E15DDE
:10E36400F94FEE83FF83AE81BF810895EE81FF8173
:10E37400A481AA930C94B91F0D901C90AE81BF8107
:10E384001296EC91F0E0E00DF11DDB01ED93FC93AE
:10E394000895ED91FD913197FE93EE9308950E94B7
:10E3A4005E21EF770E2EAA85BB851296EC91E015BF
:10E3B4000895A3E20A9FF001E855F94F0895E0910A
:10E3C4001208ABE0EA9FF001E752F84FEC87FD87B3
:10E3D400AC85BD85119608951296EC91AC85BD85EA
:10E3E4001696EC930895D001F0E00895A885B985B8
:10E3F40018960E94EA7B0895AC85BD85EC93E2E112
:10E40400F8E0FA93EA930C946533E885F985A281E0
:10E41400AA930895AA85BB85EC91EA93E3E0EA9375
:10E424000C94C542AA85BB85E0E0EC93E2E0E0935E
:10E4340024060895BF0100801180AE81BF81129629
:10E44400EC910895DB01ED93FC93AE81BF811296AC
:10E4540034CBE4E6F0E00E94467B0895F0E0ED93CF
:10E46400FC930895E2E1F8E0FA93EA930C9465339F
:10E47400E0911908A0911808EA170895F0E0E00D5A
:10E48400F11D0895A4EABBE045CFAEE9BBE0EE2759
:10E49400A10FBE1FEC910895A1EABBE0EE27A10FE6
:10E4A400BE1FEC910895BD01AAE0B0E00E941E7B5E
:10E4B400DB010895E081EA930C947C5EE0E4FAE0E9
:10E4C400E0935E0BF0935F0B0895EA930E94D6628B
:10E4D400E0E00895EA930E94D6620C945764AEE992
:10E4E400BBE0EE27A00FBE1FEC910895A1EABBE0AC
:10E4F400EE27A00FBE1FEC910895ABE9BBE0EE2719
:10E50400A00FBE1FEC91E1700895A4EABBE03ACAE3
:10E51400A1EBBBE0EE27A00FBE1FEC910895AAEA81
:10E52400BBE0EE27A00FBE1FEC910895EA81ADE099
:10E53400EA9FF001E15FFC4FA0E0A083EA81EA9347
:10E544000895ADE0EA9FF001EB5FFC4F0895ABE066
:10E554000A9FF001E452FA4F0895ABE00A9FF001DC
:10E56400EE51FA4F0895FA93EA930C94F234FA9325
:10E57400EA930E943A433A931DCCE0912D0CF0911A
:10E584002E0C30970895AFEFBFEFA083B1830895A9
:10E594000E948168E093550CF093560C0895FA9309
:10E5A400EA93E0E0F0E80895E0911208ABE0EA9F16
:10E5B400F001E752F84FFA93EA930E94CE2852CF23
:10E5C400E0911008ABE0EA9FF0010895E0E1F8E083
:10E5D400FA93EA930C946533FA93EA930C940A53EE
:10E5E400E88DABE0EA9FF0010895FA93EA93CAC973
:10E5F400E0E1EA93E0912506EA930E9467181E2F52
:10E60400089539DDFA93EA930895FA93EA930C9402
:10E614003C1EE0932506E0E0E093520CE1E3E09336
:10E62400530C0E940D2A0C94DA25FA93EA930C9465
:10E63400E762E1E4F9E0E093600BF093610BE3E05F
:10E64400EA930C947D62A091600BB091610B0895E4
:10E654000E948168E0934A0CF0934B0C0895E09378
:10E66400600BF093610B0895E3E0EA930C947D62F0
:10E67400E0932708F09328080895E0E0F0E0E093A1
:10E684002508F0932608E2E0E0930E040895E09153
:10E6940013042ACAE0912508F0912608B4CAE0912F
:10E6A4005D05F0915E0531970895FA93EA930C9411
:10E6B4006F45EF5CEA930C941446A3EEB6E07AC976
:10E6C400A4EABBE0E0911A08F0E03ECE0E94EA7BA7
:10E6D400D001ED93FC9326CEF0E0EA0FFB1F0F016F
:10E6E40021CEA3E2B7E066C9E7E0E0931808EA9315
:10E6F400E0E0EA93D9C8EA930E94A1400E94D8427C
:10E704001E2F0895EAE2EA93EDE6F7E114CD0E94A4
:10E71400C22BE1E0EA930C94AA2B1F771A930C9472
:10E724009418A0912508B09126080895E8EEF3E026
:10E734000E94A37B0895E053F0E00895A0E024FC38
:10E74400A1E0A0300895E0E0EA93AEC8E091330878
:10E75400F0913408FA93EA930895FA93EA930E94A5
:10E764008D68E13008950E948168E0933308F09346
:10E7740034080895E0E0E0934F0C0895D2DFEA17DF
:10E78400FB070895E0931808E0E0E093300808954B
:10E794000E94F7630E942B2DE093240808950E94A1
:10E7A40094180C94A146E0911908EA93E0E0EA93E6
:10E7B4000E94D52C0C9480280E94D8421E2F1A93B4
:10E7C4000E945E2D103808951A93E091C605EA93CD
:10E7D4000895E0918A0BEA930E94A117E03008950E
:10E7E4000E948168E093570CF093580C0895FA93B3
:10E7F400EA93F6C9D90118960E94EA7B0895E4E6E3
:10E80400F0E060E070E00E949B7B08950E94941801
:10E8140012CC0A93E091C605EA930895E0912F087B
:10E82400EA930A930C94C5190E94EA7BFA93EA933B
:10E834000895A0E6BBE0A3CAE0913C08E053E0934E
:10E8440022080895FA93EA93E0E3EA930C94F763B9
:10E85400E0913908EA930C94A1630E94087B0E941A
:10E86400FD7B08950E945F63EBE3EA930C94D66208
:10E87400E89423F8E0E0F0E0FBDEE0E0E0931E083B
:10E884000A93E1E0EA930C94D52CE89423F8E0E0B1
:10E89400F0E0EEDEE0E0E0931E08EA930C94AA2B8D
:10E8A400E0911208ABE0EA9FF0010895A881B981D4
:10E8B400EC91EF5FEC930895ABE00A9FF001E35213
:10E8C400FA4F0895A083ABE00A9FF0010895ABE0EE
:10E8D4000A9FF001E152FA4F0895E4E9F7E1FA934F
:10E8E400EA93EA85ABE0EA9FF0010895AC81BD812B
:10E8F400EE27A00FBE1F0895E02FAC81BD81F0E08C
:10E9040008950E94FD7B84E00E946D6B2896089513
:10E91400EE27A30FBE1FEC91D001EC930895A2E55E
:10E92400B7E00C94DC6C0E94FD7AEA0FFB1FAF0188
:10E934000895E0912D0CF0912E0C0895E32FA091F1
:10E944001E08EA0F0895ADE02A9FF001E35FFC4F33
:10E954000895A8E0B0E00E94187C0895F0E0FA93CE
:10E96400EA9308950E9449420C941842F0E00E94F0
:10E97400FD7A08950E94FD7B0E9433420C94184254
:10E984000E944942E9EBF7E1D6CB0E9418420C946D
:10E99400184220E030E0E12FE05DEA93ECEBF7E190
:10E9A400A0CBEAE0EA930C94B762E4E4FBE0FA93C8
:10E9B400EA93089510915D0500915F0508950E9402
:10E9C400D8423E2F0C94BD45EAE0F0E00E94467B1D
:10E9D4000895DF01EE27A30FBE1F0895EF81F88588
:10E9E400FA93EA930895F0E0EA0FFB1F0895E02FED
:10E9F400A0E0B2E0BBCFEA0FFB1F3296E49108958A
:10EA0400FA93EA93E0911C0CEA930E943938E132BC
:10EA14000895EA930E94DF37E1320895E6E0F0E0DA
:10EA24000C94826C0E947A46ABE9BBE0EE27A10FFE
:10EA3400BE1FEC91E1700895EE0FFF1F0C94526D10
:10EA4400EA930E943938E13208950E94440D0C94EF
:10EA5400566CEAE3EA930C9414460E94FD7B0C94F2
:10EA64002141E3E7EA930C941446EA23EA930E94D3
:10EA74004841BAC8EA930E944841B6C8DF013296B9
:10EA840079C80E94FB7AE854FF4F0895E2E4F6E067
:10EA9400E0933B0CF0933C0C08950E942A1AE0E0AA
:10EAA400E09321080E9469150E94440DE1E0E0937F
:10EAB4001B0808950E94A1460E94E40F0E94D842B8
:10EAC4000E2F0D330895EE81FF81FA93EA93089592
:10EAD400E5E0F0E0FA93EA930895EAE2EA93E4E6E3
:10EAE400F8E10895EA930E94B9150C94440DE0935B
:10EAF400C105F093C2050895FE01FA93EA930895BF
:10EB0400ECE7F8E1FA93EA93EE85FF856889798961
:10EB1400F8CEE0E8F8E1FA93EA93AE85BF858889F8
:10EB240099896DCE0E94FD7BAA89BB898C899D89B8
:10EB3400E4E6F0E060E070E00E94B57B0E94FD7BBB
:10EB440088E00E946D6B2C960895E9E8F8E1FA9349
:10EB5400EA93EE85FF8581CE84E00E946D6B289652
:10EB6400CBCFFA93EA93EE85FF8508950E94BC63A8
:10EB74000C94816884E00E946D6B28960895EE27BA
:10EB8400A10FBE1FEC910895EA930E94B3411F5F49
:10EB94000895E091C405A7ECB5E0F0E00895AF5FF7
:10EBA400EAE00E94A07B0895E091C305A7ECB5E0DC
:10EBB400F0E0CACBA0E0A083E981ADE0EA9FF001D8
:10EBC4000895EF73A5E1EA9FF001E051FB4F08952A
:10EBD400EF73ABE0EA9FF001EC5EFB4F0895AC816C
:10EBE400BD81EE27A30FBE1FAC91A0300895ABE00A
:10EBF4000A9FF001EC5EFB4F0895EA0FFB1F0F0123
:10EC0400AC81BD8185CEA5E10A9FF001E051FB4FA7
:10EC14000895EE81FF8101801280AE81BF81159637
:10EC24000E94EA7BD0010895FE013896FA93EA9394
:10EC34000895EAA5FBA5FA93EA930895FA93EA9353
:10EC4400FE013A96FA93EA930E942B6930E0E02F92
:10EC54000895E091C105F091C2050895A1ECB5E0D5
:10EC6400ED91FD913296FE93EE930895AE81BF81AE
:10EC7400EA17FB070895E0E0E0936505E093660575
:10EC840008951A930A933A932A930895FA93EA9368
:10EC9400E0910E040895A0910003B091010308953A
:10ECA400E0910003F0910103FA93EA93E0910203E7
:10ECB400F0910303FA93EA930895E0930003F09329
:10ECC40001030895A981BA815ACFF801AA81BB81B1
:10ECD400EA0FFB1FE4910895AE0FBF1FAC91A03063
:10ECE4000895D801F0E0AE17BF070895AE0FBF1F17
:10ECF400EC91EA930895EFEEF0E0EA1BFB0B089524
:10ED0400A0910E04E4E1EA9FF0012E2F3327C8CF2F
:10ED1400E0E0EA930E94904B0E94D57D0895ECE0D8
:10ED2400EA9FF001A0910D04EA9FF00108951A935F
:10ED3400E1E0E0930E04E0930D0410E00895ED810A
:10ED4400FE81FA93EA930895EF81F885EA1BFB0BA1
:10ED54000895EA9FF001F0E008953A932A935A93B4
:10ED64004A930895EAA5FBA5E20FF31FFA93EA93E9
:10ED74000895ECA1EA930C94F34B3A932A93EEA1F1
:10ED8400FFA1E40FF51F0895FA93EA93EBCFEAA5E8
:10ED9400FBA5E40FF51FFA93EA93EBCFE20FF31F01
:10EDA400FA93EA930895FA93EA935A934A93089547
:10EDB400EA9FF001AEA1BFA1F0E00895E2E0E09384
:10EDC4000E04E0E2F0E0EAA3FBA30895AE1BBF0B40
:10EDD400A4CAEE8DF0E00895E20FF31F3196FA9382
:10EDE400EA93ECA1FDA1E40FF51F31960C94986E03
:10EDF400ECA1FDA1E40FF51F0C94986EE9A1F0E0DD
:10EE0400DE0116960895ED8DEA930E94CA45E9A1A4
:10EE1400EF5FE9A30895ED8BFE8BAB89BC897DCAB6
:10EE2400A98DBA8DEA0FFB1FE98FFA8FEB89FC8954
:10EE3400AF89B88DEA0FFB1FEF8BF88FED89FE8940
:10EE4400AD89BE890E94467B0E94087B0E94A37CF8
:10EE5400EE87FF87688B798BEB89FC89AB89BC894A
:10EE64000E94467B0E94087B0E94A37CAE85BF85DE
:10EE7400888999890E94797DEA87FB876C877D87D9
:10EE840000E010E00895F8010E94087B0E94A37C32
:10EE9400EE83FF8368877987AE81BF8188859985F2
:10EEA4000E942B7DAA85BB858C859D850E942B7D28
:10EEB400AE85BF85888999890E94077C0E94D67C8B
:10EEC4000E946C7CAF015A934A930C94946BE98D25
:10EED400FA8DE21BF30BFA93EA930895E98DFA8D08
:10EEE400E01BF10BFA93EA930895F901AD8DBE8D01
:10EEF4000C94526DED8DFE8DE01BF10BFA93EA93A9
:10EF0400EA8DEA930C94F34BAD8DBE8D0C94526D47
:10EF1400EFE3F1E0EA1BFB0B0895EB81FC81AF8189
:10EF2400B8850895E00DF11DFA93EA930E94054A0D
:10EF3400E5E3EA930895E09365000C94346F0E942E
:10EF4400CC7DEE81EA930E94344A8F010895E985CD
:10EF5400FA85AD85BE8508950E944E4AEB85FC85F1
:10EF6400FA93EA930C94664AED85FE85A985BA85E1
:10EF7400AE17BF070895EB85FC85AF81B885AE1742
:10EF8400BF070895AD85BE85E985FA85EA1BFB0BAD
:10EF94000895FA93EA930C942F6CAB85BC85D4CE78
:10EFA400AF81B885EB85FC85EA1BFB0B0895D9017D
:10EFB4000E94467B0F010895D0010E94717BAF012E
:10EFC400FA01AD85BE850C94526DED85FE85E21B7C
:10EFD400F30BFA93EA930895AD85BE850C94526DB4
:10EFE400A985BA85ED85FE85EA1BFB0B0895E881AA
:10EFF400F981FA93EA9308955A934A93EE85FF852B
:10F00400B0CDFA93EA93EC85FD85FA93EA930E94D6
:10F01400D44CE0910E04AA85BB85E5CCD901F0E07F
:10F02400AE17BF070895E05CF54F44CAE091380C71
:10F03400A091370CEA170895E0911108ABE0EA9F1C
:10F04400F0010895E3E0EA930E944263F5CFE08182
:10F05400E05DEA930C94D662A091260CB091270C43
:10F064000895E2E5EA930E94D6620C94C54DF096A9
:10F07400EA930E94A163E2E7EA930C94D662EA93CE
:10F084000E94D662EEE0EA930C94D662ECE9F8E1D1
:10F09400CCCA0E940963EBE3EA930C94D662E0E3E2
:10F0A400EA930C94D662EBE3EA930C94D6625A93F7
:10F0B4004A930E9433180E2F00340895FA93EA936A
:10F0C4000C9465331A93E985FA85FA93EA930895C3
:10F0D400E552F84FA885B985A083B183E1CBE2E579
:10F0E400EA930C94D6621A93E0913908E0531E2FE8
:10F0F400EDE3F8E0B4CAE0911208A0911308EA170E
:10F104000895E3E1F8E0DACFE0911308ABE0EA9F79
:10F11400F0010895A091750B42CDE093750BEAE2DE
:10F12400EA930E94A163DBCFE091750BE05AA7CF6D
:10F13400D9011696EC9112CCF901A281B381BA934C
:10F14400AA9308950E940963EAE3EA930C94D662B1
:10F15400D9011196E0E0EC930E94BC63D2CFD901AF
:10F16400EC91FCCBE05DEA930C94D662E05DEA930B
:10F174000E94A163B4CFEA58F44F69CFEEE0EA935A
:10F184000C94D662EAE3EA930E94D662F9010895E8
:10F19400E093610CF093620CE2E0E0933608D9014D
:10F1A4001196EC930895EA930E94A16398CF0E946C
:10F1B4000963DCCCE0911A0CD9CFE0911A0CF0E091
:10F1C400DACFFA93EA9365CF0E940963ECE2EA93FB
:10F1D4000E94D6620CCF37DAAC91A0330895A09187
:10F1E4005E0BB0915F0B0895EE81FF81E093280CD4
:10F1F400F093290C1093250C0E94F71BE1E308956A
:10F2040041E050E00E940962E887F987EAE3EA9363
:10F214000E947C61E13008951A93E985FA85C3CD93
:10F22400E2E2EA930E947C61E03008950CDAAC914A
:10F23400A032089508DAAC91AB33089504DAEC9166
:10F24400EA930895EAE3EA930C947C610E940962CC
:10F254003197E887F987E88508950E94EA7BE40FEF
:10F26400F51FD001ED93FC930895E091400BF0E07D
:10F27400ED55F94F0895E0E0E093660CE093670CD8
:10F2840008950E9409623197E093400BE091590B75
:10F29400A091400BEA1708950E94C456E091400BD8
:10F2A400EA930895ECE2EA930E947C61E0300895C9
:10F2B400EC5BF44F0F01C7D9EC91D001EC931F5FC5
:10F2C400B8CAEC5BF44FA0E0A0830895EA930E94CF
:10F2D4007C61E1300895E091410B85CBE091410BD5
:10F2E400EF5FE093410B0895A4EABBE0E091410B8A
:10F2F400F0E00C94A671ABE9BBE0E091410B0C94F7
:10F304001470E091410BF0E00895E2E2EA930C946A
:10F31400D662FA93EA930C943A53E091400BF0E0EE
:10F32400B0CBFA93EA930C9409630E940963ECE26C
:10F33400EA930C94D662ECE2EA930C94D6620E94AF
:10F344002F53E0E0E093410B0895E091410B0C94BE
:10F354001470E091600BF091610B0895AEE5BBE091
:10F364000C94C16E3CDFEC93F9CFE0E0EA930E9489
:10F374009353E09335080895AA81BB81EC91E295FB
:10F38400E07FAE2FEC810895EA0FAA81BB81EC9354
:10F394008DCAE091070DA091060DEA170895E0913A
:10F3A4003B09F0E0E05CF64F08951083E0913B09DF
:10F3B400EF5FE0933B09E12FA0913D090895E093AD
:10F3C4003D09E0913C09E150E0933C09E0300895A7
:10F3D400E05CF64FA0E0A0830895E091D20DF09197
:10F3E400D30D0895A091D00DB091D10DEA17FB076C
:10F3F4000895E12FA091D70DEA0FE093D70DE09186
:10F40400D90D0895F0E0E85CF74F10830895E0917A
:10F41400DE0EF0E0E352F24FE081E0939C00E091D5
:10F42400DE0EEF5FE093DE0E08950DD9AC91AA33A2
:10F4340008950F0108D9EC91E0530C944072EA93BB
:10F444000E94D6621F5F0895EAE4F9E1FA93EA9311
:10F454000895FE013196FA93EA930895E881EA93B8
:10F464000C94D662E881F9816A817B810E94FD7BDC
:10F474000895E05CF54FE081E0300895EA930E943E
:10F484007068EA930C947C5EEA930E941065EAE546
:10F49400E0933E090895EA930E94BD66E030089522
:10F4A400E0E0EA930C94E266EA930E94FF66E0309F
:10F4B4000895E0917100E87F1E2F0895E093730092
:10F4C400E4E8F2CF0A930E94D666E0300895FF275D
:10F4D400662777270E94A37C0895EE8DAE85BF85AD
:10F4E40088899989F4DF0E942B7DA9A1BAA1882774
:10F4F40099270E94047C0E94077C0E94D67C089570
:10F504000E94077C0E94D67C0895FA93EA93E2E174
:10F51400F0E0FA93EA9308952A93ED89FE89FA9329
:10F52400EA93FE017596FA93EA930C948469EE8942
:10F53400FF893497EE8BFF8B0895ED89FE89FA934A
:10F54400EA93FE017596FA93EA930C948469AE8962
:10F55400BF8914960E94EA7BEE83FF83B4CAE885D0
:10F56400F9856A857B85AC85BD858E859F850895E3
:10F574000E94AB6BE883F9836A837B830895E881F7
:10F58400F9816A817B810895EA81FB816C817D81A7
:10F594000895E991F991309639F080EA9FE0019756
:10F5A400F1F7A8953197C9F708950024AF0DB01D60
:10F5B4000895EA0FFB1F681F791F0895EA1BFB0BD0
:10F5C400680B790B0895F195E195F0400895F09555
:10F5D40060957095E195FF4F6F4F7F4F0895EE232F
:10F5E4000E2EEA2F19F0EE0F0A94E9F70895EE0FA4
:10F5F400FF1FEE0FFF1FEE0FFF1FEE0FFF1F0895FB
:10F60400FE2FFF0FFF0B6F2F7F2F08956F2F660FB5
:10F61400660B762F0895BA2FBB0FBB0B8B2F9B2F36
:10F6240008958B2F880F880B982F0895EA17FB07EE
:10F63400E1E00CF0EE270895FA9FF02DEB9FF00D1A
:10F64400EA9FE02DF10D08957A9F702D6B9F700D48
:10F65400F89F700DE99F700D6A9F602D710DFB9FDF
:10F66400600D711DE89F600D711D8827FA9FF02DB4
:10F67400610D781FEB9FF00D611D781FEA9FE02D4F
:10F68400F10D681F781F089582D0D6DF0EF49BDF3A
:10F6940008958BD0D9DF0EF49ADF0895002498E002
:10F6A400AA0F001C0E1A10F40E0E01C0A1609A9548
:10F6B400B9F7EA2FA02D08950024112490E1AA0F90
:10F6C400BB1F001C111C0E1A1F0A18F40E0E1F1E5D
:10F6D40001C0A1609A9599F7FD01D001089557D012
:10F6E400EBDF0EF470DF08953F934F935F93002494
:10F6F40011244427552730E2AA0FBB1F881F991FE6
:10F70400001C111C441F551F0E1A1F0A460B570BD1
:10F7140028F40E0E1F1E461F571F01C0A1603A9504
:10F7240059F7FD01BC01D001CA015F914F913F918E
:10F7340008953BD0D9DF0EF44ADF0895AFDFEA2FF6
:10F744000895E894B7FF04C0A095B0951196689405
:10F75400F7FD39DFB1DFFD010EF435DF0895C4DFB5
:10F76400FD01BC010895E89497FF09C0A095B095E8
:10F7740080959095AF5FBF4F8F4F9F4F689477FDF3
:10F7840026DFB2DFFD01BC010EF421DF0895E89409
:10F79400F7FF02C018DF6894B7FF06C0A095B095C4
:10F7A400119600F8039400FA0895E89477FF02C0D4
:10F7B4000EDF689497FF0BC00024A095B095809548
:10F7C40090951196801D901D00F8039400FA0895F9
:10F7D400ED91FC9111970895ED91FD916D917C91BE
:10F7E40013970895ED93FD936D937C93089505907D
:10F7F400F491E02D08957A936A93FA93EA93089525
:10F80400689401C0E89401D09DD0182E862F612DF4
:10F81400192E972F712D1B2EBF2FF12D1A2EAE2FBF
:10F82400E12D0895119602D0FE2F1197E199FECF94
:10F83400FF93FFB7F894AEBBBFBBE09AEDB3FFBF35
:10F84400FF91089507D01196EF93EF2F03D0EF9116
:10F8540011970895E19B02C0A895FCCF9FB7F89437
:10F86400AEBBBFBBE09A8DB3E81719F0EDBBE29ACB
:10F87400E19A9FBF0895552342F4503811F4E0FFF4
:10F8840004C03196691F791F6BF050E8572711F4B3
:10F894005F93CDC05F3F31F0660F000C57956795BD
:10F8A400752F08955F9300200AF0CDC0C6C050E8BC
:10F8B400192E1522880F991F9527550F879550E803
:10F8C400072E0522660F771F7527550F6795089534
:10F8D400689401C0E8945F93F2DF703818F07F3FBA
:10F8E40008F4A5C056E1571BAAF4519558300EF4FC
:10F8F400593030F0EFEFFFEF6FEF7FE777F91AC081
:10F9040077275523B9F0EE0FFF1F661F771F5A950F
:10F91400D1F710C07727583028F0EF2FF62F672F34
:10F924005850F9CF552331F076956795F795E795BB
:10F934005A95D1F700200AF44ADE5F91089568943D
:10F9440001C0E894309760407040B1F0002426F084
:10F95400772312F400943BDE172E7EE1112032F05F
:10F964007A95EE0FFF1F661F111CF9CFEF2FF62FAC
:10F97400612D5F938ADF5F9108954F93AF01FD017D
:10F98400DA01AB01BC01CA01402D012C142E4F91A8
:10F994000895EA0FFB1F681F0895E095F0956095A0
:10F9A400EF5FFF4F6F4F08955F9381DF903871F1E0
:10F9B40050E8152604C05F937ADF903839F1703827
:10F9C40021F1572F591B13F112F4D7DFFACF583115
:10F9D40018F0AA27BB278827583028F0AB2FB82F58
:10F9E40088275850F9CF552329F08695B795A795C0
:10F9F4005A95D9F7502D512562F0CBDF38F467952D
:10FA0400F795E795739513F41EC0B7DF3EDF5F915A
:10FA14000895EA1BFB0B680B51F010F40094BDDF52
:10FA24006623A2F3EE0FFF1F661F7A95CBF7EE272E
:10FA3400FF27662777275F910895EFEFFFEF6FE7C2
:10FA44007FEF5F910895EFEFFFEF6FE77FE75F913F
:10FA540008955F932CDF703851F3903841F30124FB
:10FA64000894791F23F41CF300203AF3ECCF0F928F
:10FA74001F932F933F934F93112722279927689F12
:10FA8400A0018F9F302D410D591F6B9F300D411DDB
:10FA9400591F8E9F27D0BF9F25D06A9F23D0BE9F1A
:10FAA4001DD0AF9F1BD0AE9F110D291F391F491FB9
:10FAB400591FE32FF42F652F522F4F913F912F9110
:10FAC4001F910F9066232AF0550FEE1FFF1F661F2C
:10FAD40002C073954BF2CFDE5F910895100D211D86
:10FAE400391F02C0200D311D491F591F08955F930E
:10FAF400DEDE703821F411200AF49FCFA4CF9038B1
:10FB040009F495CF01240894970B1BF4D4F3002037
:10FB1400F3CF792F1F932F933F934F9311241127E2
:10FB2400222733274427552790E2AE17BF078607BD
:10FB3400410730F0AE1BBF0B860B410B089401C08C
:10FB44008894551F221F331F111CAA1FBB1F881F17
:10FB5400441F9A9551F7F901612D4F913F912F91CF
:10FB64001F91662332F0550FEE1FFF1F661F7A9513
:10FB740043F281DE5F9108953097604070400895AC
:10FB840000240A160B06089500240A160B0608061C
:10FB9400090608955A934A933A932A931A930A9317
:10FBA40008955D814C813B812A81198108810895E2
:00000001FF
